:100000000C942E280C942E280C942E280C942E2818
:100010000C942E280C94C40E0C94C6110C94F31658
:100020000C942E280C942E280C942E280C942E28F8
:100030000C942E280C942E280C942E280C942E28E8
:100040000C94B60E0C942E280C942E280C942E286A
:100050000C942E280C942E280C942E280C942E28C8
:100060000C942E280C942E280C94790D0C942E2888
:100070000C942E280C942E280C949A0C0C94BB0CE7
:100080000C942E280C942E280C942E28000000008E
:100090003D3D3D3D3D3D3D3D3D3D3D3D3D3D3D3D90
:1000A000205A582045766F20536572766963652023
:1000B0003D3D3D3D3D3D3D3D3D3D3D3D3D3D3D3D70
:1000C000202020202020202020205A582045766FF4
:1000D0006C7574696F6E20546573742653657276FF
:1000E000696365200000160F18687474703A2F2F2A
:1000F0007777772E4E65646F50432E636F6D2F00B8
:10010000040126010D0A0A8FE0AEA2A5E0AAA020F4
:10011000A2EBA2AEA4AEA22041544D4547413132DC
:10012000382E2E2E20000D0A0A41544D45474131EC
:1001300032382070696E7320636865636B2E2E2ED3
:10014000200046015E018FE0AEA1ABA5AC20ADA5BD
:1001500020AEA1ADA0E0E3A6A5ADAE2E00004E6F8F
:100160002070726F626C656D7320666F756E642EA1
:10017000000076019C010D0A8EA1ADA0E0E3A6A5CA
:10018000ADA020AFE0AEA1ABA5ACA020ADA020AF4C
:10019000AEE0E2E3282DA0E5293A20000D0A4861EF
:1001A000766520612070726F626C656D20617420CD
:1001B000706F72742873293A200050417820000033
:1001C00050427820000050437820000050443520F1
:1001D000000050457820000050467820000050472D
:1001E00078200000E80102020D0A8FE0AEA3E0A033
:1001F000ACACA020AEE1E2A0ADAEA2ABA5ADA0211B
:1002000000000D0A50726F6772616D20697320687B
:10021000616C74656421000020022E0221022F020D
:100220000A0D91AEE1E2AEEFADA8A52000000A0DE7
:10023000537461747573206F66200000504F5745EA
:1002400052474F4F443D00002C20564343353D005C
:10025000540270020D0A82AAABEEE7A5ADA8A52054
:10026000AFA8E2A0ADA8EF204154582E2E2E0A00D0
:100270000D0A41545820706F7765722075702E2ECC
:100280002E0A00008802AC020D0A87A0A3E0E3A7B3
:10029000AAA020AAAEADE4A8A3E3E0A0E6A8A82007
:1002A000A220465047412E2E2E2000000D0A5365F5
:1002B00074204650474120636F6E666967757261AE
:1002C00074696F6E2E2E2E200000CE02DA0287A0F7
:1002D000A2A5E0E8A5ADAE2E0000446F6E652E002D
:1002E000E40204030D0A8FE0AEA2A5E0AAA020AAB2
:1002F000ABA0A2A8A0E2E3E0EB2050532F322E2EB9
:100300002E0D0A000D0A50532F32206B6579626F53
:1003100061726420636865636B2E2E2E0D0A0000E7
:1003200024033603202E2E2EADA5E220AEE2A2A598
:10033000E2A00D0A0000202E2E2E6E6F2072657333
:10034000706F6E73650D0A004C036403202E2E2E11
:10035000ADA5AEA6A8A4A0A5ACEBA920AEE2A2A52F
:10036000E20D0A00202E2E2E756E77616E74656484
:1003700020726573706F6E73650D0A0080039803B9
:10038000202E2E2EE1A1AEA920AFE0A820AFA5E03F
:10039000A5A4A0E7A50D0A00202E2E2E6661696C8B
:1003A00020746F207472616E736D69740D0A0000A1
:1003B00006031C079FF07425E80345107C172A12DA
:1003C0006518BF242309F11DC4C4C4C4C4C4C4C473
:1003D000C4C4C4C4C4C4C4C4C4C4C4C4C4C4C4C4DD
:1003E000C4C492A5E1E220AAABA0A2A8A0E2E3E0E7
:1003F000EB2050532F3220202020202092A5E1E234
:1004000020AAABA0A2A8A0E2E3E0EB205A5820A8C3
:1004100020A4E02E202092A5E1E220ACEBE8A82069
:1004200020202020202020202020202020202020CC
:1004300092A5E1E220424545502F544150454F5589
:10044000542F434F564F5820202092A5E1E220A27E
:10045000A8A4A5AE2020202020202020202020207D
:100460002020202084A8A0A3ADAEE1E2A8AAA0206D
:1004700053442F4D4D4320202020202020208FE06A
:10048000AEA3E0A0ACACA8E0AEA2A0ADA8A520466B
:100490006C6173682D524F4DC4C4C4C4C4C4C4C479
:1004A000C4C4C4C4C4C4C4C4C4C4C4C4C4C4C4C40C
:1004B000C4C450532F32206B6579626F617264201F
:1004C0007465737420202020202020205A58206B2F
:1004D0006579626F617264207465737420616E6403
:1004E0002065746320204D6F757365207465737487
:1004F00020202020202020202020202020202020FC
:10050000424545502F544150454F55542F434F5667
:100510004F582074657374202020566964656F20DD
:10052000746573742020202020202020202020208B
:100530002020202053442F4D4D4320646961676E75
:100540006F737469632020202020202020205772A0
:1005500069746520466C6173682D524F4D202020D0
:1005600020202020202020206C05300616050E8E2D
:10057000E1ADAEA2ADEBA520AAABA0A2A8E8A82051
:10058000E3AFE0A0A2ABA5ADA8EF3A16050F3C186B
:100590003E2C203C193E1605103C456E7465723E9B
:1005A000202D202284A0222C20A2EBA1AEE0160553
:1005B000113C4573633E202D20228DA5E2222C2084
:1005C000AEE2ACA5ADA02C20A2EBE5AEA4201605B2
:1005D0001283AEE0EFE7A8A520AAABA0A2A8E8A8E6
:1005E0002028E2AEABECAAAE20A220ACA5ADEE294D
:1005F0003A201605133C5363726F6C6C4C6F636B3F
:100600003E202D20E0A5A6A8AC2054562F564741E9
:100610001605143C436170734C6F636B3E202D20B4
:10062000EFA7EBAA20A8ADE2A5E0E4A5A9E1A00010
:1006300016050E55736167653A16050F3C183E2C7A
:10064000203C193E1605103C456E7465723E202D07
:100650002022596573222C2073656C65637416051E
:10066000113C4573633E202D20224E6F222C2063C7
:10067000616E63656C2C20657869742016051248DC
:100680006F742D6B6579732028696E206D656E75AA
:10069000206F6E6C79293A201605133C5363726FF4
:1006A0006C6C4C6F636B3E202D20746F67676C65BC
:1006B0002054562F564741206D6F64651605143C33
:1006C000436170734C6F636B3E202D206C616E67CD
:1006D000756167652073776974636800E0060807D1
:1006E000161A0A83E6160A0C3C183E2C203C193ECA
:1006F000202D20A8A7ACA5ADA5ADA8A520E7A0E119
:10070000E2AEE2EB150F0000161A0A487A160E0C3C
:100710003C183E2C203C193E202D206672657175D8
:10072000656E6365150F00002C074807160E078AD3
:10073000ABA0A2A8A0E2E3E0A0205A5816230784A9
:10074000A6AEA9E1E2A8AA00160F075A58204B65E9
:1007500079626F6172641623074A6F7973746963F3
:100760006B00160B0931203220332034203520361F
:100770002037203820392030160B0A5120572045C9
:1007800020522054205920552049204F2050160B2C
:100790000B4120532044204620472048204A204B2C
:1007A000204C2065160B0C63205A205820432056FD
:1007B0002042204E204D2073207316260A1816243E
:1007C0000B1B2046201A16260C19160E0F536F66A7
:1007D000745265736574161E0F547572626F4B65A3
:1007E000790016050765202020312032203320347F
:1007F0002035203620372038203920302031203253
:100800002020702073207020200720072007160565
:100810000960203120322033203420352036203723
:10082000203820392030202D203D201B2020692019
:1008300068207520206E202F202A202D16050A748E
:10084000205120572045205220542059205520491E
:10085000204F2050205B205D205C202064206520FC
:10086000642020372038203916050B63204120539F
:100870002044204620472048204A204B204C203B43
:100880002027202020652020202020202020203408
:1008900020352036202B16050C73205A2058204373
:1008A00020562042204E204D202C202E202F20206C
:1008B00020202073202020201820202020312032CA
:1008C000203316050D632077206120202020202072
:1008D000207320202020202020612077206D20639D
:1008E00020201B2019201A2020302020202E2065B7
:1008F00016051052617720646174613A16040F0086
:100900000409340916051392E0F1E5AAE0A0E2AD6E
:10091000AEA520ADA0A6A0E2A8A5203C4553433E2D
:10092000202D20A2EBE5AEA420A8A720E2A5E1E2BD
:10093000A02E0000160A135072657373203C4553B5
:10094000433E2074687265652074696D6573207418
:100950006F20657869742E005C0974090D0A92A5F0
:10096000E1E2A8E0AEA2A0ADA8A520ACEBE8A82EDD
:100970002E2E20000D0A4D6F7573652074657374FB
:100980002E2E2E2000008A09A0098EA1ADA0E0E342
:10099000A6A5ADA8A520ACEBE8A82E2E2E20200001
:1009A000446574656374696E67206D6F7573652E39
:1009B0002E2E20200000BA09C8098DA0E1E2E0AE89
:1009C000A9AAA02E2E2E2000437573746F6D697A2C
:1009D0006174696F6E2E2E2E2000DE09E8098FAE3D
:1009E000A5E5A0ABA82100004C6574277320676FB4
:1009F0002100F609100A2020202020208DA5E220C9
:100A0000AEE2A2A5E2A020AEE220ACEBE8A82E0068
:100A10002020202020204E6F206D6F75736520727E
:100A20006573706F6E73652E00002E0A4E0A2020CB
:100A30002088ACA5EEE2E1EF20ADA5AAAEE2AEE0E3
:100A4000EBA520AFE0AEA1ABA5ACEB2E00002020C3
:100A5000202054686572652061726520736F6D6532
:100A60002070726F626C656D732E0000700A900AC0
:100A700020203C456E7465723E202D20AFA5E0A578
:100A8000A7A0AFE3E1E2A8E2EC20E2A5E1E22E00BC
:100A900020202020203C456E7465723E202D20725F
:100AA00065737461727420746573742E0000B20AE9
:100AB000EE0A1623122092A5E1E2204452414D2075
:100AC0001620138FE0AEA2A5A4A5ADAE20E6A8AA7D
:100AD000ABAEA2162014A1A5A720AEE8A8A1AEAA8D
:100AE000162015E120AEE8A8A1AAA0ACA800162304
:100AF00012204452414D2074657374201620134C0B
:100B00006F6F707316201450617373162015466151
:100B1000696C0000180B240B16170C90E3E1E1AA96
:100B2000A8A9000016170C456E676C697368000071
:100B3000340B760B16020282EBE5AEA4160203829A
:100B4000E1F120E1ADAEA2A016020491E2A5E0A57C
:100B5000E2EC20AC2FE1E52E16020584AEA1A0A2A6
:100B60002EA7A0A4A0ADA8A516020682EBAFAEAB3F
:100B7000ADA8E2EC20001602024578697420160246
:100B800003526574726965766520616C6C2016028B
:100B9000044572617365206368697020160205411F
:100BA0006464206A6F621602064578656375746531
:100BB000206A6F627300BA0BCA0B159F208DA5E2E5
:100BC00020E4A0A9ABAEA2200000159F20204E6F0C
:100BD0002066696C657320200000DE0B020C160293
:100BE0000A159E97E2A5ADA8A520466C617368150D
:100BF0009F16020B3C4553433E202D20A2EBE5AE51
:100C0000A40016020A159E5265616420466C617349
:100C1000682E2E2E159F16020B3C4553433E202D69
:100C20002065786974002A0C3E0C16020B159F880B
:100C3000ADA8E62E534420AAA0E0E2EB0000160285
:100C40000B159F53446361726420696E69742E2092
:100C50000000560C660C208DA5E220534420AAA06B
:100C6000E0E2EB21200020204E6F2053442D6361F1
:100C70007264212020007A0C8A0C208EE8A8A1AA98
:100C8000A020E7E22E205344200020534420726528
:100C90006164206572726F7220009E0CAE0C202081
:100CA000208DA5E22046415420212020200020460E
:100CB0004154206E6F20666F756E64212000C20C57
:100CC000D20C20208EE8A8A1AAA0204641542021C1
:100CD00020002020464154206572726F722021202E
:100CE0002000E60CF60C208E2C20A3ABEEAAA0ADC3
:100CF000E3ABAE21200020477265617420676C6908
:100D00007463682120000A0D1E0D16020C159E202A
:100D100093A2A5E0A5AD3F203C593E20000016025D
:100D20000C159E596F7520737572653F203C593EB6
:100D30000000360D4A0D16020C159E91E2A8E0A0A7
:100D4000ADA8A52E2E2E2020000016020C159E45C3
:100D5000726173652E2E2E20202020200000620D4F
:100D6000760D16020C159E87A0AFA8E1EC2E2E2E54
:100D700020202020000016020C159E577269746511
:100D80002E2E2E202020202000008E0DA20D1602D7
:100D90000C159E8FE0AEA2A5E0AAA02E2E2E20203C
:100DA000000016020C159E5665726966792E2E2E6D
:100DB000202020200000BA0DCE0D16020C159E87B3
:100DC000A0A2A5E0E8A5ADAE2E20202000001602CE
:100DD0000C159E436F6D706C6574652E202020206D
:100DE0000000E60D060E160D0687A0AFA8E1EC2068
:100DF000A220466C617368524F4D20A7A0A2A5E0C7
:100E0000E8A5ADA000001612064A6F6228732920DB
:100E1000636F6D706C657465642E0000200E300E7B
:100E2000161507A1A5A720AEE8A8A1AEAA2E00001E
:100E30001611074E6F206572726F727320646574AD
:100E400065637465642E00004C0E5C0E161507E198
:100E500020AEE8A8A1AAA0ACA8210000160E075356
:100E60006F6D65206572726F7273206172652064A8
:100E7000657465637465642100007E0E8C0E20200D
:100E80002084A0E2E7A8AAA83A200000202020534E
:100E9000656E736F72733A2000009E0EB20E2020B2
:100EA0002020208DA5E220AAA0E0E2EB2020202037
:100EB00020002020202020204E6F206361726420BB
:100EC000202020202000CA0EDE0E208AA0E0E2A012
:100ED00020E3E1E2A0ADAEA2ABA5ADA020002020B2
:100EE000204361726420696E7365727465642020AA
:100EF0002000F60E0A0F202087A0E9A8E2A020AE6D
:100F0000E220A7A0AFA8E1A82000202020202052A6
:100F1000656164206F6E6C79202020202000220FF4
:100F2000360F202087A0AFA8E1EC20E0A0A7E0A525
:100F3000E8A5ADA0200020202057726974652065C7
:100F40006E61626C6564202020004E0F680F88ADD2
:100F5000A8E6A8A0ABA8A7A0E6A8EF20AAA0E0E278
:100F6000AEE7AAA82E2E2E004361726420696E6936
:100F70007469616C697A6174696F6E2E2E2E00003F
:100F8000840FA00F53442F4D4D4320AAA0E0E2A0B0
:100F900020ADA520AEA1ADA0E0E3A6A5ADA02E009A
:100FA0004E6F2053442F4D4D432063617264206681
:100FB0006F756E642E00BA0FCE0F8EA1ADA0E0E368
:100FC000A6A5ADA020AAA0E0E2A03A200000466FAE
:100FD000756E6420636172643A200000E00F1610A1
:100FE00016100B8DA0E7A0E2EC20A4A8A0A3ADAE44
:100FF000E1E2A8AAE320160C0C5B205D208FAEA4D2
:10100000E0AEA1ADEBA920AEE2E7F1E220A22052D2
:10101000532D3233320016110B53746172742064F5
:101020006961676E6F7374696320160C0C5B205DD9
:101030002044657461696C6564206C6F6720746F0F
:101040002052532D323332004C105C108EA1ADA0D3
:10105000E0E3A6A5ADA0204641540000466F756EA2
:101060006420464154006A1084108FAEA8E1AA2083
:10107000E4A0A9ABAEA2AEA920E1A8E1E2A5ACEB49
:101080002E2E2E00446574656374696E67206F664A
:101090002066696C652073797374656D2E2E2E0041
:1010A000A410BE1097E2A5ADA8A520E2A5E1E2AE8E
:1010B000A2AEA3AE20E4A0A9ABA02E2E2E005265B6
:1010C0006164696E67206F66207465737420666959
:1010D0006C652E2E2E00DA10F21084A8A0A3ADAEFF
:1010E000E1E2A8AAA020A7A0A2A5E0E8A5ADA02EB5
:1010F0000000446961676E6F7374696320697320CF
:10110000636F6D706C6574652E000D0A6F757420C9
:1011100000002C20696E20000D0A3B434D44000066
:101120000D0A3B41434D443431000D0A43532075B1
:1011300070000D0A435320646F776E004D4D4300DD
:1011400053442076310053442076322B205374616F
:101150006E64617264204361706163697479000038
:1011600053442076322B20486967682043617061C0
:101170006369747900004F43523A20004353443A64
:1011800020004349443A20004D616E7566616374E6
:101190007572657220494420202020004F454D2F54
:1011A0004170706C69636174696F6E2049442000FE
:1011B00050726F64756374206E616D65202020200D
:1011C0002020200050726F64756374207265766908
:1011D00073696F6E2020200050726F6475637420F5
:1011E00073657269616C2023202020004D616E754B
:1011F000666163747572696E67206461746520004E
:101200002E3230002E3139004352433D00000D0A8A
:101210003B5265616420736563746F7220000D0A30
:101220003B353132206F7065726174696F6E732067
:10123000697320736B69706564000A0A20049F015A
:1012400000023516DF0064974C7F44600E94D01482
:10125000A0E0B1E00E94801600E21FE725E30E94B3
:10126000BF16EAE3F2E10E94F414ECEDFFE00E9405
:101270008D16FB8A99D206D30E94750FE1F30537CC
:10128000C1F3023749F00A3549F011FDF4CF0637B2
:1012900091F7477F64960895EB8AECCF0B89002382
:1012A00019F008E04027E6CF4A7F4260DBD2DAD26D
:1012B000E0ECF0E00E9476140E944D14D3D2466018
:1012C000E1D2E0E4F2E10E94F414A1E0B3E0BB8BD0
:1012D0000E948016C7D2EAE4FFE00E947114F092E7
:1012E0002501FA8AA9D212EA0FEF0E94E71610E24E
:1012F0000E94FE16ACD211EA0FEF0E94E7162FEF04
:1013000000E080D2EEECF1E30E9413172A9531F44D
:10131000AED2E0E8FFE00E9471143AC2013081F7DA
:1013200008E070D2E4EDF1E30E94131780E002FFC1
:1013300080E4898B14E00E94FE1673D207E70E94B6
:10134000031712E00E94FE1609E60E945B17098946
:101350000E945B170E940A17002379F002FFEDCF6D
:1013600001E050D201E40E9403170023C9F742D2E2
:1013700038D210E1ECE3F1E11DC03CD232D211E0F1
:10138000E0E4F1E109890023A9F00AE33BD20AE78E
:101390000E940317DE0126E00E945A170D932A953A
:1013A000D9F712E0E6E4F1E1088106FF03C016E098
:1013B000E0E6F1E1109325011A8BEF93FF9357D2EA
:1013C000E6EBFFE00E947114FF91EF910E9476140A
:1013D0001A8911FF0CC04BD2E6E7F1E10E947614A6
:1013E000DE0124E00D910E94C6142A95D9F711EA76
:1013F0000FEF0E94E71609E005D209E40E940317E7
:101400000023B9F40E941A170F3F99F0DE0121E181
:101410000E945A170D932A95D9F729D2ECE7F1E1EA
:101420000E947614DE012FE00D910E94C6142A95C9
:10143000D9F711EA0FEF0E94E7160AE0E3D10AE4B8
:101440000E940317002321F40E941A170F3F09F48A
:101450009FC1DE0121E10E945A170D932A95D9F709
:1014600006D2E2E8F1E10E947614DE012FE00D9150
:101470000E94C6142A95D9F7FAD1E8E8F1E10E9452
:10148000761408810E948814F2D1ECE9F1E10E94FF
:1014900076143A89098134FF0E94CC1434FD0E94ED
:1014A00088140A8134FF0E94CC1434FD0E948814F1
:1014B000DED1E0EBF1E10E947614DE01139625E027
:1014C00034FD26E00D910E9491142A95D9F7CFD1D1
:1014D000E4ECF1E10E947614088534FD098502955B
:1014E0000E948C140EE20E949114088534FD098537
:1014F0000E948C14BCD1E8EDF1E10E947614DE016B
:10150000199634FD119624E00D910E9488142A95B5
:10151000D9F7ADD1ECEEF1E10E9476140E8534FDE1
:1015200002950F700E947C14E0E0F2E10E8534FD1C
:101530000CC01D85007F1F70012B02950F930E9428
:1015400076140F910E947C140CC00F70035018F495
:101550000C59E4E0F2E10F930E9476140F910E947F
:101560007C1485D1E6E6F0E10E9471141DB710935A
:1015700004011EB710930501C0930601D093070123
:10158000E5EAFBE0E0935B01F0935C0111EA0FEF09
:101590000E94E7160E943619AF93BF938F939F93D3
:1015A00066D1E8E4F0E10E9471141091260102E195
:1015B000112321F006E11A9509F002E30E94881434
:1015C0009F918F91BF91AF9180E090E00E94D61AD9
:1015D00007C00196B096F83019F40E94D61A01F5AA
:1015E0001081153EB1F31123D9F00385087D89F7E9
:1015F000EF93DF01E2E2F6E10591002331F01D9166
:101600000117D1F3FB2FEF91E4CFFB2FEF91848DE6
:10161000958DA68DB78D082F092B0A2B0B2B39F42E
:10162000B7C05445535446494C4542494E006FEFAC
:1016300071E00E94CB1B8C839D830E94A91B0197A4
:10164000AF09BF09009128010A950823039500936B
:101650005501009128010E94B21B8093560190937E
:101660005701A0935801B0935901F0925001828D17
:10167000938DA489B5898093510190935201A093D1
:101680005301B0935401F3D0E0EAF0E10E947114E9
:10169000F092030102E0C02E14E50E94E7160E94BA
:1016A000F7250E94DA1B002331F1E0E0F4E0A0E02E
:1016B000B2E00E94292600910301002391F3F092E9
:1016C0000301AEE1BB89BB8B0E9480164F934C7F18
:1016D0004460009159010E948814009158010E94B1
:1016E0008814009157010E948814009156010E94AD
:1016F00088144F91D6CFE0E0F4E0AC81BD81B170A9
:1017000011960E9429260E941C26CC24002714E54D
:101710000E94E716AEE1BB89BB8B0E94801600E2F7
:1017200028E00E94C416A3D0E8E0F2E10E947614FB
:101730000B810E9488140A810E94881409810E94EA
:10174000881408810E94881423C0F8941091040121
:101750001DBF109105011EBFC0910601D091070168
:1017600078940F9384D00F91E2E5FCE0013071F0A2
:10177000E6E7FCE0023051F0EAE9FCE0033031F04A
:10178000EEEBFCE0043011F0E2EEFCE00E9471149C
:101790006ED0E6EDF0E10E9471144C7F446072D08F
:1017A0000E94750FE1F350CD2227B22FB55FABE059
:1017B0000E9480162F930B891FE9201709F410EF60
:1017C0002EE10E94C9162F912395223071F7ADE0CA
:1017D000BCE00E94801600E243FD0BEF0E94BA16A7
:1017E000089500E10FD0EAEDF1E30E941317002302
:1017F000C1F708950BE306D00BE70E9403170023FF
:10180000C9F7089543FF08954F934A7F42600F93AD
:10181000E8E1F1E10E9476140F910E947C144F914F
:10182000089543FF08954F934A7F4260E0E2F1E15B
:101830000E9476144F91089543FF08954F934A7F75
:101840004260EAE2F1E10E9476144F91089543FF6D
:1018500008954F934A7F4260E2E3F1E10E947614DB
:101860004F910895EBD043FF08950BE3A8C0A1E08A
:10187000BB89B395BB8B0E948016E0D043FF0895CF
:101880000BE39DC0A0E0B1E00E9480161FE70E941C
:101890007D16EAE7FEE00E9471141AE7EAE9FEE02D
:1018A000B59903C01CE7E6ECFEE00E947D160E949D
:1018B00071141AE7E2EFFEE0B49903C01CE7EEE111
:1018C000FFE00E947D160E947114089510D018E068
:1018D00010939A004D7F416008950DE001D00AE019
:1018E00000909B0005FEFCCF00939C000895F092B1
:1018F000980015E010939900F0929B001EE0109361
:101900009D000895F4DF18E910939A004E7F42601D
:1019100010E01093080110930901F0920A0110E8F9
:1019200010930B0110930C01F0920D0195988D9A74
:10193000BE9808951F931FB71F930F9300919C00AB
:1019400010910D01103890F4AF93BF93B3E0A091C4
:101950000B010D93AF77A068A0930B01BF91AF91DE
:10196000139510930D01103708F0959A0F911F9160
:101970001FBF1F9118951F931FB71F9310910A0146
:101980001123A1F0AF93BF930F93B3E0A09109018E
:101990000D9100939C00AF77A060A09309011A9568
:1019A00010930A010F91BF91AF9105C010919A0059
:1019B0001F7D10939A001F911FBF1F9118951F93B1
:1019C000AF93BF9310910A011038E0F7B3E0A091F4
:1019D00008010D93F89410910A01139510930A01D0
:1019E0007894AF77A060A093080110919A0015FD3C
:1019F00003C0106210939A00BF91AF911F91089598
:101A00001F9310910D011123B9F0AF93BF93B3E071
:101A1000A0910C010D91F89410910D011A9510935D
:101A20000D0178941F3608F49598AF77A068A093BD
:101A30000C019894BF91AF911F9108950DE0BFDF05
:101A40000AE0BDCF4F93427F4260EF93FF93E6E9F8
:101A5000FAE14CD7FF91EF91A0E0B0E0EFDF0B2F60
:101A600057D70A2F55D700E2AADFA9DFEF93FF93DC
:101A700080E101918BD78A95E1F700E2A0DFFF9129
:101A8000EF9180E1019188D78A95E1F75096B230C5
:101A900029F74F9108950D0A3B20202020202E3059
:101AA000202E31202E32202E33202E34202E352091
:101AB0002E36202E37202E38202E39202E41202E53
:101AC00042202E43202E44202E45202E460010E09A
:101AD00010938B0019E010938A001BE2109387008B
:101AE00012E31093860010917D00106110937D0029
:101AF00008951F931FB71F9310910E011395109314
:101B00000E0129F410910F01139510930F011F91ED
:101B10001FBF1F911895AF93BF93F894A0910E012A
:101B2000B0910F017894A80FB91FB068A083B1835A
:101B3000BF91AF9108959F93918197FF12C08F93AA
:101B40008081AF93BF93F894A0910E01B0910F01E3
:101B50007894A81BB90BB6FD07C0F182BF91AF9175
:101B60008F919F9108940895BF91AF918F919F910C
:101B7000889408951127939A000000000000000047
:101B80000000000000000000839B116093988B9A76
:101B900000000000839912608B98112361F0BF9AB6
:101BA0000E94C025C79A00FDC798A0E0BCE6A150DE
:101BB000B040E9F7F5CF0E94660C8FDE8EDE8DDE39
:101BC000E0ECF0E00E9476140E944D14E0E0F1E0B9
:101BD0000E94711415E51BBB1AEA1ABB12E818BB68
:101BE00015E017BB15E115BB1AE014BB959A8D984B
:101BF000189A10981998119A15E1109365001AE037
:101C00001093640084E191E00197F1F7002719B384
:101C1000153509F0016016B31778103809F0026025
:101C200013B31F71153109F00460859B086011B171
:101C30001370113009F00061109163001F711531AC
:101C400009F000621AEA1BBB15E51ABB15E018BBC8
:101C500012E817BB1AE015BB15E114BB95988D9AD5
:101C60001898109A199A11981AE01093650015E1C6
:101C70001093640084E191E00197F1F719B31A3AE7
:101C800009F0016016B31778153009F0026013B33C
:101C90001F711A3009F004608599086011B1137042
:101CA000123009F00061109163001F711A3009F0C1
:101CB0000062002329F4E2E4F1E00E947114089527
:101CC0000F930E94DC25E2E7F1E00E9471140F916E
:101CD00006950F9320F4EAEBF1E00E9476140F9141
:101CE00006950F9320F4E0ECF1E00E9476140F913A
:101CF00006950F9320F4E6ECF1E00E9476140F9124
:101D000006950F9320F4ECECF1E00E9476140F910D
:101D100006950F9320F4E2EDF1E00E9476140F9106
:101D200006950F9320F4E8EDF1E00E9476140F91F0
:101D3000069520F4EEEDF1E00E947614E4EEF1E079
:101D40000E9471140E94DC25FFCF1AB712601ABFDF
:101D500019B7106119BF12E013BFF0921501F0928C
:101D60001001F0921401F092160108958E98969A3F
:101D70001F931FB71F9317B71E7F17BF1F911FBF5A
:101D80001F9114981C9A18951F931FB71F932F9398
:101D90000F9300911101209110011091150117FD71
:101DA00064C0293081F02A30A0F4222329F48699D6
:101DB00059C01E7F239580C00695869B02C000688F
:101DC0001E25239579C086991E2510FF4BC02395AB
:101DD00073C0869B47C020931201009313011C9887
:101DE000149A20E822BF21E026BF27B7216027BF31
:101DF000209114012223D1F4013E51F10A3A89F1D4
:101E00000B3A01F10E3E69F10A3F59F10E3F49F1DB
:101E1000003E41F0003F41F010681093160100931E
:101E200017011FC012601EC014601CC02A952093A9
:101E30001401C1F4009117010E37A1F416E81093B4
:101E400016010FC0F092170121E02093140109C080
:101E500012E8109316010EE70093170127E0209374
:101E6000140111270027222727C02930A1F02A308A
:101E7000E1F02B30F0F4222319F4116023951CC0FB
:101E8000079528F48E98969A1E25239515C0969846
:101E90008E9A239511C010FD04C096988E9A2395B2
:101EA0000BC08E98969A239507C08E98969A239584
:101EB00003C018E00027222720931001009311018E
:101EC000109315010F912F911F911FBF1F9118950E
:101ED0000E94C0251091160117FFFACFF09216014B
:101EE00012FDF6CF0091170108950E94C0251091B0
:101EF000160117FF08C0F092160112FD04C00091F0
:101F0000170198940895189408958E98969A17B783
:101F10001E7F17BF14981C9A11270C9BF6CF1A9599
:101F2000E1F7F8941C98149A96988E9A00931101F0
:101F300010E810931501F0921001F0921401F09244
:101F40001601F0921201789484E191E00197F1F783
:101F500096988E9A86E695E00197F1F7E8E1F1E030
:101F60008FE090E00E948B0D14981C9A109115013F
:101F7000187041F4E8E1F1E00E949B0DB8F78E98EB
:101F8000969A18940895F0921201E8E1F1E084E144
:101F900090E00E948B0D10911201112341F4E8E1B1
:101FA000F1E00E949B0DB8F7002718940895009166
:101FB00013010895219714981C9AE0EEF2E091D451
:101FC000F0921201E8E1F1E084EF91E00E948B0DC4
:101FD00010911201112331F4E8E1F1E00E949B0D10
:101FE000B8F703C000911301D1D40FEF31D0F092B4
:101FF0001201E8E1F1E088EE93E00E948B0D109170
:102000001201112339F4E8E1F1E00E949B0DB8F7C9
:1020100036D006C000911301B9D40A3A09F02CD089
:1020200002EF16D029F40BEA1CD011F403E819D002
:1020300000EF0ED011F402E00BD003EF09D031F421
:1020400000E006D0EBEDF1E50E94761421960895AC
:102050009DD45BDF71F097DF91F098D40A3F61F473
:102060000895088390DF59F091D41881011721F465
:102070000895ECE7F3E005C0E8E4F3E002C0E0E235
:10208000F3E00E947114989408952597FB82E8E488
:10209000F2E20E94F414E0E0F9E03FD610E81C837D
:1020A000E2EEF7E03FD604EC2DE26ED6E0E1F8E098
:1020B000F292EE23E9F7F0921201F88200911201F8
:1020C000002319F00091130171D00C8107FF15C096
:1020D00007700C830DEE6AD018DF79F054DF69F0D9
:1020E00065D00A3F51F40C8161D00FDF31F04BDF36
:1020F00021F05CD00A3F09F492D01091160117FF2D
:10210000DDCFF09216010091170119832B8112FF88
:102110000CC011FD09C0063739F423952B832330F9
:1021200020F0DFD525960895FB8211FD17C012FD22
:1021300011C0AC81B1E00E3711F4AB27A068BB0F22
:10214000073711F4AB27A068BB0F083511F4AB2794
:10215000A068AC83033811F4A8E410C0043811F46B
:10216000A8E70CC0003808F5000F11FD0160EEE48F
:10217000F2E2E00FFF1DA491AA23B9F0BA2FB770C5
:10218000BB2309F0B395A695A695AE73A43208F0CB
:10219000A395AE3108F0A395AD5FB95FB1D50981C4
:1021A0001EEA02FD11ED21E0F4D588CF0F93F092E5
:1021B0001201E881F8E00193EF70E8834C7FA5E01D
:1021C000B1E19ED5E881E3952DE02A83F8E0E3951F
:1021D000EF70E98300810F931EE0003E61F0013E45
:1021E00051F01DE0003F39F01BE00D3E21F01AE0F8
:1021F000053808F41FE081D500E2BCD50F912A8193
:10220000222329F085D3E9812A812A95DECF4260F5
:102210000E94881400E20E9491140F910895A9E28F
:10222000B7E06ED50C811CED01FF10ED22E0B1D5B9
:102230000C811CED02FF10ED22E0ABD50C811CEDF2
:1022400000FF10ED22E0A5C503052F10DF010000FF
:10225000580000003800280018002000700000001E
:1022600060005000400030000A000900000000003B
:102270001D5D0C0000000D75120011000000000033
:10228000000014001B0013001A00190000150000C4
:1022900024001C002300220029002100006500000A
:1022A0003D002C002B0032002A003100006D0000A0
:1022B0003C0034003B0033003A00390000000000CD
:1022C00000004400430042004100490000000000BB
:1022D0004C004B004A005200590051000000000021
:1022E00054005C9953005B005A006100000000003C
:1022F00000006300000062006900000000000B00A5
:10230000740073AD6A00000072000000000000005D
:10231000000000000000000000007100000000004C
:1023200094820000937D9281000000000000957966
:10233000A57A9C859B00A38D9A8408009100680073
:10234000AB00A48AA900A178A28980880000162584
:102350000F576865656C203D16250C4C2020204DDC
:10236000202020521625115820203D1625125920D4
:10237000203D000016040A15DF0003022F13DF01C1
:10238000090A2204AF01230A0D0ADF001F931FB7B9
:102390001F932F930F9300911B0120911A0110910D
:1023A0001E0117FD22C0293081F02A30A0F422231B
:1023B00029F4879917C01E7F239540C00695879BF7
:1023C00002C000681E25239539C087991E2510FF7D
:1023D00009C0239533C0879B05C020931C0100933F
:1023E0001D0111270027222729C02930A1F02A30FA
:1023F000E1F02B30F0F4222319F4116023951EC074
:10240000079528F48F98979A1E25239517C09798BB
:102410008F9A239513C010FD04C097988F9A239527
:102420000DC08F98979A239509C08F98979A2395F6
:1024300005C01127879B12E00027222720931A014D
:1024400000931B0110931E010F912F911F911FBF2D
:102450001F9118954B7F4260E8E5F9E00E947114E6
:1024600044602A97F8948F98979A15981D9A1AB7EE
:1024700018601ABF19B7106219BFF0921E01F092CE
:102480001A01F0921C017894EAE7F3E20E94F41436
:10249000A4E0B3E035D4D2DAE6E8F9E00E947114A2
:1024A000A4E0B4E02DD4CADAF0921C01EFE1F1E02F
:1024B00082E090E00E948B0D10911C011123A1F786
:1024C000EFE1F1E00E949B0DB8F70FEF5FD29FD1D3
:1024D000B9F0CBD1A9F05AD20A3F91F4F0921C0185
:1024E000EFE1F1E088EE93E00E948B0D10911C016A
:1024F000112339F4EFE1F1E00E949B0DB8F76EC0B3
:1025000070C000911D0142D20A3AC9F700E05CD0C8
:10251000A4E0B5E0F5D392DAE6EBF9E00E9471149D
:10252000A4E0B6E0EDD38ADA03EF45D008EC43D05F
:1025300003EF41D004E63FD003EF3DD000E53BD0B0
:10254000A4E0B7E0DDD37ADA02EF35D0F0921C01D7
:10255000EFE1F1E084E190E00E948B0D10911C010D
:10256000112331F4EFE1F1E00E949B0DB8F736C082
:1025700000911D0109870AD2002319F0033009F0E8
:102580002DC0A4E0B8E0BCD359DA08EE14D002E0C4
:1025900012D006EE10D003EF0ED004E60CD004EFFC
:1025A0000AD0A4E0B9E0ACD349DAEAEDF9E00E9440
:1025B000711444DA4EC0EAD12AD171F056D161F0DB
:1025C000E5D10A3F49F408950B834FD129F0DED1BC
:1025D0001B81011709F40895FF91EF91EAE2FAE0F7
:1025E00002C0E2EFF9E0EF93FF9328DAE0E8F3E2CC
:1025F0000E94F414AAE0BBE083D3FF91EF910E9404
:102600007114AAE0BCE07CD3ECE6FAE00E947114FD
:102610000E94680F063719F00A35D1F723CF00E082
:10262000C02E14E50E94E716002710EAD0D3002739
:102630001DEACDD300271EEACAD3F8948F98979A43
:1026400015981D9A19B71F7D19BF789442602A9674
:1026500008954C7F02E0C02E14E50E94E716E6E8DC
:10266000F3E20E94F414E8E5F3E21985112311F076
:10267000EEE4F3E257D316E91C83FD8218E71E83CC
:10268000FF82F886F0921C011985112331F0ADE22A
:10269000BFE036D30F810E948C14A9E2B1E130D3A0
:1026A000AC81BD810E949B14A9E2B2E129D3AE8125
:1026B000BB270E949B14BBE0BF93A4E221D31FED74
:1026C000088500FD1EEA23E064D31FED21E061D3FD
:1026D0001FED088502FD1EEA23E05BD31FED21E01C
:1026E00058D31FED088501FD1EEA23E052D3BF91A8
:1026F000B395BE3008F3009103010023B9F0F092C6
:102700000301AC81BD81D196D196AF930B2F10EA16
:102710005ED30F911DEA5BD3AE81BB279C96AF932E
:102720000B2F10EA54D30F911EEA51D30E94750F5C
:1027300019F0063709F473CF00911C010023D9F278
:10274000F0921C0100911D0103FFD5CF08838DD0AD
:1027500091F209838AD079F20A831985112319F03D
:1027600084D049F20B83088107700887AC81BD8152
:1027700089819927188114FD08C0A80FBF1DAE33A9
:10278000BE0550F0ADE3B1E007C080950196A81BEF
:10279000B90B10F4AA27BB27AC83BD83AE81BB273E
:1027A0008A819927188115FF0AC080950196A80F84
:1027B000B91FBB2311F4AA3F30F0A9EF04C0A81B36
:1027C000BF0908F4AA27AE831985112329F00B81CC
:1027D000AF81A00FAF70AF83E4E7F3E2A3D2426012
:1027E000088196D000E29DD0098192D000E299D074
:1027F0000A818ED000E295D01985112321F00B813A
:1028000087D000E28ED000E28CD04C7F3DCF1127E4
:102810000D9BFDCF1A95E1F7F89400931B0110E88A
:1028200010931E01F0921A01F0921C011D98159A46
:10283000789487E691E00197F1F797988F9A89E469
:102840008A95F1F7EFE1F1E08FE090E00E948B0DC7
:1028500015981D9A10911E01127031F4EFE1F1E00C
:102860000E949B0DB8F718940895F0921C01EFE1B7
:10287000F1E087E090E00E948B0D10911C01112384
:1028800039F4EFE1F1E00E949B0DB8F71894089538
:1028900000911D01F0921C010895ECEFFFEDEBBEDD
:1028A000A791B6910A2F0F71D9F01B2FAA0F111FF4
:1028B000AA0F111FAA0F111F1F7091F01D3080F475
:1028C0002B2F26952F73293058F00F9308E229D02B
:1028D000022F12D0012F10D00F910ED009E221D07B
:1028E0000895EB0DFF1D85919591FC010591002345
:1028F00011F017D0FBCF0895005D07FF0053085E6D
:1029000006FF0851045F05FF0C500A5F04FF0650E4
:102910000F93029501D00F910F700A3008F0095FF4
:10292000005D40FD0E94700C41FD0E94DF0C42FDE5
:102930000E94BA160895E4E8F9E224E000278591A0
:102940009591A81BB90B10F00395FBCFA80FB91FE9
:10295000002321F400E20AD0002703C0006306D060
:1029600000E32A9561F70A2F0063DBCFEF93FF9313
:10297000AF93BF932F93D5DF2F91BF91AF91FF916D
:10298000EF9108951027E80364000A000F93C0DF59
:1029900000E2C7DF0F910895003208F40EE2C1CFC4
:1029A000A0E0B1E0ADD117E783EC94E006C2A0E06F
:1029B000B0E0A6D100E210EF25E3E1D100EB17E78C
:1029C00083EC94E0F0D100E210EF25E3D8D14C7F06
:1029D0004460A0E0B0E094D1E0ECF0E0A3D10E942C
:1029E0004D14E6EEF0E09EC12897A591A883B5911D
:1029F000B98315911A8312501B8315911C831250B1
:102A00001D8315911E8315911F837AD11E8175D167
:102A10000AEDB0D104EC2B81B7D10FEBABD1A8817B
:102A2000B981B395B9836CD11E8167D103EBA2D173
:102A300000E22B81A9D103EB9DD12F8120FF03C0A0
:102A400011E021E0A6D12D812A952D8341F7A8819F
:102A5000B981B395B98354D11E814FD100EC8AD18D
:102A600004EC2B8191D109ED85D12F8120FF03C08A
:102A700011E021E08ED12F8120FF08C0A881A3950D
:102A8000B981B3953DD111E02A8183D11E8135D121
:102A9000289608956197EA83FB83FC82F98287DF99
:102AA000EA81FB81A591AD83B591BE83BF8315916A
:102AB0001887159119871A8715911B8715911C87FF
:102AC00015911D8715911E8715911F871591188BDC
:102AD0001985110FE10FFF1D088502501985139507
:102AE000019F1B2D169521F0E00DF11D1A95E1F7C0
:102AF00007D11B8502D10AED3DD104EC3BD12885DD
:102B000022502FD104EC36D10FEB34D1AD81BF81EF
:102B1000B395BF83F5D01B85F0D003EB2BD100E23A
:102B200029D1288522501DD100E224D103EB22D1E6
:102B300011E021E02ED12A852A952A8739F7AD8127
:102B4000BF81B395BF83DCD01B85D7D000EC12D1F9
:102B500004EC288519D109ED0DD111E021E019D13E
:102B6000AD81A395BF81B395CBD011E028852E5FB1
:102B700010D1ED85FE8500E00995AD81A395BE815C
:102B8000B3951C81B10FBCD01C85288502D10E9451
:102B9000750FC1F00A3559F10537B1F10237E9F186
:102BA0000D37F1F00C36E1F00A37D9F00936C9F0EB
:102BB00011FD08C00637C9F00835A1F00E3799F0AD
:102BC000053091F0FE010E949B0D08F7ED85FE8512
:102BD00001E00995FE018F8598890E948B0DD7CF62
:102BE00027C02BC03EC067C02EC061960895D8DEB6
:102BF000EA81FB813A961C81110FE10FFF1DA5911F
:102C0000B591FD0109954ACF1C81112309F4BFCF6D
:102C10005FD01C811A951C83B0CF1C8109850A9551
:102C2000101708F0B4CF54D01C8113951C83A5CF86
:102C30001C814ED011271C83A0CF1C8149D019853F
:102C40001A951C839ACFACDEEAE5FCE2CDDEE8E61D
:102C5000F5E063D00E94680F21CF030D2509CF0155
:102C600022960B2D0E5F043008F00027B02E06953B
:102C700082E090E00E94ED2593DEE0EBFCE2B4DE22
:102C80001EE93BD0E4E1FBE048D02297FE0180ED55
:102C900097E00E948B0DFE010E949B0D38F00E9470
:102CA000750FC9F311FD02C00835D1F22296F6CE98
:102CB0000D0B1B039F01AE240A2D0E6F1FEA0E940D
:102CC000E7160A2D81E090E00E94ED250AD0E6CEBD
:102CD000AD81A395BE81B395B10F12D01B85288518
:102CE00058C00DEE12D941F04ED931F00A3F21F40F
:102CF0000A2D0095017009D90895012F1AEA67C0BD
:102D000015E3B19FBB27A00DB11D1197B77018EA4D
:102D10000A2F5DD019EA0B2F5AC0EB0DFF1D8591CC
:102D20009591FC01C09A1CEA1FB958D00591002367
:102D300071F0053121F0063131F04ED0F7CF059119
:102D40001AEA45D0EFCFA591B591DADFEBCF089520
:102D5000C09A1CEA1FB942D001913ED02A95E1F7F2
:102D60000895C09A1CEA1FB939D0059135D02A952B
:102D7000E1F708951F931CEA2AD01F9108950F933D
:102D8000012F1AEA24D00F911CEA21D02A9531F4A0
:102D90000895012F1BEA1BD02A9521F0C098C09AF4
:102DA0002A95E1F708950F93012F1AEA10D00F9199
:102DB0001CEA0DD0019731F40895012F1BEA07D0CA
:102DC000019721F0C098C09A0197E1F708950F93F9
:102DD000C09A1FB903D00F91C0980FB9779BFECF4F
:102DE0000FB1C09A08953F933FB7C0FC0E94AD1841
:102DF000C1FCE09203013FBF3F9118950FEF5BD0FC
:102E00001A95E1F708950F9312E0F8DF0F9153D070
:102E1000002751D000274FD000274DD000274BD09E
:102E20000FEF49D007C012E0E9DF16E0059143D06B
:102E30001A95E1F710E20FEF3ED00F3F11F41A950B
:102E4000D1F708950091250102FD07C0880F991F51
:102E5000AA1FBA2FA92F982F88270FEF2CD001E592
:102E60002AD00B2F28D00A2F26D0092F24D0082FA4
:102E700022D00FEF20D08FEFDDDF8A95D1F00E3F0B
:102E8000D9F74F9343FF0AC0427F4260EF93FF930D
:102E9000EEE1F2E10E947614FF91EF9180E092E082
:102EA00009D001930197E1F74F9113E0A7DF9894C0
:102EB000089508950FEF43FF8FCF4F934A7F4260ED
:102EC000EF93FF930F93EAE0F1E110DD0F910F9381
:102ED0001FDD0F91C0980FB9779BFECF0FB1C09A3D
:102EE0000F93E2E1F1E102DD0F910F9311DD0F91FC
:102EF000FF91EF914F910895ECEAF0E375DDE2EB7D
:102F0000F0E372DDE8EBF0E36FDDEEEBF0E36CDDB8
:102F1000E4ECF0E369DDE8E2F7E0FFDEE2E6F7E0AB
:102F200001DFE0E3F8E0F292EE23E9F7FABADBBA68
:102F3000F4BAF5BAE0E0F8E0A09AA9D0A098A19A76
:102F4000A6D0A198A29AA3D0A298A39AA0D0A39801
:102F5000A49A9DD0A4980091630025E09DD003B36E
:102F6000001F001F001F22E097D0E0E0F8E0ABE078
:102F7000B9E0C6DE03817FD003857DD003897BD095
:102F8000038D79D003A177D004A175D0048D73D0BF
:102F9000048971D004856FD004816DD0ABE0BAE0B4
:102FA000AFDE028168D0028566D0028964D0028DCE
:102FB00062D002A160D005A15ED0058D5CD00589EC
:102FC0005AD0058558D0058156D0ABE0BBE098DEDD
:102FD000018151D001854FD001894DD0018D4BD059
:102FE00001A149D006A147D0068D45D0068943D01E
:102FF000068541D006813FD0ABE0BCE081DE008198
:103000003AD0008538D0008936D0008D34D000A168
:1030100032D007A130D0078D2ED007892CD007855C
:103020002AD0078128D0A6E2BAE06ADE03A523D021
:10303000A4E2BBE065DE01A51ED004A51CD000A55E
:103040001AD0A6E2BCE05CDE02A515D0AEE0BFE07F
:1030500057DE06A529E010D0AEE1BFE051DE05A5A0
:1030600028E00AD00E94750F11F0063709F062CFF0
:10307000F4BAF5BA089521E01FED037021F01EEABD
:10308000033009F011ED85DE1FED21E082CE00272F
:103090000A95F1F709B328E010811E7F079508F023
:1030A000136011932A95C1F7989408950706260C8A
:1030B000DF0109081706DF0022090905DF000C0EF1
:1030C0000D03DF001C0E0C03DF002197ECE8F1E399
:1030D0000E94F414ECEDF6E00E948D1601E014E578
:1030E0000E94E71607E00883A4E1BAE00E94801678
:1030F0000881000F000FE2E9F1E3E00FFF1DA59149
:10310000B591EF93FF930E949B14FF91EF9105916E
:10311000009323010591009324010FE713E50E941A
:10312000E71601E0C02E0E94680FCC24063779F024
:10313000053719F0023731F0F4CF08810E3088F7E7
:103140000395D1CF0881002361F30A95CCCF00E02D
:1031500014E50E94E716219608950F93EF93FF93CD
:10316000F0912101E091220100912301F00F0091E3
:103170002401E01FF0932101E0932201FFEF04916D
:103180000E94EC16FF91EF910F9108950808200618
:10319000DF014C00B5006B00000197006A01D6000A
:1031A00000022E01D402AB0100045C02A805560304
:1031B0000008B804500BAD0600107109A1165A0D95
:1031C0000020E212412DB41A0040C325825A40006B
:1031D0000000009548000001AA875000000200FF8F
:1031E000E0935B01F0935C0112EA0FEF0E94E71697
:1031F00010E204DE11EA0FEF0E94E7162FEFEEEC6B
:10320000F1E311DE2A9511F401E092C10130B9F722
:10321000E4EDF1E308DE80E002FF80E414E0EEDD9F
:1032200007E7F1DD12E0EADD09E645DE082F43DEBF
:10323000F1DD002351F002FFF3CF01E4E4DD0023D0
:10324000E1F747D14BD110E10FC043D147D111E095
:10325000882351F00AE7D7DD2DDE0F9315E0CEDD90
:103260000F9112E006FD16E010932501EDE5F1E067
:10327000D192D192D192D08280E090E0A0E0B0E0F3
:103280005CD132D111F003E053C1EEEB00810F7736
:10329000A1F4E2EC0081013051F0043041F006303D
:1032A00031F00B3021F00C3011F00E3031F4E6EC3F
:1032B00081919191A191B0812CC0E0E0F6E035853B
:1032C00000E010E028E037950F1D2A95E1F70A95F8
:1032D00009F4139506850784002909F013950389DD
:1032E0000488002909F4139500A101A0002902A077
:1032F000002903A0002909F413950589007F003FE8
:1033000009F41395143009F0BECF80E090E0A0E0FE
:10331000B0E08093330190933401A0933501B093D2
:1033200036010BD1E1D009F0AECFE0E0F6E0038545
:10333000002319F40485023011F004E0F9C0A0E084
:10334000B0E086899789092F082B21F484A195A1E3
:10335000A6A1B7A180932D0190932E01A0932F01D8
:10336000B0933001A0E0B0E083899489092F082B45
:1033700021F480A191A1A2A1B3A180933B019093DC
:103380003C01A0933D01B0933E0181899289A0E068
:10339000B0E0092F082B19F000E1E4D1DC01BF9364
:1033A000AF9300890093270180912D0190912E0108
:1033B000A0912F01B09130010A95880F991FAA1F83
:1033C000BB1F0A95D1F76F917F91E5D1668577850F
:1033D0006093310170933201DED180933701909375
:1033E0003801A0933901B0933A01EBE3F1E0BDD18C
:1033F000E0E0F6E00585013408F09FCF0093280156
:10340000B1D180933F0190934001A0934101B093CB
:10341000420102E0BB2359F4AA2349F4853F9D05EC
:1034200030F401E01FE0853F910708F400E00093CD
:10343000260180E090E0A0E0B0E0002331F00A95A2
:1034400021F084A595A5A6A5B7A580932901909301
:103450002A01A0932B01B0932C0180934B019093F0
:103460004C01A0934D01B0934E018F939F93AF9366
:10347000BF938091310190913201A0E0B0E0E3E38D
:10348000F1E080D18093430190934401A0934501E2
:10349000B0934601EDE2F1E075D18093470190933E
:1034A0004801A0934901B0934A01BF91AF919F9108
:1034B0008F9111E0082E092A0A2A0B2A39F01F934E
:1034C000C0D0ADD01F9110F41395F9CF10934F01D8
:1034D00008950BE798DC0023E1F70895EAEDF1E3A6
:1034E000A2DC0023D9F70895EEEFF7E0019105354E
:1034F000008109F40A3A089543FF14C04F93427FB4
:103500004260EEE0F2E10E9476140B2F0E948814D4
:103510000A2F0E948814092F0E948814082F0E94E5
:1035200088144F91E0E0F4E08DDC09F0089502E0AA
:10353000E0915B01F0915C010994EDE5F1E001910E
:10354000081749F40191091731F401910A1719F488
:1035500001910B1741F180935D0190935E01A0935F
:103560005F01B093600143FF14C04F93427F4260FC
:10357000EEE0F2E10E9476140B2F0E9488140A2FCD
:103580000E948814092F0E948814082F0E94881412
:103590004F91E0E0F6E056DC51F2E0E0F6E043FF68
:1035A00008950E94220DE0E0F6E008958F939F9326
:1035B00011EA0FEF0E94E716A0E0B0E000E1D2D0E0
:1035C0008F93009128010F93CDD000914F010A9560
:1035D000081738F40F910F919F918F910FEF0023EF
:1035E0000895A0914D01B0914E01082F00238091C4
:1035F0004B0190914C0129F00F9323D00F910A9524
:10360000D9F785D00F900A940F910021800F9F1D4C
:10361000AF1DBF1D92DF9F918F91002708951FE07E
:1036200000912601002319F4873F910708950A9518
:1036300019F4873F9D050895873F9D05AD05B107A6
:10364000089511EA0FEF0E94E7160091260100236A
:1036500039F10A9579F0880F991FAA1FBB1F082F0F
:10366000892F9A2FAB2FBB270AD03196A191B08119
:10367000BF700895A0E0B0E0082F892F99270F931D
:10368000AF93BF93E3E4F1E07DD057DFBF91AF91FB
:103690000F91E00FFF1DE00FFF1D819190810895B4
:1036A000FC01EE0FFF1FE80FF91FF695E795082FB5
:1036B0008F2F9927AA27BB2786950F93EF93FF9308
:1036C000E3E4F1E05FD08F939F9337DF9F918F9179
:1036D000BF91AF91B170EA0FFB1FA191F83031F4A7
:1036E000AF93A0E0B0E0019628DFAF910F919081F9
:1036F0008A2FA0E0B0E0069540F4969587959695C0
:10370000879596958795969587959F7008950B2F29
:103710000A2B092B082B59F4E7E4F1E080912D01E5
:1037200090912E01A0912F01B09130012BC00297F2
:10373000AF09BF090091280104C0880F991FAA1F73
:10374000BB1F0695D0F7E3E3F1E01CD0E7E3F1E01F
:1037500019C0892F9A2FAB2FB0E001E0B695A7953D
:10376000979587950795D0F708950191081B802FAD
:103770000191090B902F01910A0BA02F00810B0BD7
:10378000B02F08950191800F0191901F0191A01F0A
:103790000081B01F0895860F971FAF1DBF1D0895AC
:1037A000D8DFEDE2F1E0E1DF082F007F092B0A2BE3
:1037B0000B2B089511EA0FEF0E94E716E6E5F1E002
:1037C00001911191012B1191012B1191012BE1F12B
:1037D0008091510190915201A0915301B0915401F7
:1037E00096DF00915001800F9F1DAF1DBF1D84DE2D
:1037F0008091510190915201A0915301B0915401D7
:103800000091500103950093500110912801101769
:10381000C9F4F092500115DF809351019093520149
:10382000A0935301B0935401E6E5F1E0008101500B
:10383000019300810F09019300810F090193008119
:103840000F0901930FEF089580915101909152015A
:10385000A0915301B09154015ADF00915001800FA3
:103860009F1DAF1DBF1D48DE0091500103950093C1
:10387000500110915501011B0895E0936101F093EF
:103880006201E3E6F1E010E8118310E0128318E032
:103890001383D6820895E3E6F1E00081118162810D
:1038A0007381A481B5810680E0916101F09162018C
:1038B000002012F0C1F062C00790E0936101F09324
:1038C0006201E3E6F1E0F68200831183A483B5830D
:1038D000A62FB72F0D92B850B770B85FA283B383ED
:1038E000002D9894089592E08FEF110F11F4179125
:1038F000111F881FD0F79A9549F402E0859580F052
:103900000395839551F093E08FE3EFCF9A95B1F44F
:10391000869590F29395E9CF080F94E08FEFE5CF6D
:103920008395D1F49395879560F1991F110F11F448
:103930001791111FC0F7090F96E0D7CF9A9511F490
:1039400001E00BC09A9529F4839531F495E08FE15D
:10395000CCCF9A9509F7982F87919A95A82FB92FD0
:10396000A60FB71FB850B770B85F0D90E093610114
:10397000F0936201E3E6F1E0E682A6CF0A9591F7C3
:10398000B2CF18940895160209159F436869700014
:1039900049443A2000003A204D3239463034300054
:1039A0003A416D3239463034300016020A159F43D1
:1039B00052433A20000016020B5344636172643A8A
:1039C00020464154000016130E159F205BFB5D201E
:1039D00045726173652063686970200016010B15DC
:1039E000AE00000111079F00000811069F001101A1
:1039F000240D9F00000E350A9F000B041F06CF0107
:103A00000B041F06AF01202020203F3F3F3F202016
:103A10002000202020656D70747920202000A802ED
:103A2000990C7A782062617369633438200059D523
:103A3000915C7A7820626173696331323800E339CE
:103A40003CF274722D646F73202020202000446F9C
:103A5000D787616C636F676C756B70656E004845E6
:103A6000474C6865676C756B202020202000455608
:103A70004F4465766F646F732020202020001E6500
:103A80001EB361746D325F63706D20202000BCA492
:103A90002C297862696F732073746D6E7500272E00
:103AA00023687674722D646F732020202000203CE0
:103AB0004449523EB30042D000E949D017EA03E03E
:103AC00086D980E090E060E070D0E02F81E06DD09A
:103AD000F02F34C0E0E0F4E0A0E0B2E000810F3F5E
:103AE000E1F000EA34D017EA01E071D913EA082FB7
:103AF0006ED914EA092F6BD916EA008168D917EA42
:103B000005E065D901E068D903E066D916EA5FD916
:103B100063D91081012707FDFBCF319601961197DC
:103B2000E9F6089500E813D000E111D017EA03E0A8
:103B30004ED916EA4CD950D907FFFDCF00EF07D078
:103B400082E18A95F1F717EA03E041D908950F93CE
:103B500017EA01E03CD913EA05E539D914EA05E58D
:103B600036D916EA0AEA33D917EA05E030D901E076
:103B700033D913EA0AEA2BD914EA0AE228D916EA59
:103B800005E525D917EA05E022D901E025D913EA90
:103B900005E51DD914EA05E51AD90F9116EA17D9DA
:103BA00017EA05E014D901E017C915EA062F0FD965
:103BB00014EA092F0CD913EA082F09D916EA0FEFD6
:103BC00006C917EA0BE003D98827EFDF01C004D943
:103BD000019320230E94FC2501966F1D1197B9F7D0
:103BE000089566974C7FFB8AFC8A02E80D8BA0E063
:103BF000B8E020E200E80D931FE0FD921A95E9F786
:103C00002A95C1F7E2EEF9E30E94F414E8EEF9E335
:103C10000E94F414EEEEF9E30E94F414E4EFF9E3E9
:103C20000E94F414E0E3FBE00E948D16A7D40FE09D
:103C30000C8BE6E8F9E30E9492163DDFE13029F4AF
:103C4000F43A19F4E0EAF9E306C0E03239F4F23E5E
:103C500029F4E6E9F9E30E94921611C0EF93FF936D
:103C6000E0E9F9E30E949216FF91EF910E2F0E9476
:103C7000881400E20E9491140F2F0E948814EAED2C
:103C8000FBE00E948D16D98AFA8A3ED6B0D7222749
:103C9000992766272E839C836D83E6E0FAE3E09301
:103CA0006A01F0936B01E0E0FAE0A0E0B4E02FEFEE
:103CB00088DF20936C012497E6E9FAE0AFE6B1E0F3
:103CC000B9D7EEE1FAE313D621F1E9E0FAE0AFE289
:103CD000B0E0B0D7EEE2FAE30AD6D9F0E3E6FDE0D1
:103CE000A8E0B0E0A7D7EEE9FAE301D691F0E0E072
:103CF000FAE0A7E0B0E09ED7EEE8FAE3F8D549F0A5
:103D0000E0E0FAE0A8E3B0E095D7EEE7FAE3EFD51C
:103D100021F4E0936A01F0936B01249688279C813B
:103D20009C5F6D81A0E0B8E317EA0BE050D82091CA
:103D30006C013BDF01C050D820235ED7019611975C
:103D4000D1F720936C019C81945C6D81E0E0FAE0F6
:103D5000A0E0B4E036DFE2E1FAE3239521F4E0935A
:103D60006A01F0936B012497E8EFFDE00080118079
:103D700022803380EEE5FAE3BAD5B1F0EEE6FAE35D
:103D8000B6D591F0EFE2FBE0A9E0B2E053D7EEE464
:103D9000FAE3ADD549F0E2ECFCE0AEE2B1E04AD79F
:103DA000EEE3FAE3A4D521F4E0936A01F0936B010A
:103DB0002496E0916A01F0916B01A5E0B8E00E81D4
:103DC00010E1019FA00DB11D2BE005910D932A95E7
:103DD000E1F79AD50E94750F29F011FD03C006374F
:103DE00009F472C09C816D8110E4910F6F1D2E81CA
:103DF000239525FF4FCF20D7EAEAF9E30E949216D8
:103E00000B810E9488140A810E94881409810E94F3
:103E1000881408810E948814E6E2FCE00E948D1656
:103E20001DB7109304011EB710930501C09306013E
:103E3000D0930701E7E0F1E2D3D9AF93BF938F931B
:103E40009F93E6EBF9E30E9492166091260101E34D
:103E500012E3662329F016E36A9511F003E312E3F7
:103E60001F930E94BA160F910E94BA169F918F91CC
:103E7000BF91AF91A4D3DC861FD4FC860D890F714E
:103E80000D8B7CD30E94680F053741F0023779F023
:103E90000A35A1F00637B1F701E0F2CF0D8906959A
:103EA00088F31C89102309F4FACF0D8BE7CF0D8915
:103EB000000F40F31C891023C1F7FACF0D891C892C
:103EC000012301F3069510F466960895069508F40B
:103ED00089CE069508F4C5C1069528F40D890068B9
:103EE0000D8B4CD3E0C1069508F0CCCF0D8900684E
:103EF0000D8B44D3E6E0FDE00E948D160E94680F12
:103F000011FD02C0053351F0A2E0BCE00E94801612
:103F100000E21FE92DE00E94BF16B0CF1EE00E9414
:103F20007D160B8920E0069518F50F932F93220F2D
:103F3000220F2F9317D505E42CE00E94C4162F9171
:103F400023952F930FD505E42CE00E94C4162F91E2
:103F500023952F9307D505E42CE00E94C4162F91DA
:103F6000239500D505E42CE00E94C4162F910F91F3
:103F700023952830C1F6E2E3FDE00E948D160B89FF
:103F80000F3F11F4CFDD2DC06FEF63950695E8F775
:103F90000F936F9300E8DBDD15EA0F910F930E94FA
:103FA000E71600E3D4DD6F910F916395683068F4F4
:103FB0000695D8F70F936F9315EA062F0E94E71620
:103FC00000E3ECDD6F910F91F0CF17EA03E00E9460
:103FD000E71616EA0E94E7160E94EC1603FFFCCFD4
:103FE000A5DDEEE5FDE00E948D161AE00E947D162B
:103FF00020E02E83E0E0F8E010E1129FE00DF11DDB
:1040000080818F7311F0813208F055C08A8B992717
:10401000AA27BB27108116FD8096019700912801E1
:104020000A950823039500935501009128019ADB16
:104030008093560190935701A0935801B093590172
:10404000F092500181819281A381B48180935101CA
:1040500090935201A0935301B0935401108116FF25
:1040600006C020E22F93A6DB2F912A95D9F72E8147
:1040700079D499276E81669597956695979515EAF7
:10408000062F0E94E716A5E5B5E0AD87BE879F9392
:1040900091DB9F9188271EDDAD85BE85B25038F437
:1040A00007E50E94BA1615E5A10F15E0B11F1A89A0
:1040B0001A951A8B51F72E81239525FF9ACF3EDD55
:1040C00017EA03E00E94E716EAE8FDE00E948D1679
:1040D00020E02E83E0E0F8E010E1129FE00DF11DFA
:1040E00080818F7311F0813208F071C08A8B99271B
:1040F000AA27BB27108116FD809601970091280101
:104100000A950823039500935501009128012ADBA5
:104110008093560190935701A0935801B093590191
:10412000F092500181819281A381B48180935101E9
:1041300090935201A0935301B0935401108116FF44
:1041400006C020E22F9336DB2F912A95D9F72E81D6
:1041500009D499276E81669597956695979515EA86
:10416000062F0E94E716FF86F88AA5E5B5E0AD8721
:10417000BE879F931FDB9F918827E0E0F4E0A0E0DB
:10418000B2E017EA0BE00E94E71612DD02C00E94BF
:10419000EC161191011711F0EF86E88A019611973C
:1041A000B1F7AD85BE85B25070F40F851CE000FDFF
:1041B0001EEA0E947D1606E50E94BA16FF8615E5E6
:1041C000A10F15E0B11F1A891A951A8B81F62E815D
:1041D000239525FF7ECFE6EBFDE00E948D16EAEFEA
:1041E000F9E30889002311F0E0E0FAE30E94F414F7
:1041F000E2EEFDE00E948D16ECE1FEE0088911F090
:10420000E8E4FEE00E948D160E94680FEBCCF89463
:10421000109104011DBF109105011EBFC091060140
:10422000D091070178940F93ECEDF9E30E94921678
:104230000F91E2E5FCE0013071F0E6E7FCE00230CE
:1042400051F0EAE9FCE0033031F0EEEBFCE0043041
:1042500011F0E2EEFCE00E948D1607E00C8B02E00C
:104260000FCEA0E0B8E011E00B89012399F40B898F
:10427000012B0B8B24E0FD92FD92FD92FD92FD92AD
:10428000E2E1FAE38BE005910D938A95E1F72A9537
:1042900091F702C090969096110F30F70C8900614B
:1042A0000C8B32D3EBCD08D20E94680F0537D1F0CA
:1042B000023739F10D37A9F10A37D9F10C36A1F1DE
:1042C000093671F00A3569F0063771F7BC85BE5FB3
:1042D000A2E10E9480161FE922E20E94C916CECDFB
:1042E0003CC04BC00B850023F9F20A950B870C8567
:1042F000002319F00A950C8703C00A850A950A87DE
:10430000D2CF0B8519850395011770F60B870C85A5
:104310000A3018F403950C8703C00A8503950A87B1
:10432000C2CF0B850A5008F400270B870A87FC864A
:10433000BACF19851C3028F40AE00B87FA860C875F
:104340000BC00B85065F011710F0012F0A950B8734
:104350001AE01C87011B0A87A6CF19851C3028F498
:104360000AE00B87FA860C8707C0012F0A950B8796
:104370001AE01C87011B0A8796CF0B85E0E0FAE064
:1043800010E2019FE00DF11D0385002379F0828D7D
:10439000938DA489B58980934B0190934C01A09390
:1043A0004D01B0934E010BD1FC867DCFEF83F88792
:1043B000848D958DA68D0FEF1FE3800F911FAF1D8C
:1043C000990FAA1F990FAA1FAA8BF98ABC85BE5FF5
:1043D000A2E10E9480161FE122E20E94C91694D237
:1043E0000E94680F0537C9F00237E9F00B3639F043
:1043F000043759F00A3509F1063791F76DC009897C
:10440000002371F30A95098BEACF09891A89100FE5
:10441000103230F70395098BE2CF0989045008F474
:104420000027098BDCCF09891A89010F0C5F003244
:1044300008F000E2011B098BD2CFE0E0F8E0098927
:1044400010E1019FE00DF11DEC83FD831091280127
:1044500010935001EF81F885828D938DA489B589E1
:104460008093510190935201A0935301B093540152
:10447000848D958DA68DB78D6FEF71E08CD969D93C
:1044800020E2809730F129F18D879E8729D020E2A4
:104490002E83009150010A95A1F4809151019091D1
:1044A0005201A0915301B09154010E94211B8093AD
:1044B000510190935201A0935301B0935401009184
:1044C0002801009350012E812A9511F78D859E8534
:1044D000D7CF8096282F04D0D98AFA8A15D2CECC8D
:1044E0002F9311E0098906950695002319F0110F05
:1044F0000A95E9F70B890123D1F40B89012B0B8B6A
:10450000A0E0B8E009890C7110E1019FA00DB11D78
:1045100024E0FD92FD92FD92FD92FD92E2E1FAE32C
:104520001BE005910D931A95E1F72A9591F72F91CC
:104530000091280110915001011709F02064AC810D
:10454000BD812D93009151010D93009152010D9366
:10455000009153010D93009154010D93EF81F88563
:104560002BE001910D932A95E1F7AC83BD830C8973
:1045700000610C8B09890395098B0895222711E0AE
:104580002E831D87B22FBE5FA1E00E9480160D858D
:10459000AC891FE9A02309F417E9AD890A2329F0A2
:1045A000AA0F10F010EF01C01F712FE00E94C91672
:1045B0002E8123951D85110F15FFE2CF0895E0E0B0
:1045C000FAE0EF83F887F986FA86FB860E94591A8B
:1045D00080E090E00E94D61A07C00196B096F830AD
:1045E00019F40E94D61A81F41081153EB1F31123FB
:1045F00059F01E3219F411811E3279F703850E7DB0
:1046000021F0003151F71FC031C00085023549F05B
:10461000023419F70185093401F702850E3439F0A7
:10462000DCCF01850F34C9F602850D34B1F6078D54
:10463000002399F6068D158C048C0E181F080F099F
:1046400060F2083050F6AF81B88520E2EF93FF9317
:1046500001910D932A95E1F7FF91EF91AF83B88710
:10466000298523952987203350F4B7CF2985213018
:1046700081F0222321F40C8907700C8B0AC0E0E042
:10468000FAE0662779857A9500810E3209F4639500
:10469000CDD0E0E0FAE0298503850E7D038741F463
:1046A0001BE0008188D001931A95D9F7759601C057
:1046B000B0962A9589F7089522272F93B22FBE5FCF
:1046C000A2E10E9480160C851FE9021709F410EF81
:1046D0000E947D160A85020F1985011768F0212BAB
:1046E00031F4E6EBFBE00E948D1626E101C022E2E8
:1046F00000E20E94C41659C0E0E0FAE010E2019F17
:10470000E00DF11DEF9328E00E94A81600E20E9440
:10471000BA1623E00E94A81603EB0E94BA16EF9186
:10472000EF93FF930385002329F0EEEAFAE30E945A
:10473000921607C0848D958DA68D51D003EB0E94F3
:10474000BA16FF91EF91008D0F710E947C140EE25A
:104750000E94BA16008D118D1795079502950F705E
:104760000E947C140EE20E94BA16018D0695005B31
:10477000043610F00456FCCF0E947C1403EB0E9418
:10478000BA1607890695069506950E947C140AE3D9
:104790000E94BA1616890789111F001F111F001FDA
:1047A000111F001F0F730E947C142F9123952B3033
:1047B00008F483CF0895013488F00B3570F0003889
:1047C00068F0003950F0003A30F0003F38F0083F10
:1047D00028F401600895005B0895005E0895E2E208
:1047E000F8E425E02E2C00270590159080199109FA
:1047F000A20910F00395FACF800D911DA21D002390
:1048000029F400E20E94BA16002704C000630E9447
:10481000BA1600E322242A9539F7082F00630C9476
:10482000BA16A0861027E80364000A0067170CF088
:104830000895962F970F9695862F27D0262E23948E
:10484000372E3214B4F0721534F0862F922D33D0F7
:1048500010F02394F8CF361634F0862F932D2BD0FA
:1048600010F43A94F8CF23141CF4822D932D0DD01C
:10487000E8CF862F932D09D03F927F93732D7A95A1
:10488000D5DF7F916F916395D1CF891709F4089592
:10489000EF93FF93DF0120E2829FA00DB11D929F55
:1048A000E00DF11D0C9110811D9301932A95D1F714
:1048B000FF91EF910895EF93FF93DF0100E2909F46
:1048C000A00DB11D809FE00DF11D13851E7DA55F1C
:1048D0000C910E7D011741F4AB502BE00D9111911D
:1048E000101711F42A95D1F7FF91EF9108950591D2
:1048F000001549F40591011531F40591021519F4DB
:104900000591031501F40895E0E0F8E022272F87D0
:1049100029D000811EE007FD17E02F8509892017A7
:1049200028F0BA890B0F201708F410EFBF8500E1BB
:10493000B2FD10270E947D16359628E00E94A81629
:1049400000E20E94BA1623E00E94A8162F85239544
:104950002032E8F20B890F3F21F4E6ECF9E30E94E4
:1049600092160895A22FA3701DE0A19FA02DA395DC
:10497000B22FBC71B695B695B15F0C948016239793
:10498000EEE2FAE438D00E94680F063709F431C02D
:10499000EAE8FAE430D00E94680F063751F10A2D98
:1049A00001700C6F1FEA0E94E7160E94680F0F93B8
:1049B0000A2D0E6F1FEA0E94E7160F910637C9F005
:1049C000A0E0B0E00E948016EAEBF1E005EC19E00F
:1049D00021E00E94BF1605EC1AE021E00E94BF16FC
:1049E00005EC1CE021E00E94BF16319779F70E9488
:1049F000680F23960895A0E0B0E00E9480162591EC
:104A0000E983FA83222391F02883E981FA812591B1
:104A1000222341F0159100E2103108F40BED0E94C1
:104A2000BF16F5CF28812A9579F7E9CF08950307B6
:104A30007007600750074007300720071004000088
:104A40000307F007E007D007C007B007A0079004EE
:104A500000000D070F070E070D070C070B070A07CD
:104A6000090400000307F007E007D007C007B007FC
:104A7000A007900400000307700760075007400775
:104A80003007200710040000000003350000030772
:104A90001007901909079007100003072007A019B5
:104AA0000A07A007200003073007B0190B07B0075B
:104AB000300003074007C0190C07C0074000030778
:104AC0005007D0190D07D007500003076007E01901
:104AD0000E07E007600003077007F0190F07F007E3
:104AE000700001350000000025970C834F934C7F28
:104AF00011E50E94E716088310EA0E94E716098371
:104B000012E50E94E7160A8310EA0E94E7160B835B
:104B10001A81012B51F41C81112321F017E70E9407
:104B20007D160BC0E4E7FBE402C0EAE7FBE40E9469
:104B3000F414EEEAFAE00E948D16ABE2B4E10E94B2
:104B40008016A881B9810AD0ABE2B5E10E94801637
:104B5000AA81BB8103D04F9125960895AF93BF934F
:104B6000119600E209F40EE30E94BA16BF91AF91CC
:104B70000C949B141E12150577001E121505AE002D
:104B80008F939F9300910001809101019091020108
:104B9000000F881F991F08F40E2597FD0E2596FD1E
:104BA0000E2591FD0E250093000180930101909345
:104BB00002019F918F910895E0E2F0E0F192EC33D1
:104BC000E9F7E1E6F192E636E9F70895E199FECFDB
:104BD0009FBB8EBBE09A0DB30895102FF7DF10171F
:104BE00029F09FBB8EBB1DBBE29AE19A0895D88243
:104BF000D982DA82DB820895EF93FF93188101272F
:104C00001127000F111F000F111FECE5FCE4E00F4E
:104C1000F11F059119810127088305911A81012748
:104C2000098305911B8101270A8304910B83FF915E
:104C3000EF910895DCDF0DD0088000940882198080
:104C4000109419822A8020942A823B8030943B82DF
:104C500008950191D1DF1197E1F708950000000058
:104C6000963007772C610EEEBA51099919C46D0779
:104C70008FF46A7035A563E9A395649E3288DB0ED4
:104C8000A4B8DC791EE9D5E088D9D2972B4CB609B7
:104C9000BD7CB17E072DB8E7911DBF906410B71D94
:104CA000F220B06A4871B9F3DE41BE847DD4DA1ACD
:104CB000EBE4DD6D51B5D4F4C785D38356986C13FE
:104CC000C0A86B647AF962FDECC9658A4F5C011477
:104CD000D96C0663633D0FFAF50D088DC8206E3B55
:104CE0005E10694CE44160D5727167A2D1E4033C67
:104CF00047D4044BFD850DD26BB50AA5FAA8B5358E
:104D00006C98B242D6C9BBDB40F9BCACE36CD8327C
:104D1000755CDF45CF0DD6DC593DD1ABAC30D92623
:104D20003A00DE518051D7C81661D0BFB5F4B42126
:104D300023C4B3569995BACF0FA5BDB89EB8022823
:104D40000888055FB2D90CC624E90BB1877C6F2FA8
:104D5000114C6858AB1D61C13D2D66B69041DC76A3
:104D60000671DB01BC20D2982A10D5EF8985B1717C
:104D70001FB5B606A5E4BF9F33D4B8E8A2C907782B
:104D800034F9000F8EA8099618980EE1BB0D6A7FC2
:104D90002D3D6D08976C6491015C63E6F4516B6B7B
:104DA00062616C1CD83065854E0062F2ED95066C30
:104DB0007BA5011BC1F4088257C40FF5C6D9B065A5
:104DC00050E9B712EAB8BE8B7C88B9FCDF1DDD6202
:104DD000492DDA15F37CD38C654CD4FB5861B24D68
:104DE000CE51B53A7400BCA3E230BBD441A5DF4A32
:104DF000D795D83D6DC4D1A4FBF4D6D36AE96943F5
:104E0000FCD96E34468867ADD0B860DA732D04449F
:104E1000E51D03335F4C0AAAC97C0DDD3C710550CA
:104E2000AA41022710100BBE86200CC925B5685771
:104E3000B3856F2009D466B99FE461CE0EF9DE5EBA
:104E400098C9D9292298D0B0B4A8D7C7173DB3596B
:104E5000810DB42E3B5CBDB7AD6CBAC02083B8EDFC
:104E6000B6B3BF9A0CE2B6039AD2B1743947D5EA09
:104E7000AF77D29D1526DB048316DC73120B63E338
:104E8000843B64943E6A6D0DA85A6A7A0BCF0EE497
:104E90009DFF099327AE000AB19E077D44930FF052
:104EA000D2A3088768F2011EFEC206695D5762F749
:104EB000CB67658071366C19E7066B6E761BD4FE86
:104EC000E02BD3895A7ADA10CC4ADD676FDFB9F963
:104ED000F9EFBE8E43BEB717D58EB060E8A3D6D625
:104EE0007E93D1A1C4C2D83852F2DF4FF167BBD153
:104EF0006757BCA6DD06B53F4B36B248DA2B0DD856
:104F00004C1B0AAFF64A0336607A0441C3EF60DFF8
:104F100055DF67A8EF8E6E3179BE69468CB361CBE1
:104F20001A8366BCA0D26F2536E2685295770CCC06
:104F300003470BBBB91602222F260555BE3BBAC547
:104F4000280BBDB2925AB42B046AB35CA7FFD7C238
:104F500031CFD0B58B9ED92C1DAEDE5BB0C2649B29
:104F600026F263EC9CA36A750A936D02A906099C5C
:104F70003F360EEB8567077213570005824ABF95CF
:104F8000147AB8E2AE2BB17B381BB60C9B8ED29252
:104F90000DBED5E5B7EFDC7C21DFDB0BD4D2D386A9
:104FA00042E2D4F1F8B3DD686E83DA1FCD16BE811C
:104FB0005B26B9F6E177B06F7747B718E65A0888ED
:104FC000706A0FFFCA3B06665C0B0111FF9E658F7E
:104FD00069AE62F8D3FF6B6145CF6C1678E20AA028
:104FE000EED20DD75483044EC2B30339612667A7AE
:104FF000F71660D04D476949DB776E3E4A6AD1AEFD
:10500000DC5AD6D9660BDF40F03BD83753AEBCA98B
:10501000C59EBBDE7FCFB247E9FFB5301CF2BDBDF8
:105020008AC2BACA3093B353A6A3B4240536D0BA01
:105030009306D7CD2957DE54BF67D9232E7A66B39E
:10504000B84A61C4021B685D942B6F2A37BE0BB44B
:10505000A18E0CC31BDF055A8DEF022DF89400249E
:10506000E1E0F0E00192EE31E9F7E0E2F192F131B6
:10507000E9F7E394DA941FEF1DBF10E11EBFA0E033
:10508000B1E01D93DD92ED9281E090E00E94E62573
:10509000A02E82E00E94E625023008F00027000FD3
:1050A000B02E0E94BA0D1FEF1093650010E0109310
:1050B000640018E010936200109361001FEF13B9B1
:1050C00010E012B91FEF12BB10E011BB1FED15BBB2
:1050D00010E014BB19EF18BB17E817BB1FEF1BBB81
:1050E00010E01ABBE8E1F2E00E94EF28009B03C049
:1050F0009D9B0CC014C0E0E5F2E00E947114009981
:1051000005C0ECE1F2E00E94EF28F9CF2AEA2F93E4
:10511000ECE1F2E00E94EF282F912A95C1F7E4E834
:10512000F2E00E94711411E01EB910E71DB9109150
:10513000610011601093610083E98A95F1F7109185
:1051400061001E7F10936100019BFECFE0E0F0E064
:10515000EBBE0E943D1C0E944B1C21F00FB9779BB7
:10516000FECFF9CF029BFECFE0E0F1E0F192F1310A
:10517000E9F710E51DB9EAECF2E00E94711488E24B
:1051800092E00197F1F7C0E0D3E00E94820C0E9408
:10519000A50E0E94670D1AB710621ABF19B71064E6
:1051A00019BF78940A2D0E6F1FEA0E94E71600E0DF
:1051B00014E50E94E7160E94DA0F01E010E50E9454
:1051C000E716E8EDF1E50E9476140E947116E0EB17
:1051D000F3E00E944A15FBCF2D2D2D0D0A000E94F1
:1051E0007114ECE3F2E00E94761400E39D9901E370
:1051F0000E948C14E8E4F2E00E94761400E3009927
:1052000001E30C948C14FFFFFFFFFFFFFFFFFFFF84
:10521000FFFFFFFFFFFFFFFFFFFFFFFFFFFFFFFF9E
:10522000FFFFFFFFFFFFFFFFFFFFFFFFFFFFFFFF8E
:10523000FFFFFFFFFFFFFFFFFFFFFFFFFFFFFFFF7E
:10524000FFFFFFFFFFFFFFFFFFFFFFFFFFFFFFFF6E
:10FF00007F8386898C8F9295989B9FA2A5A8ABAE84
:10FF1000B0B3B6B9BCBFC1C4C7C9CCCED1D3D5D894
:10FF2000DADCDEE0E2E4E6E8EAECEDEFF0F2F3F44E
:10FF3000F6F7F8F9FAFBFCFCFDFEFEFFFFFFFFFF02
:10FF4000FFFFFFFFFFFFFEFEFDFCFCFBFAF9F8F7E9
:10FF5000F6F5F3F2F0EFEDECEAE8E6E4E2E0DEDC01
:10FF6000DAD8D5D3D1CECCC9C7C4C1BFBCB9B6B31A
:10FF7000B1AEABA8A5A29F9C9995928F8C898683E0
:10FF8000807C797673706D6A6764605D5A575451EE
:10FF90004F4C494643403E3B383633312E2C2A27BE
:10FFA0002523211F1D1B1917151312100F0D0C0BE4
:10FFB0000908070605040303020101000000000010
:10FFC0000000000000000101020303040506070809
:10FFD000090A0C0D0F1012131517191B1D1F2123D1
:10FFE00025272A2C2E313336383B3E404346494C98
:10FFF0004E5154575A5D6063666A6D707376797CB2
:020000021000EC
:10000000FF1F627FC23C006088FFFF8008900122D2
:10001000400688C60011FC0304024410014841292F
:10002000F32026F5E61035009AFFD30C10D3040810
:1000300019B1E0EFC6982003644FF301F8FF00FF09
:1000400015E00254800B5001872A049E68FBA00231
:10005000B4050A39F34005A8E686A0CE69B312A01C
:10006000D30A86D0D8E0F6C674C005B838F302606B
:10007000F94C121BFF98FF0505B38086C7C0A3C6C5
:1000800040B477F4D0FF02ACF84079CB40610BA8C4
:1000900030FD022093F9D0FC42C003689E0DF43479
:1000A000801297E81026C401F204CD68D0A001D3D5
:1000B00070D518437848120D05D3C9671AFD40C69C
:1000C0002784F3B0FC6610A3D3B1BEF57C18892752
:1000D000EB30ACF9E09C01BD07C0481E58036072CC
:1000E0000CB369ED06B1C09F03FB0FE0413C679C78
:1000F00036D330DD1CA883D385C0F3E4A6F3153CCA
:1001000034D0FB2084E1E01008454206020A40FD9D
:1001100081A414F6402361219B30451039B2444B31
:10012000D312922620C3BF92888610F0363C20A2BC
:1001300009F9FAB8F88049FA9826A1584F0C67686F
:10014000670493050B7B138211D93009E434D3C0C3
:10015000C1243739400D5AD32611FB3A23C6041B5C
:100160007EFBD319F119C4CF037826A0013CA780E8
:10017000B31ED083628719A6D3F0BC4808C4E0CA76
:10018000F13CF314D3FDC624E6091EFB80411A6F2F
:10019000724018FC428494D347666A92D830088F24
:1001A000B2A906C1FC8D191421066647DB81C6E998
:1001B000E8FA80354646C0E7C8B3B31304B388D124
:1001C0008530DE9EFFC026C04B252053F3749A492C
:1001D000E5ABC0FE2637A814427E8B213EA4047FE7
:1001E0009D0218421A4083BB68D6AB34ADD60122BB
:1001F000A1F870B3DACA067B9811214AD490FA05A7
:10020000F945C604F6FEB01090776D17014C61C534
:10021000EB0CAAF706C63D98805E4487FE0122A635
:10022000AF0A98D3D3983CCFC022D38042F35FCC9F
:10023000660DB397E6DF3E64F898B5F3F298FC726A
:100240003D0FC8FD0844A404AB82C253A0C34120A3
:10025000F085841044C8F79C0A0411AEEB35015AAE
:10026000B30AB5B32584F38BE61A39272022D321AC
:10027000914C10EC40400ACF1C0CCE31F98FA112EA
:10028000FF1640025804032001D3240073044039B0
:10029000F90311CC79879AB3A48566C07B28FC98B2
:1002A000BD92902BF3CB47E93345083EC751FEE0A2
:1002B00001BDD2B29F20198358100B9E22F38804EF
:1002C000B0990C8278DD46E667C1B736ED419E985D
:1002D000AF5060980B026B2C88D298166B74C60FC7
:1002E0006219CA30FE1B5D7F40E3A54C049082EF8B
:1002F000A402F3DF9901C2B361CB25B3EE412FFB1A
:10030000C2F198772BB341DC9AD40440F30C3DDB67
:1003100008A2F8E3324698E2040B64E60C80F3028C
:100320003EC014123389FE1DDF8DAA7D984C47C64E
:100330002BF198F87F148C1305DA70AEFCA6179A8F
:10034000801A15403CFEA830849083B242D74803FF
:1003500088C5E6F6106919FCEAC002425E9893145B
:10036000D3F0A02FF3F7B94021045E98B130DD330C
:10037000AF0CB375D988BFFFD59820EAA503E17EFD
:10038000F397310CF564A79998C7B3F1D67D0F7A2E
:10039000984072D38108F3FE9A17C60CE90A64C725
:1003A000FF04BF05E19765080CD201FEA7A44A101F
:1003B0002001AE41C13681672B660494F614279460
:1003C00020DFD59104F35FD2B1F0BDE621E068FDF6
:1003D00084FC300646C004FF748B60128C0201104E
:1003E0001A04EF65C56020CFD95B671766BF3A2254
:1003F000C020981003AF40C73F30D70822E77F04E2
:10040000D2024476FD1178FD60417A98F2BC98EEF4
:100410001D30902C883CB316C403589D53E62C081D
:100420009AB326EDB005B903407717308878F38F7B
:10043000E530107C02FB1968FB8840BCE5BCA5EEEA
:10044000A2910F393C402128F7F3CC3FB3A632E00C
:10045000C1BEACEF02A5BC5E4A35F33F66457B37B3
:100460007130A0B3BD18B3B040202B58CEC5E35DAA
:100470003F9B308141B830FF3F1EA517F3A79198ED
:100480000C348D90FCFBCFC2067C4208405A02C45B
:10049000A090164243F4D75093978BDB717E7F0771
:1004A000D5B310725BD49E430B29200D6D62343698
:1004B00091EDC0932883B46C623E98B1020E0E3069
:1004C000CA22126631730CF53008E8FEF36919F19F
:1004D0002BE09D30100C82798B170CE02412650FF5
:1004E000408FB2B312D5B34879FA09D319D3ADE22C
:1004F0000ADCF56478785E0F110850FA42362D7DDB
:1005000026804408046A1705720E1402B5573997FD
:10051000C59B632DB30254B3227E73D044A0E36025
:100520000220E38480BC3BB64957E57E2A83FF80E6
:1005300041B04F477388048376C7973DED04402848
:1005400073236014DB4C826962B7CEC4CE9011BABB
:10055000FE0AD9B26639AA8149F41DAFEB328CDDAF
:100560001E08F1F97BD29007EDF020163C98DB9B3A
:10057000300379F2C8CEDB49F93010171AD00638AB
:10058000EF3798CBC8B830B7E0FD7F7A7EC240081D
:100590002D240402BCC5FE4B2361E33FA0643F361B
:1005A000E206BEE526F3A610D740FC3D9233BDF926
:1005B000CDC0AD04A599D780CDB3C08265C828460B
:1005C00090E6CD5EB280B36B977B658EABB3020CC9
:1005D0003DEF80408865C8726AD275EF5003F8B865
:1005E000A41D3480427F6650A35E8B6464C81B09DF
:1005F00054ACB06598C8101312D56139C1A101631C
:1006000099060F1AE827D3F34504EC1018FEED31D4
:10061000023CB6C8ED6310AAEF04CFF2981EE46363
:10062000FB8041EF00A5BDA5797FFBD90806204ED0
:100630004B500CE67FDA320B8A13ED2E26986416A7
:1006400070170FE79BC12077F232100F1B45B4E300
:10065000FE0804AD2D5586544E1AFD29806EB6183D
:10066000EAD11BC6E7803BF73208F7C22488A660B0
:100670002621040E84103AFB5095E621E35BF5FC3D
:100680001730B00B12018E1847A12BDA9CFB060421
:10069000C0E103211306855AF39DB7E37C5374B080
:1006A0009A0BB44CCD8E01FF2610E72D2C823B40D7
:1006B00078BBFDDF9805F0001EC4AE03576A20A882
:1006C000C504F3FF318B2C8AC8EF1E9883C08318B2
:1006D0006BE0E2CB6B2BBBC998D360CD010DA3F8C7
:1006E00065C82B2940F31F6127824B3A02CF92D075
:1006F0004D369082B97FCBE12F12787205D4241A3F
:1007000043F2D30CA6849581FB8B452F6BF6D24226
:100710004CF3D4CCB3CE3236D7F2C09BB3E5C81E6F
:10072000FFF33BEA20FDF3E214EE421A40CCD5A8D9
:100730004E8490229A6E420365CF2184F3AF6D15EB
:10074000417A16FCC0C812D75208B99821A401E01A
:1007500035F342A2AFC67E1C84B0100CFDC53D9897
:10076000826636F18101715F9FE4981FBFC8A2B114
:10077000D7C097D216305FF5E8981ECEFA7FF29870
:100780003C60BBCDEEB118C8BD980C42D3F38FC608
:10079000DA49EC1708AEB35FC490CB1E20B3CA1180
:1007A0003AFC0414CCF5032D212068AD401A0BB39C
:1007B000BB2727C8DF08410A68BD681025E0F36D34
:1007C000F37DF97E50340CC3FE66501009064028B4
:1007D000B4B0B6C3B3C80AC604C0831813F9621212
:1007E0008C8240F36765C87B5E42C15E989E23F9A8
:1007F00084023042E09941AC05B6AE141E23E16993
:10080000FB60272C8007BBB1D7A558E5C878985561
:10081000E48B1946E6778A98EDCBC85F69980BE0C0
:10082000D30581B0165A3277886B1997FA64D5864A
:1008300066EFBF422DC87CE5B85DF3F343BA62B101
:100840003F666559E03D0E02801008AFAF9910E495
:10085000169BFDB349B02006C07D426551F9C873AF
:10086000B3100387624CF68205310976937DCD265D
:10087000C168B3BB8C6709F382585D1701CEE605EA
:10088000D8FF75ED8590F53994C8DCC3A184C0A06C
:10089000C239F34823F359E836F302BE986DF731B5
:1008A0006AF314BA34BC98BC5BEE91D96B96979EF0
:1008B000A68B04C8FECD33843C985A7EF998B111BA
:1008C0008C713032FFB8F96FBDD2202E26EC240E89
:1008D000DE5309F32BBBD5B8E096BB6FCB7EEDFBA7
:1008E0005718AFD05C9802E016F0FC942CD30C386B
:1008F0009FFC242BCBD23E9B44080C21675505E579
:1009000024145EC5E1230A21E82884D8CCF34BBA2D
:10091000B18BFAF4ED689F2BE0F75C42FC6FAEED13
:100920007CD088F88401902C42C0EEF30493D2E985
:10093000DE9604C0008BE032AF16C5E077AF984971
:10094000EDFE103F01014C824530093BF32458B5C0
:10095000620441AD7F50FEE0412C88EB05F1002B95
:10096000C8570222F0305F16C4037ABB10963008D5
:1009700025CB3011FD98406993C8C61EAE047F3068
:100980000B60800C20D0FADF8801E7A50A7306D33C
:100990001571F33A6665C8BF5A64F998F9A84759C2
:1009A000F5643D66010870FC27ED04760058FB10E5
:1009B0001361222CF27B87E0F3642059E88831CE62
:1009C000F59891C619CBB35197B348A4B38CB1EB4A
:1009D000C708FDEBABC3983B30C840E9A17022C704
:1009E0001042CD4843D00D2C6E04FDA2E318ECB1AB
:1009F00002AFC0BFA0637334EFED281086EC203C3B
:100A0000F8ED3401C8CC2CE3EA1FE23077E4C8FBF0
:100A1000C017068DD24612D9F5B53DEC6419C03920
:100A200048B3388EB3D52907DFF95E98F20EE0019E
:100A300038F36B621C4DAF3B3CB098FB1A80A54865
:100A40007BD2100859F5C111849840A841770974E8
:100A500041B60DCD3E11AAF82802651A022299D995
:100A6000C8AD24AF293F5E6649928817095BFECF67
:100A70008011E212C024E3180160EB144CDF9809E6
:100A800002402288FF04626024808151308E02D7A8
:100A90002D0559658851FCAF463B985EC10C800519
:100AA0003097F3287F7F124C5E641789FB6BE798C1
:100AB000F13DFE9801715DB676C808078DB39103CC
:100AC000A213E8D7C598F4D9C8AC41BBC8CF98C821
:100AD000C81F0D2030F8802E89CBD5F3C80CAF820B
:100AE0003FE5815DDF61ED98A005A3B3D1026A66A1
:100AF0006DE098593E989D0866200CCA41734C19C8
:100B00003176C424B369E94B08A6E58818200BDECA
:100B10005E2D5C7DE4086AB3B984B3C26AB39E906B
:100B2000C62026C84AB3ECEB77B5BCC884FCC68C9B
:100B3000FFE5B3048DB7D330FFFA8610F123566773
:100B400001F36670290B211B6CD388FD6895CFF3E8
:100B50004B1C76DA88FE2834936718B3D9396D496F
:100B60008506663EFFB39804B3A0B1A123B46366C3
:100B700013FD7D40B3F7B0FDB2048F5132B18D4407
:100B8000CDB3CC5D44171356F398FBC6BEF9CF31F5
:100B900079C6D398FFCF384A602B1AFCE540D9C7F5
:100BA00016DFBB5914F6102450F823E6581B16FF25
:100BB000582E242CFF981916B308112CC110CFD829
:100BC000C8FEA7AC624031766710C8FAFF885B1E8A
:100BD0007E58044E6FB340993720FDEC6DED0B024B
:100BE00020924E4DAB02018A281441D8DD7E216F40
:100BF000E3CF9E90A5FA25C0EAA50ACE3A40286D1B
:100C00008AB406A69C28C48B5979CB1480BCA50A4B
:100C1000FE400BE0F366A9400578E4FA2003D81003
:100C20008D790134F27157783779249CBC15478C43
:100C3000C6FF5D6402A360B80A8A080D54AB1102B6
:100C400060A5406E212DB0FFCC4E7FCC477FFB0EC0
:100C500090FBF4C145C32F8F2D06965E60CBAF107D
:100C600015EBB1339A6C108050EF82C65BFB2B9171
:100C7000CF045B72FC04D38CC2F31A8D2ACC42A33E
:100C8000C69B9BA8FF13582510E7ACE748F31BCD84
:100C9000C17D982064794B8687FFB65188FF607BC1
:100CA000B0AAE5FFCCCBF9025FCD09FEE9C25EB385
:100CB000C4FFE3088D80FAB224B658D4E341F3624E
:100CC000DB962FD332C775550A46F19FE1D939FD1E
:100CD000A6D21D6EDAD8C6B37B80616BB318FF62F3
:100CE0009B49B080C9A258B7FF1625D525CB271040
:100CF00055FC08843F0CB0B8B776490112E62E02C5
:100D0000D9F70661BEAC62FB35F51008897984BF5E
:100D1000D8327F9AC2043066B7ECE47FECCC30580E
:100D200063029F25A7F8B386EBFF403BDBB058FB7F
:100D30003126406518845CA2D8A8FB9E568B981972
:100D400063FD1EE8FF1BB870DED77522E30C015A65
:100D5000801CF3E6624625CD98820290C67FB65A83
:100D600038FF21A68D5FF5F68101C1970DEFC08494
:100D70003DAED978F9CBEE8433B65820A2FC843549
:100D80000C8F3B16E0FE2013D9E3FC637BE305EDFB
:100D9000E04004E6C6FBE3D9E8F8A441D261AE8E98
:100DA000F17FF0F9C454CC8066BF10ECC15FD23043
:100DB0000170289681498DCD34A0F97CF1A4E471AD
:100DC000880D1210A1C2A0F9441CB305B936806683
:100DD00068B2059401ED721B8299F991F8AD440651
:100DE000EDC7500A5FC99C2DF5B4100906F133FB1D
:100DF00029B40DB62033B31A055288FE1F42D51E02
:100E000004A06D72813D9C684C8558FE8FDF083AC6
:100E1000B168111F56620801210C8186108D1803DC
:100E200032BC24380D0499E6CDCE6F824397FE2361
:100E3000088C421CD71844202102F9F2D937E93B2B
:100E400083EF28FB3219EE158040CFDA3665BE50AD
:100E5000FAF9FEE847C8A40F1072A26FEE518C4257
:100E60007C89F1BB79CC19276B020898D458F88E8D
:100E700037BEF2A6235DD665678089726918C8FB04
:100E8000C02CC676FF94FE6F9AEB18D968FFB2901B
:100E9000F649962A0277585692A408CD5E8E10F134
:100EA0000B88FF65FEF140C7341DD409C5BD30C8AD
:100EB000B7FF14E5ADD26CC7D8400663BEE320FF90
:100EC0004082C4C4A0AF1401490A34B228EB78F3BD
:100ED000940FE6F30DB25008E32896D305BFF4A1B2
:100EE0000AE0F340C6DEC64DFF88FABA250ADF766F
:100EF000CC201AEB0FB0F96089A719B6C999FE6723
:100F00001BB9FD7E8FFECD08C4391568B0FED7CC65
:100F1000A8F3B33756FC015F98FA649FBCFEC6DDA8
:100F2000560463C620FDD4629A15A530BED0FCF8E5
:100F30005EDD19FF40AD1A180FA5A4963420BBD36F
:100F40001404934A40B8033E17148A0620C6ED42A3
:100F5000035BE418FE1EFB903FEF98DB9E13D7D98E
:100F600028FD60023C61ECC0C5064FF20C800130E8
:100F70007A9DC09A4B0B8233F3DAFF3C0856BD1EB4
:100F8000CDC328600AF3C936F36B66B8FAEDD8C44E
:100F90009CF5DE1312F89B113B4412CA2E38223CFA
:100FA0001D80FC897AFA02C8FFC0F88089D3300915
:100FB000991804B2137D0D834B660A12E23019B6FC
:100FC00039449C19CD392110DC30DB9804318DE097
:100FD000FAB3013CF9F0F2401EC0038C36E081F612
:100FE000B21E4093B309F33C621FB7C82C20D31A3A
:100FF00016D062D30FE47B2CA007F2CDC67FCCF9CC
:101000005FD94CA64018471B062F4E882D66B1B7F6
:101010000066E466AC68BB3DF79F106403962CF352
:10102000DBE347B311F4B39BDB600416FD32D0A2BF
:101030009C0D6EC620FD9598BBE470FB35FC34A872
:10104000AC842FF7C52008053EF340428210EF4DD7
:101050009824F321AAD924D5F81203140A77A29868
:10106000442CAF2EFC5F812014841A14F37BFFC044
:10107000F96FC695EB66443C715A2DA8F80666DFF9
:10108000CC6CFF509730664350C06ACC480C90B689
:10109000F0479998E6B3BE98BF04C598E979619383
:1010A000FCDFA8FBC5E3806C9423113C655F47E53A
:1010B0009896E06EEBC705EF6BF5984011FCE1DF09
:1010C0005C8440DB9B48B9FDBF3E16A442760844D1
:1010D000F54CC226A808480EF932F38490CF21B30C
:1010E000B6492B82DE658C8045B0061240B3C80934
:1010F0006AE2D7E9F979DE9007B09A7F7F176041FD
:101100000480079037A3447898ECF32C084FDE98BE
:101110004016D08213BD983CFD8805B1201EC81A28
:10112000F33427F80448C006407FDF7FCCC406A014
:10113000DE5B84663612082DEB98815EE43702414F
:10114000C6B5F36FE492FBF9A8E06AB3A101F3AF6F
:10115000BF18CE98F37E16F59803FE98A234C65BAE
:1011600073136E83FA57958BB2BACF19D137D182E8
:1011700042FF2F983326B62FFE1410B5487FAE9845
:1011800004518D82F0E2E300C9DB491FD320CC4635
:1011900065FF589BFA6E30C5434676914402F49839
:1011A000B0BFB1D2984248C414B308D37F17B191ED
:1011B00098E036441880FAAFD1FE2C751F46A591F1
:1011C000F7781742DD34E498CB677A4B81D419D78E
:1011D000E8ECAB96C642CFDAEAFD84819D10E9C007
:1011E00028AA865173FC46A193857FEB32518CB0BF
:1011F000ED5720B0C5328198A34F9F84093006FD7A
:1012000046C120880083B77A17FFE001F4B2F0BC32
:10121000F6935DF3E698BC305C16677FB971802861
:10122000EDD3B83DBD98E0CA413CD3E623C403DB0F
:101230007DE3F88C017AB2C0DFEFECF59818FDFE83
:101240005EE567658EE7EDF571AFAB9806D68B046A
:10125000CDB311FAFEB279B388F9989FFD7F293496
:10126000DE98B21A7C98B830D9B34081F8105F6E1E
:10127000699BC8025CCBC842D3FC9835349D9BF86F
:1012800002C20F02EE08034BFE90B3C850DA030807
:10129000734A54FB648BD0E11659FF246BAB806317
:1012A000043BD72DFCEB30C0209A065318FDF941C2
:1012B0002626B019C4EF5698E299E2FA1869E09828
:1012C0006D837D9806D0C120F3468D9BA8FD1EE559
:1012D0009A44684895101CE298CBFF119831D9A820
:1012E00019090D7BB1206BC4307522F3B5FF12CB09
:1012F000FE80942180999958FC60BB7AEAA0D73B84
:10130000C8804911CEC83002BF5258BF203AC81118
:10131000302C839B8EF322DBE4A9FE6CC2C850B54F
:1013200078CBC827CD98966E0CFBDB4DEDF020F9FD
:10133000D5D70FE29A9866C819D7AE17F0E50FC94E
:10134000C8666BFBA4A05C96C8E62396C8BE982F1F
:1013500088F298232DC66E6DA283FD7CB2E3B35351
:10136000D07ED887058F1ADCF898069E986AC66BDF
:10137000CF7CB8FC208447ED64C82699C84664B980
:10138000C889A404B6213221BF7F50D620805AD507
:101390007998D9C82DF87F0B8896F9C310ACFF0255
:1013A000A3F8F45FCFF398F87D01195D647F1F30D7
:1013B000E898102DBD988236F380ABBA50550F08CF
:1013C000CABEF05B61037A98C096D303ACDAA8F981
:1013D000DFEF82E2B729E61808803AF0986FE23032
:1013E0000CCCD86DD5B3057FA5C448EA9596C8FD49
:1013F000C7E56AFF80077E8C22D7AB37D99586A0D8
:10140000D27E8E62D49088D5D946647E320657D378
:101410006B24892BC8911012F34122F1136BEF4B0F
:10142000D0FF60405EC52D2672C8334CB4C8F69814
:10143000812CDBECD38FD7A73C7991801EC8E85E66
:1014400098F2013C8005C67BF38318204DBFE32B47
:10145000C86D50CFCBC8C80F0466DF25C8ABB966CE
:10146000178999A579C8DA83607B70E1FAD1405178
:10147000F96902A2B321FE6E305810F29837C637D0
:10148000665CB3348E961A26BE98AF269B45F360F1
:1014900057E1FE20041DD9C86DADDC1504BE61C83E
:1014A00024B3F2C8DF40B83FC898F3B3C850C9109E
:1014B0002AF20F10C27CFB2CEE632DC8C0E432B3BD
:1014C0002D806FE698AD934010FB5CCDC8FC0130D9
:1014D000FC5D7EE62940D980DF35C88297DB9940E4
:1014E0005BC96239C82BC6F4CCE0B3D230FF9A0492
:1014F000D38B5D34CE21686F95C8B247D1CE3252BE
:1015000072C8F1ABF341F2EF04616632FE1A0D0AC4
:10151000DD9618ECC98041E6FC26A49384FE62CADD
:10152000403033FECD4E49D30858EDFF962C80490C
:10153000300106C1FD280805A10041EE0EE8FC605F
:101540005FEA96F5B9C8B20C33C8605C1667E67BF3
:101550003C2BB830B2D5FF5D98889DC8C002AF0A59
:101560008D19FBC2F85DC472C8C8F6E51201DBEC48
:10157000784721C8DA81FF7749FC317E309EE067E9
:10158000E5C874D1B3F83AFE58A48E76C80423AEE9
:10159000D9E8FE10B2C842A76994C89DAE81153043
:1015A000F6EA9828F08EAD56B392ABB32899635003
:1015B00022A44DD285047998DF7E1975D3ED645845
:1015C000FF91F75C1ADE1BEA1BECFD3ABF11C2E08B
:1015D000FC306BC63167B52B18FFA35350E015A63E
:1015E00040C88A4157925A44E7C83CA06AD9B544DA
:1015F0006DF884813930805C3DBB0FDA9807F0E3E9
:101600008A6DF60FA0F82CA269FCFE80BEEE423077
:1016100082699BC806658C12BE6E08043F13DA9877
:10162000802249AB107EF36CB3FA78FA841130C98A
:1016300068109904ED21DF5B89DB16A27C32B3F3DD
:10164000FB96802FEDE5300313F4E0090682C06EAF
:10165000B193F09809B3FCD7E08197D2AFC540CAE7
:10166000C8CBF5BD9844711919F3DB19287DEDB984
:1016700030C4A583E0E8CBD3F1BC8BEF569880F75C
:1016800049FD8CF9D2AE8D159331FE98BC90665908
:10169000F3FACC0231FE36301D66D3C4201AF3FBB8
:1016A000AB20FB69E0859B2DB330FD980865991947
:1016B000BC30CD2302E088FE98B904B3142BEB7A3A
:1016C0003798FCFD87847DA7AF173045247FA0980D
:1016D00009520DF004C539300AA608D225A276B306
:1016E00021809D09AE410E3016D8FA8CE053963019
:1016F0000C4AED10DCB6FE2330F1434673DFD519FA
:1017000058E99838645ED27F7D91E4010980DE98C3
:10171000D1D002F32CE620DD5FFD04C530E7787AF6
:10172000988278B38007E0BC1C90038E0901F35BBC
:10173000E337E5848154A350A1B6DBDB94300CF38E
:10174000672C66089ECED4808920A1FF38989E9C85
:10175000591043FE851302ED46C8047B1709F0308B
:101760000126A120987A0260082C36F3166D44C732
:10177000B372EA020AD3AFB35D11D70226BDF801F6
:10178000036020ED0149FEB7A59848F3FE98B49098
:10179000F49878D739E4AD980705BB36BF00305CC4
:1017A00030DD16D0E898689B2C88FD9883BF78DDE3
:1017B0007E10E0FF35602006B496D57953FE9895EB
:1017C0008866D277F35A4917BBDABC9FB3C0304062
:1017D0002FB32E0FBBC4D68B618BE29B4F3798E59E
:1017E0003091FE98AC989724482D99044DBB57B37F
:1017F00004F1300ABB5614AEDD79FB029810236069
:10180000F72F20C068F8636BFF046FB1319D371666
:101810006DFF48F8749CFFD96C01C6F372AC22D7F7
:10182000768B40A6B563D3A8FF018243FF98FFB132
:1018300028A36638D1C71639900986666F5B3BE5E9
:10184000DEE6FA2C6605CB7340754610A3F370FCF8
:1018500011925146B15AD120C480B13737E035A436
:1018600076E438F920091FCC6E197BC80210629EFD
:1018700097765CAC056CE100B1C526FF50FCC13722
:10188000E87F56C115B3FC60A7EDE54041846BCFFE
:1018900014196CE488FB8FA30D0F0856B210BD66B7
:1018A00069C67C5FB66168F915AC3780AF33DADBA7
:1018B000FF18FDF867FCB4062F9A2FC852F681D4A2
:1018C00002C545B0D689F3590820D140FFF3FB3E4D
:1018D000EE3001C204E9BD78A04B370A13EAAE52DC
:1018E0009988B33084D7DB4945DDB70CFAE352B9A8
:1018F00078B3487492C00460A305ADF489BF9B42DD
:1019000038AA0803AC41B291C7020472C080E7D480
:101910002844216570131266CCFDFF209641632B8D
:10192000FF0211E6ECD0FDCFF90F9F4AAE8158B40B
:10193000829F6C19A093D735E289B1FCCF37F8CDDF
:10194000CE88845ECAB6FF332ECC91FE04185B6746
:1019500018CAAF994B7A6263A65A3FDBB1FE3FECDF
:10196000987F4C055D4588B3FE5683201CB656B85B
:10197000FF4F5C9CB5B2083E08CFDB963FF6A70848
:10198000FB117AFFA0D066C33EB35FCBEE8C7DD057
:10199000650C2A0065CB586530FECBE3C809D44DF1
:1019A000D866B00191D5086102DEFFC716CD04A646
:1019B0003225D6627B48A9F86099A6FC3FE66514FB
:1019C000FDCC825A6680C8E3A00D4DBCD3C63866F4
:1019D0000163DE6C61476C9FFE4BC04C3093D64C6C
:1019E00020FE4CBD08C5A8B2FC96E00412FE7E089D
:1019F000C454D901BDB1FE45890119D60054D8455A
:101A0000FAAA40E5308088F162988CB40C33EBCCB4
:101A100073F7F2D0FB08B00247F6E590FDC67FE908
:101A2000047A4308D81E818A316DBDDEE630B1FEEE
:101A3000CCB7EB3108FD3F5D6FE3CDD980B201013A
:101A4000CB58BC20A9A31AEEAFEB04F3E37FA3CCE1
:101A50002E3FA966231262BE15B1012DDA85203B07
:101A60000E54FD0840983490D879ED325508046B37
:101A700010B622A0528BBC76F98008CAF53501B9A0
:101A80006BEC2349F90A28D0E9A6EA501D2210EE92
:101A9000D6856B0281D019E1400528D9A4CEB34088
:101AA00080056DFB453FFE18C28028BD85DF06A678
:101AB00011FB05A96EEEFA507384B80D0320CCDB40
:101AC00010047C8A30FC5A42400D2803DFE606FBF6
:101AD00028406F98D8B4411A5E2001CE480309020D
:101AE0003A8629813837DD0F114063819160A3FF69
:101AF000F57D3CE5C58DF5853BF398B34DF60108C2
:101B00009DC6EEDFE33BE7B8F8CFC9FB8CC6E034F7
:101B100002BECC0C81545D621F64716AE20ECDCBB3
:101B2000EB34C79919FF102CBE9F9703BE9AE69815
:101B3000F3B72D72047C2C0510DCCB6E8DD9FCFF25
:101B40005EEEB80963C7F9CFA02FD53325DDE4D009
:101B5000FC409BE6141CACFFC86B4EFCE30A19D595
:101B60000D209CF6B030B348AFA1CE32AA5B0E5820
:101B7000FE6DB78C23D3F0C078B23EA60B3BF6DCEB
:101B8000824F76410488EB95FC7DC8F102D129CDC6
:101B900008002635A57BE7B1E9E3AF597B9C30B25D
:101BA000F87E84C596BA3067EC6140599388B1F9E4
:101BB0005DB028C35300028BFD6366B379538C6D0F
:101BC0001C7B43C8FA018CAD45023E8ABD180862F1
:101BD000A6BD5BE741FD018C74B1B1E635F8109408
:101BE000BC64F4B11A3057663452F7EC0368F9213B
:101BF000B568FDC46F90DE0DB62004732AA001D72E
:101C0000348026691AD3681208E06DF3D079B2A146
:101C10005FEFD828FEDFEC92202FD215FC06C028FB
:101C2000181703E6913C0601F07962C00378F5E3EA
:101C3000E00110B3929901D38966D36025D3E06C9B
:101C40009BDCC61E07950FE6D464B37F61FD40A2FE
:101C500070E63784C073E52402ED04C28180461A21
:101C6000798325D3012AFA6BA222E0ECFD4264ECD1
:101C7000AF2199E782F9FC7894929394B69A590926
:101C800046E89B1F0B601280829645DC7F9C407467
:101C900001EE67808149F12DD33DC5014C0237200B
:101CA00050FF00263226022609BD08FFF3800732C6
:101CB000401EC8839378CF390C670AB4ED00E05713
:101CC00026CAF9261919F3F0F3830478A240F359D0
:101CD00096F9B9CECB300885FEEC7639884139E5E6
:101CE0003AA7A26E7218521B58029AE668FC2FEBB4
:101CF000E6994218070144ED21B31AB32245B361B6
:101D0000D72080D9E3FB4F23D3D7024F12D3212012
:101D1000845B675B49D21801B34C87775FFC80FD19
:101D20000584900610427A8468EFAF755DB8C0E90B
:101D30009868E0B2A2167A24ACF8B20194D3B384C6
:101D4000E3080921DCA4F3DF1242E9980DA53BFA70
:101D5000D8FD9646069E34631D2A6DF2C3D7C69EF3
:101D6000FF68F9E001FF159806FB5E02FE51FF5D7A
:101D70009860E6C57AB386D3D6981E9F312DF3FDC1
:101D8000980C73D338F9C02840AD20ACC5E2A262EC
:101D900024226ACD6220DE980A0113215E0A6AF8C5
:101DA000CE0544D3100402CEA602415EFCF3BF82EE
:101DB000C698CD0473C37BFBF89023E3EB0218585D
:101DC000180C8C6FF12C59D101A3731987EFB33024
:101DD0001001124EE0040920042403F30A9912C6EC
:101DE00058A3986088814BB325FE502C8188B23A65
:101DF000A6C082F5C508DE98FB30401ED003FC98D3
:101E00002310F198D388054F26D358100B9FE2F387
:101E10008005B1204819787A0F60F7D8F8FE840B56
:101E20001008D2064016816F5F0CEC24C053598312
:101E300046F3279ABA11D2DC5166811FDC12471291
:101E4000F8985A80F6BA7BFA1509DEA59804C013F3
:101E5000C1A2C0EC8BC2270DF389021946FE98DFA0
:101E60003002D9171326814C84F5B01026C0D484D3
:101E7000B37FBA8BB8FF10E25A2FBCDC376A755EAD
:101E8000C5BBD29A500821E35012D560047B47426B
:101E90000876F7EC2884F93A0AD339DAF65B4FFA78
:101EA00091D7A0842BFF01196EE4E8F9F60906200A
:101EB00069AA88B30F7F9F98DB64624E3350F83075
:101EC000B81080D33BE5D1F3F97B49D312D32B571C
:101ED0007050FC5347A0105FBF44B3535EC5C2C4EB
:101EE00042AD056DE20C28F8305BC735680485C348
:101EF000102A507F222904B8AB56D3C5F9B928E17E
:101F0000FABF048FD7F83F704CD66F2A22E7CB2058
:101F10000240D99041FA7CE38408B07946C14488F4
:101F2000D3F460100C82EAE806C128D33AF240628A
:101F3000D3C8FB2F34A5E4301895197EEBB8F1B95E
:101F40005058D9100F2619DF28EE71413CE63D1696
:101F5000C4BC78EF23A5F34E2F232F8BED1BF80C79
:101F600034FC135D57FC10AEB840D86CA67901CE96
:101F70002F66E5F33020397593FD642DD836880C33
:101F800062DD9282BBE3FE23E08CB4E43016ADE662
:101F90005D1760F6927E97FCA96B02D3587F4B17B2
:101FA000F3CBB38B238E30FE72B0F81505DB0577CB
:101FB0003B0E60010DBCB5B3C842BB48DDC508206F
:101FC000349C193DE901A0067A2750FC95C8F39787
:101FD000C8E48ED382A8B388FD6BE6C56658375631
:101FE000FFB710D545FB69DC703DAF1995B946C701
:101FF0008465C87C25EBDE0EE28CC9DE5DCA45E94E
:102000006B21577FE032423BF53220F7DF7A8B417C
:10201000B796F8F920508440801AFA8142080C14CF
:102020003B6D38EE2840ABC7C5394430B304548308
:1020300028B820E3228C5ED720E79B08F050FC8B69
:1020400070F373F93F20300906C02432A093E8BF33
:10205000BA300E161903C70460F614448011782EA6
:102060009880D3C0FD885804F9C8BF416E5D4AD33B
:10207000442C763A89FC6057819869CB3016F3E896
:10208000E2EC413C10D6B3E401EF339833C8166C50
:10209000F35C304993089F2B4DEBF9CFB0F1D81C7E
:1020A000324C62F4BDC510677998AE9ACF9FF3C2E7
:1020B000CAE48FD3E60393FB5BED733060102FAD62
:1020C0006BB30258C498D47A05DBF833A864D3D331
:1020D0008F10C8C88FCEC898048BD3AB1E9ECAFA87
:1020E000B001345F19EBD268BA17BDA5D43DFD50DD
:1020F000086978AE6D040A9BF97F0291C38410D7FA
:10210000801A9D5697C8663F425BD37303A0FD6358
:102110009EBC796DDD016A11636CD3B0FCAE465D87
:10212000CAC2C8CA60740C193D3FC08004FDD1CB3F
:102130008801083F57AF3CF203C0FEBBB1B017C0E7
:102140001A1DD3DF17C0FE8C91BC807E324406205E
:102150005FD635EC02E1B82421CC842FCEDC9F84FD
:102160007E401014B76B08AC0488C8811AE882025C
:1021700048042075CC033AF83988941C949466B4CA
:10218000A624C306461E045935896DC47E73C2D782
:10219000D64A46AAB485FE7F12C19E74132011242C
:1021A000EF74A5264022C69D20AA81097EFBFF5B15
:1021B000467998706AB5EFF5B80264C89646096F1B
:1021C0007F52E0413C8805F09C80E08358BFD3D328
:1021D00098B1D3C47F1D03BDB6FD0C93D4177824EA
:1021E00061590B18B2BB9D0501100499F3777F303C
:1021F0003404C1F7BF8328C8385712A88B22E69948
:10220000B3A1FB0E2607C042EF74C5042C027C204C
:10221000F33F2FC8E8584CCFFDCC8005300226DCB8
:102220003DBB13D4A584195E5E5E6BBF4139C8E027
:10223000FDE0029075AF4202A9AF01E926DFA4D00C
:10224000877780084CE0A201B0B3755FA0AF01644E
:1022500078144284BB8625C8C6FE8BAF08698B24E0
:1022600084E7FA6E8A5E486299D963FC1E6EDAEBE7
:10227000F8E041B1BEC47C18080378AF993B98D20E
:10228000C51EC3BB4482F6013C08026AD181EF013E
:10229000781C7F173D9F5EEB8BC4FC8B9DDEB8FFE7
:1022A000207067D7E682F7270A0177E0A010EBC815
:1022B0004842BA0C8121F1ABCE66A86610F572D304
:1022C0004220D3EE403D815E8B5FBE43BDFC0131B9
:1022D0009EFE4FEF0A0640C028189AA1B12C66D284
:1022E0000A46BE59ED82B65187C69AB34174F4418D
:1022F00002D3FF60148C8250100842DDC120EC8BA9
:1023000001849CF3E399FDCD7B2CD5B07898669938
:10231000C82B192EC8C8E8BFE0010C8804666AAF54
:10232000E6EE6630B020E002ECCDC801D305796B53
:102330007B8B100BA7602A38FA80DF4110A2B5779B
:10234000B629E238F398F22DB5EF316C6FD9500110
:102350001F942739E0088177CDD9D320FE8BAD03B8
:102360003BEA31BBFBC2CD113019C02519A3E016E1
:10237000B3FC3C0204981085B34C25DEE69BB9E320
:1023800009CB9910D308D3B923B349370B46788BBF
:10239000FAD30A4C8211CE2EFFB06B94A0F3EB8AD5
:1023A000FC6A770E30F310D202C9C8C03BE82004A3
:1023B0003FD5E520E178AF42E2E80DE4202B8FCB5A
:1023C000FDC99891350328FC67E902E6FF6E6D822E
:1023D000247E2A0B14CBC8C78D59C8FDD680016650
:1023E000F524A68413F83085F3467ECC726BC7E0E3
:1023F000EC31FD16AFEDFE78BB40379BE0F1237961
:102400000F01B3EFFE8C21CDF58074B1804A827547
:1024100048C4F401F30881011A32B3007FCC05EB04
:102420008480888B3DC778E021307E719B024157C4
:1024300091980F3286FF04CDED1AAFD113532B02C2
:10244000ED2201C580088F6004E52C8849D59DA93F
:10245000AF45C6F106400498AB93E75FBEB000C538
:1024600026C132B50B89BE72371078FC5C30FF880C
:1024700000F0200EC083780D7130715065F57998A9
:10248000715D71309FBA492CE53D2065C816E07337
:10249000A89007C6165E9844F3D3C4D8FE77A9B2B5
:1024A000C037037F2430307AB400C9F58662392EF4
:1024B0005E78854218D70403B76B820164E8AF39B0
:1024C000349857D3D01130EDA0B3AC26BF7B873002
:1024D00033604235E091A6406BB309B0AF204BA505
:1024E00058D3CF191EC6A6136024F7B350FEA00917
:1024F000701BF7AE182140F130732FC202814240A9
:10250000EE68000DCBC8386546A25E98801AFFB809
:1025100036F34AC6FEF39882F35BF865C86D8318FC
:10252000DEB72D421456F80A37CA3020F49838C561
:1025300053E2801CD38930F3F0EB201880A8644666
:10254000CFF737C00108771210E0701D0E03F35A61
:1025500082AF042398F3DE198089844039B9871B40
:1025600008860C8EEFCCE8044A50CFEC0C10886E35
:10257000546AAA5B56BB0420D54851D37E2130044F
:102580000675F31802D386EB81AF2466A98AF9DEBB
:1025900031BEB989D7EB2C37CB306587DE8B4567E9
:1025A00096DCBE9F6DAEF48811B0B3D5242ED4DA7C
:1025B000A3E6DD2206B5AF01F79320028C7F7F48AA
:1025C000FA6BEE9806C883B830FF7D98314016C488
:1025D0008375D178ABB4396DBB900315F8E895C815
:1025E00095D5C63D9E985C03BF2028C8F3BD7AFAF6
:1025F000436670C0A480666107717D6ED920BCD827
:10260000B482B9CCA0B4056DBBD0024E66F3F2B271
:1026100091E366C6F3D318B3BB407FB6E521FCBE99
:10262000983DFF0B6004CFB32106C2088D58037E8E
:102630004BC8A75E36CAD6A78489E5D388733D62A6
:1026400081332691F316AFC256F80BEB529059BF67
:10265000C0FA696346FF56582EFBFFE8FBBF20A572
:1026600004D2FE796719F3CBAC221B60D3B8F930E2
:102670004876FF98FF2C34936718D1D939741746E0
:10268000090D66D8FB97DB74200E47B56A38F9BB95
:102690000CAD108C51F3373FAC2D6017BD4BFDB026
:1026A0002047FACCFB7F208BCB324CBA1F1353DF71
:1026B0001FFD32FB853FEAB108D6E010FFC656E3A6
:1026C000025AB710C7DB93B0FC1B407C20B040A57A
:1026D00046D0BFF96C582A312F8FEDBF98FE4DE6DA
:1026E0008C3A31F38D7542F8BFDE7FB17ECD9AE32F
:1026F000108C285F103A2B63BB29E0803481406640
:1027000068BCB744F0EF4FF23A31D425B208B0DAE2
:10271000D9DB445EB9A602E690F9F2AB40F3509BD8
:102720003411048160C1E04AF00A6CD10825F5B388
:10273000AC28DB40CD909538ED08932E0CD580F079
:10274000041658FEE741CB848131EE02ED497FA9A2
:1027500090A750F9050211831560B352B22E8F78FD
:10276000F5CF50DB89DE01206BB6287BE264FD806B
:10277000401BF3233FED6AFE06C43DCAA8DDFF42BD
:10278000DAA144D304BA2913CDDB7F37822CE64C7F
:10279000B0DFDB2F010833F9ACF5FD48B710479BDC
:1027A0000470A60B126E31CF1E3314FA1ADFA70085
:1027B000FF70FC4671678178634B0B801AEE4D0801
:1027C000FFC44C8364F20318FACECDAAFA8B977F2C
:1027D000D91F2BB48828E1C57715A0B1F9554A1047
:1027E00018CD5DDD6048FEE9CB10BD69E7DEFDB6C2
:1027F000B6D83E8FD93526E0FB1147FE8DF342F95E
:10280000B873B2A74CCA33DECD58FBC5BE98C7FE1D
:10281000DEC7BE7FC3FCB12E0581808D6D368D363F
:10282000B309F83B96A662BB80C6DDD378FB808CEB
:10283000FA6101C2DFC675FF6146D857FEB662FD78
:10284000021398D4FEB613A8FCDFEB60859B7BFDDA
:102850000B963404304CECC8FB205F969901177B33
:102860003868FF71C2856B650217CE1B18F9CB5C07
:102870007F018B65F5162D3F08C837EDCF363ADA64
:102880005848E6C46640C808EC6ED80D0FCDBF04AA
:10289000CAAE88E3323C31FD3BE051D31031824077
:1028A0003A08024138CEF3ECB97150F0B1FC8330F4
:1028B0003D7430018E6F8AA8FAB720F5E8088A7A4D
:1028C0000110F5F5208FF9E7668FFD8F3431CF8D3C
:1028D000B7E32FA8D8F2018EDEE3C673D3D8FB612D
:1028E0001FDB3F2CAB806FDAD728F932DD961C0452
:1028F0007F6DEF0840EDA055C4B23780DD7AD60178
:10290000F22C343C03EEF8B602173DBFB6AE100110
:10291000A0A62C824B534A09E44071BDD901B8816D
:10292000DAD4FC4EEAE7E0F88FDF528840B305972F
:10293000DEA02E688040DD2A68A26A9173BA60A882
:10294000C10570A112ECAB3CDB288001D0EE24B9AC
:10295000C8F10CBAFE0506A8FD0EC0222C864F89D0
:10296000180206A2204D7AD9849098024CF6A0D085
:10297000011B5440700D7F7908C08041AF1423A61D
:102980007BFE5E3C14A7FC78425008EF128064D5B1
:1029900015402EF1103C04B31B1BE48C40BCAE3937
:1029A00059A0A7DAB7E618FC17C0A33404B6F9009B
:1029B000F36AD6A322255F340914E7C9F711A08F63
:1029C000A51E4E04A3E081101D1DF3C3CAF8827931
:1029D000D7E748F8C6D8C341BF28CC04E0DFD69972
:1029E0000457939922CCFB6A71668B25DE08B45D8F
:1029F0008CBDAEECC428FA53855EE1BA63508FCC2F
:102A000031D5FF6C24D0FA57764950527780C6777B
:102A1000D302B208332EF94BFBC07E3D361F287916
:102A200040CBBF0A13E4DE08B6E2F8D02FFBC3FBAD
:102A3000228036F3F8A766FD849FCBE74A0B33B6B6
:102A4000706CB34BA2101DD3241FD64750FFBE2578
:102A5000CE6CC4200151AC8067F55598E9D8C0FB15
:102A6000E175FF67613EB78CFC0818D59A2108D93B
:102A7000B2207FD8D24000B1388D58FC01F9779C44
:102A800002CB18FE851B59B120A07418829240D940
:102A9000F5E85A15E7849006A21A40B40375E0845D
:102AA00006D0FF680368120D36F9347397A001BD94
:102AB00034F8429903BD0DF3779F0AA7EE8DE6BB6C
:102AC000FB8D6A42203B0AF314B8FAFBE001318027
:102AD000F43B1864669F0FFD3C2006C05E8CC30368
:102AE000609B0CFA303BC53AD6F9C4F21E100312B3
:102AF000E05FF3DFC21ED0030279E61F19BB4D1160
:102B00004D6F1C2110D5D920777240444D6430019F
:102B100088F5B3FF1E0816A221425BEC3FE638FCA5
:102B20008041100AD640C188FD74B92C02C01576C8
:102B30008D58270820841919B3FC76BF30FF4558FB
:102B4000040860216BCC8002981B934EE9BE0610EE
:102B5000192C3E5DF0401EC8D51988CF07F2F3C08E
:102B6000035932F304F3CE1BB4D33CBE3193E07966
:102B7000E0E476AE62F039D3E68139D3A0FF664B4C
:102B8000E1C1FA01FFB9D94118420EFD8CF347CEDD
:102B9000AC4DB318E561AE490321F3B58361E69806
:102BA000F9E305306D40C014D58C3845BAF3720B8B
:102BB00042702BB19E23FFCDE0D0F3582D135AF66F
:102BC00060FDF6D2802479FD424808F777BFA580E2
:102BD0001012421A406AF36CCFB5246FF83284FAAF
:102BE000D8F46B68E9442484E010A342F3FF7884AE
:102BF000EC1068FE6BADC5D6190CAAF80631CA23D5
:102C0000E0C6BC0EFFBCD25D16E498067FD7CC9719
:102C1000989E8BBFB33C97B386F898BFE0CF78F30C
:102C20008BCDD37D7EF0D6FA086B0182EEAACB3A2B
:102C3000B2F463F0040028C97D026E196FBE40052E
:102C40000401E118E08588115E7028C018E3F39153
:102C50001880B74AF83C5444C404480B098BA1FAC5
:102C60006B1240F57209A23021CD76B3850490DE57
:102C700045EE012480FB318FD3E13AE65B96A6E076
:102C8000BF03F02F16C48269EF989005B120DC1EB7
:102C9000C8F3A3042235FF60DC412CC65E6BFC79CF
:102CA000200B62410CC08FB04BF30140E697FD044E
:102CB000A190C2A22D8132C2720A4120F2F3F31117
:102CC000E64540108DB3356C04DC82405B01C7F3F0
:102CD000F8990B51F9CA2285C098020BD5CF26A5C9
:102CE000C0BA038AEEF809DFA45149A1F3FAD36A06
:102CF000E6CC51B0F4FD4A01E53010256EA09A20D3
:102D00009D852F4D264293027BB8103467F94BA660
:102D100074DA424871686E6BE75EB6E6C8FB31A8AC
:102D2000CF80F63031C544F6887BFF20FAE8800179
:102D30003153D3325E0FDE5DC0CB23808C39DF3759
:102D40006BFB394F3798E27E35F36BE6D8FCC357FF
:102D500077400110FE1E2194C284AB2F38764808BC
:102D600031106FAD4B217A22E1D28B7E9AEC9C5BC5
:102D700002C4D0F8FE30100940410818068B601FCD
:102D80008C8011879206FAC1208800A3EE70020899
:102D9000CFD72E844130C90826F9E0FD8920128C56
:102DA0008241DF7F4BD311FF65B0EF08D8F8E630E2
:102DB000B020B96A783419E2F3C007F0D316C446DC
:102DC0000B60DE402CB264F8DACDE03CE00432E087
:102DD0000258D351C6EECBD382B93041853CB0F313
:102DE000FB0C8010CD416FDA9110EA64F28B08B3CE
:102DF0005B41AD66088B66AB7EAB13D66B20FAFCED
:102E000046F3BD6412FCEDF71640C088A0B32C9ABF
:102E1000ED094BB358F34E58230A8E8AAFB376862A
:102E2000136014C5B3C63085E6E598F3C5E00159D3
:102E3000C80565F57D8AAE5FC8FD92B4089A19ACE5
:102E4000A2A1E2F3335F7FA30DC6F2C8B4CBD3F2E5
:102E50007E2866C656FF3076CBE36A1A79FFE8FC17
:102E6000E00169D60720D3299E0C4059C85F32354E
:102E7000F483DA176833B38B19F4320164FCC003AE
:102E80007A400CE2BBC6ED323CD360B93DF438F871
:102E900020DDD1A61020DF9AA2283C4B3E024BFB3E
:102EA000C7306C212DE091F780DF94C8D3A380DC7C
:102EB0008DF4BD438403F2F8AF8069DA16C2EE6088
:102EC0001CFB9C8111310AB3C8042FD4FD2509B71E
:102ED0005BC37D2A67C80602393905A3D3EF20807A
:102EE000491BE5D3834FE77F09D81941002E19C844
:102EF000C83A7820F2C5F3B8F3C8015E8B46466A3B
:102F0000B3EA77E09007E7C87810EC0FE401ACAFC4
:102F1000C8659880FBAD7EA8C29B8B0361BCB8DB03
:102F200037C801EE1C10D86EC9CBC8FDE583A5607B
:102F30002841FD516BAFFC8130082185F98935F6B8
:102F40004695C8E7988A530A3FD32BBBCC8B47EDF5
:102F50004DBC9857921A30E9A2A740B1C468F82630
:102F6000EA9B11B95D137F0630AC8481C850D1084B
:102F7000696391BB942256F8318483EC3FA3246E9D
:102F800021A415195694C8C6AFA06D7EB0FCF930C7
:102F900082666D1299C642F9E4634CFFA8F8C02618
:102FA00008D007C10605C6309E9829840C409D0FA5
:102FB000E83080AABA50D4BA4A06E07AF51ED003A7
:102FC00012FDAC41DF7F097EBF10FF6B7E20489D64
:102FD000300580400685C212097E5DF7A3AC4860CB
:102FE00010A5CBB308AF6DB101485ED3DFEF6DCA5A
:102FF000BD63B81108B8DD70E37AFEE330FF1086D8
:103000004022080521F062024C80BE3008124122A5
:10301000669389DD8CC45F0B90443001460176D104
:1030200003659324A6FAAF5E1B5F724EB30670F879
:10303000FF7DA5B00016C0027B98E2819A3CB0B03B
:10304000CEE80218440C363620DA846CAB3DD388C7
:1030500007027B988378F7100BE0812F1920C8BBFB
:1030600012E0C62658FC570524AA44A2DF3661E5C3
:10307000A5F95620B621D83B7655A067D67E4DC817
:103080004606A697FC2F1080DA965A0E617B7E4981
:10309000FB5FE65E98C01058AE0A483082B33B161C
:1030A000C4FDB804A08CBFB60167D0399364B39354
:1030B0009819C04C2FF832193EFA5719B29AA00647
:1030C000DA9F6F08210D2084771068F31A6AF99C43
:1030D000F6621EF47FEF7F1AF6962884EFC07F42D7
:1030E0001B0801A140C9D2D86CFCE72C5901FCA3F4
:1030F000A9931663D5E0F90709354321EBC583F59C
:10310000FC085C8536F390BC98677852B47EDD4944
:1031100090DBA16BBE491C100333BFFF380F50F882
:103120007396461077DC8928771C15F35DBEBF01C6
:10313000CCC4B366D53310B749E473B6F2F56B0867
:10314000C8E5843E43F98049BDC5C1F942980003F2
:103150002094C9810486F3F02818018379244C0255
:10316000792C88C0B31E51100A22E15F39070C8206
:10317000B850549BD3A16086A0C649B649B95DF04A
:103180003F26C48358100FD760419CB8F3AF031E8D
:1031900098D63C8004D7ADB14E5ECC9B0545E57812
:1031A000929BD3E519B03BD3027840BD7E08D75837
:1031B000FE56AB5DD5E42B4A8084D1F310AD03AF4E
:1031C0009633CBBB1785F7011008027DB3D99B79E5
:1031D00051786B970FF3356620EBD7170526391911
:1031E0001362B230F3321AE6C808F3B33753148AC5
:1031F000D302B826F7F5B351DF7FF6081820939B6A
:10320000F63AD1F910F09821BB38D508210365842E
:1032100034E97BC4084081680D64F9FBBE5173D367
:10322000C9F942D377D11E18DE5E37E121FBCD9874
:10323000FF69E798184D8F1730197D8618E55AF603
:103240007B7AFFD0EF23985390DE62290F5390C210
:1032500007F4811803926239632B65D94AAAF8E40E
:1032600051D38679A537190E489755916B86F9C8C1
:10327000E8C0FA2CB88E26698508200C8128F4391C
:1032800097E02079B99BA4AF342FE1F082BB08010D
:103290004F3C995C57E0C090FC18FB840530041D3E
:1032A000440067D52112C30C823AA826C0CDCA03B8
:1032B0003DC7800930089A1A9189EDAB12B3FE011F
:1032C0008811BF0C5BAFC024BCF857ECBA5108E0C2
:1032D000FAD10F23EEB0201EFB3CBC987F19F120E1
:1032E00016C483180F0FE42CF3EFA2EAD3F398BDB2
:1032F000785959A87EDD49CB235893193C5AF9AF28
:103300008CA22C29D522217D126BF606C0D720086D
:103310009F9896BB71B3796B1E5AD3DA200CF76471
:1033200018082F66C8C87838FA50518E2EC0489EAB
:10333000E060244C8292E0861974962301E0622AB0
:10334000B309F46B04C8C011D35B0C8445B39878FF
:103350008BAD78FF0F0A70FAB0018490DF0610E59C
:10336000C5C6304F8B988311E293CB38B830FEB589
:1033700024FA7E14F3C6F79B35A9FB7ED83603CE1C
:103380004BC89308BD9878A0FF13B707F16A7AA5D8
:1033900088EF7A98E48018C04DF30F63089CD1F74A
:1033A000C3013920723080E6E0C8019318E0D38869
:1033B0002FF3E7161050F8880C6D46867C98E53997
:1033C00082AFAE9840337C976628F898AE38328347
:1033D0003D98417F9798B9C058FF0474E10846446E
:1033E0006618000701625A48BBBD1788041367C8F6
:1033F0008251EDB008024DB3F32E305BCA497923F8
:10340000C3B44CFB32D5F311C316C798AEFA155DA1
:1034100019ED98C400DC30B401F698C083B830EFE1
:103420005AC507E583AFEBAFE890100517173017C3
:10343000039A98E5C8B7BE9850FF0C80105FACE7C0
:1034400098F03015E598FA5583CAC8F6988005D7E4
:10345000B63D02E6669FEFAF035E98826679F3DEC3
:10346000B83AC6A8FAE74A1226C0914296F3610A12
:10347000ED853EF126C2049856E057C89B987DCA58
:10348000B311840597B28624F40B3CC47A1145B37A
:10349000DA1113FB9F980C38FD2C6DFF046FD66377
:1034A00010B2FFBCFF23DB4B6F4C8FE3F339AC2230
:1034B000636CD3B8F906090BFF981C33668CD17185
:1034C000D3ABB0FC496C6689FE50E8CDEBB615E98C
:1034D00057666CF6BF0132A2FBF8C4C044BCF3CF00
:1034E0003CB731DCD38DEF4FC66CE6CBF8127ECC07
:1034F000B415DC818C4CF3C32D280866F9819FCB71
:103500007DFE04BF23E5813871C53E6F331F6DB367
:1035100030FD0C1E5DDF4067F5A58CFE19FFC5CCA4
:10352000E67CC5CF6C33B8FF5868ED33410CAE7FF5
:10353000DD6E38FE089E7BB102AFACC1960D9B26B6
:10354000E5FD0820A8FF80407052468BE50437DB7C
:1035500005010815E069ADCD16FAF89CF370FD2061
:10356000CDCDB0F780A66850018ED5660A3DFD0529
:10357000A13088B92B010440D04BD818CEAC3D27E0
:10358000CE03810C48E4F98025BB4D9005C2E1B81B
:10359000CAEEBE0C036CA5504468F16A347EA5E502
:1035A0002CF7BA35A076D2FD802DD4241C63FF847D
:1035B000B204FF9D38DDFA4ADB50445FD9FA205C43
:1035C000EDB18435BFA0AF590FFEE13BF4C8F8D68A
:1035D000EE80BCDC6475470BB3F6CCE5AF5B428094
:1035E0001B3CFD88C6D3D971D928F9BE17B101CECD
:1035F000362FFB913F886198BE32C20F0C17C26E06
:10360000EC6308FF22EDB902849F6E5D176172FFC3
:1036100001FFB1CF2E68EFD8FE04D7D4C701FE6FEB
:10362000B0C3CAF331481DBC96D3CAF989F36CE61E
:10363000D9B0FEDC922CB3376CFFD0FB11F6987634
:103640007A90FF099B4961F9FFBFFB0088FF021BCD
:103650005BD704F9E3843AD7D7F8FBD988FBC6B027
:1036600020D15D58B4F9FB37044FD8CCFBF91E8745
:10367000E6B37E9813FAA280EFD876FB707167F3F9
:10368000A550FF46BFBCA820E6AEB7EBEDDE018B30
:103690001903FDB16DFD4C58FC9ED62CDA750C015A
:1036A00062CD5918FE8B2FC92016C58629CB66011D
:1036B00012FAE5CBC87D3072BBCC47F6D830FDC7D7
:1036C000F7BE0163FD1E6EF7B2FE968C202DFA4EFA
:1036D0000100E5C7F96198D8FC20FFDBA5A8E880C8
:1036E000ADF5F240A9CD97F0FA2D80F5FC106C6392
:1036F0006BB594A60327D69A4F9EF09C79D3AB8FD7
:10370000D0FEA58037029FFB92408C0449B509B5D5
:103710000833F6C79DABB8FC6C66F704012008F9C6
:1037200045C2FCB41710018121A6BDA0406CCDB9E3
:10373000101602709007AD8F01CFB46EEEA0FDF1B0
:10374000B4EBFD148252514841334518A0E9024FB1
:103750003B23C0032836B9204AB3019EB3408009F9
:10376000B081431A8F123DBDB31477DC5CD893A9A6
:10377000FD66603F6C111518A4421F081991806204
:10378000700614B38A10B128E6228994B406EFBCFF
:10379000158AD4F772900E85F98F5E5E6930E82342
:1037A000BE8098EF105217FFACD601FFD9F810FE7B
:1037B000F72FB35826088E6EC2404DFD21CCF81A63
:1037C000E87E3B81D3F75B8878ADBC53C400EC4303
:1037D000F43490D0B50435875AE180B47A90FA4D2C
:1037E000718A19A3397C62FB44DA04907BBB4801DF
:1037F0001D1C80B771D3ABC6ACFE46F9570BCED5B6
:103800001B31FFBEEE59B8FF58A201E76C6D2026B0
:10381000DDD5FD8B6EC940F351C9EC26046698C90D
:103820009B9FE8FD62684202E8BA19BD62261F3319
:10383000CD9B90F97813BB18EFC03FD66D71CCF3D8
:10384000FCBF47ED66FE59DFB634408EE6F0F90462
:10385000C5BFB002B001BB5B15C8FB37766C403505
:10386000C6023AA1D950FEBF4FB308CD24CCB07DDB
:10387000FF286BC6301D6D46BA88DCCCCD7B148921
:10388000FA6280F34F083305A081FC0668F66AC42B
:10389000627DB1B7805E0C04F56B967CF96F6BDCD2
:1038A000BE18F9068BEB1ADFEDA101348006BC10BF
:1038B000C86CF1A8C3227DCF2AD0D340036878D347
:1038C0003683F3D30DA6A0F320FACCFBE673770B77
:1038D000FCE8FD7215E0013D91995DC0031CF30FFA
:1038E00088013009C027F2FD7840B1021EA74DD3F0
:1038F000A007C023D36F03605AD3800EF3D30C808C
:103900009BC698FBCF1A3F0C483B1F1582FEDD4635
:10391000F3261ADA1008693E02E0BC88F32D09A7E5
:10392000FEC5D8F9805130FFE74D03A3FC4C02726D
:103930006740BFC243EB60120C6C6AF7374930092D
:10394000B44660670C2C23D341F3D3B9802D689B18
:10395000F9463CBF851E21191446F33946B020199B
:103960002646F3E4C48919E0F12FD359E0E244F389
:10397000E63EA8FF8041305E2665970192FE8744AF
:1039800052FD92108CF3F2FF6DD3080678B4F3E089
:1039900041F3D37FA6B4C8B309F13224A50B1910A3
:1039A0007CED4EC0080193B302D3846793B3D30177
:1039B0000602424FD3DD218C049684D38CF361023E
:1039C0009133F373D8F9DE345EA98F424877B9C5D5
:1039D000218434DFBB02C9E5F328B784E53024AA8B
:1039E000F8B2FF2778D308092143E0BE066AC6E390
:1039F000212484EC10C473A5648F902D792A8DA89E
:103A0000D270B38C199F17C5468DBEF302DF5E6678
:103A1000AEB386FB4BCFD36DE03C2010F361DFE506
:103A200098D164005FC3D68240D718C4868F011036
:103A300069DB1211B2C5DBD6960AACF80544E8D3AF
:103A40004001D3160241B3C1051610F1F3D389200A
:103A500004898153BDFC4340D20248740C3E820469
:103A600072F312C0AEE6738C81B2DBCE38B367E678
:103A7000D309201F4C8004823043F37AC62456F3C6
:103A80005662A7AF3CFDB020DD16C4EFD260413CCA
:103A900080DC05F1C97BF32C08625E9873D38258F1
:103AA000F4100F6441F36AC6D30B62D3D8FE6BC225
:103AB0007F59982B0C84A924C16BF7D8717289297E
:103AC000FF442C01121072E0403093223BF3AE739E
:103AD0006B127BFBE4CCCCDD2659D37246093BF359
:103AE00026C0DACD210CEB973F2BE2C3A598D398E3
:103AF00015A3E578F18CBC10C2041882C68BD3DF05
:103B00005160FC10208415FD47DC0868D2A6359A68
:103B1000104277A70A2119A2C2B3D46DD38037BF50
:103B2000089E0DF185901000C7F3400868D3D96056
:103B3000FE5C3061EAFF98B930317EF87DC00362E7
:103B40004BE7C42601F0C680182F4DE3AB3FAEB162
:103B5000E33DF87EB83D33B9C9F071C6ABD350FF31
:103B60009B0CDEA02721605381F3804237F8411B74
:103B70009EE9A8B2430437C0101878C5CFDB22FDF8
:103B8000201014CD02031A04E5D3AFFC8489100180
:103B9000FC46C20059042344A8914194F3C104E2B5
:103BA0000B5EB85FAC0D9B9CB28408FED316C1209F
:103BB000180413B93D819F51F322C02418CF051377
:103BC000D38C8241F3300A60FA192CEB8807F09B02
:103BD0006A83785F73B8F02016465AFB100FE441F1
:103BE0003C5FB77F6C5D714185D30FC5C6E46BF355
:103BF0005E8B43C6E1F8858C106BD591F5CEB70985
:103C0000EC9597F33FF5919A66AF8035B2ED64106D
:103C100017D373AAC020F3836AD3DDC0FAB776A2A4
:103C2000E0535101E0735DC0083696039EB8627C94
:103C300030BDC2B302D72084B59826C1EB98135685
:103C4000D3E8FBEF3B60F761427230A0EE4D50D0FD
:103C5000F408FF9C2C1BE41902F08FA010D2281A44
:103C60003B3721A4017E9D9F91C85F9CC898F85660
:103C7000090AFF98E330FD161E4726EC1CAF19BF5A
:103C800052DD1CE001099DCACA4557D306FAD9C4C2
:103C90000312ED4441EFC61804031135F382ADE27F
:103CA000D0FC1F3CD52EC865410E2DBC6FE34050A3
:103CB000379E3722ED0E2822ED109A134145E02061
:103CC000BC10C651D7F3ED82EAFADB96FA16C210A1
:103CD0009804E26A3FF4FF260805636010F02C8424
:103CE00001B0D88EB5622201F580FE324402305117
:103CF000F3597C73BFF33AC808FBE3304F5BC5034D
:103D0000F898B4A3CEF5413CCEDD49E62DE0057D23
:103D1000980BB3E0B3C8F0B6FC3B728F30EA125D8B
:103D20003608B61C27E4E5ED7F52EAE004D4C6FD70
:103D30003FCF3BC8A9FB54ED58BCF1B7B850074280
:103D400018117BB305316CBBB51452F88AB3262227
:103D5000CED52364074C028479C6D9C801F9C8EBD3
:103D6000D0FF102EC8F2D20DB30DCA2084F525B2B3
:103D7000DF6978AEB3A3B830BCB2D3971040E5A8E2
:103D8000AFAD6B4073C848B3F9F830B43CDFAFBC9B
:103D90003F2CED168CED69FF18766EC808F7D2C877
:103DA000037A5AFCFB013CA007C4FFEC107F98B8D3
:103DB0008FF23201F0D3B9031059C82EF3F26BE33E
:103DC000304EEB6490FA8D88F5C62059C84A698256
:103DD0002DF55DCD08F6756F40B043D3B941A250C3
:103DE00038CDC881FBF7AD503FA03AC8C8FA74D9A6
:103DF0000626C274FF836022808144B000C0264042
:103E000030F209495A4D1DB66DC74655F803F18D7C
:103E1000F8C00448D28BE06F7344F1F9F3ACA3FD12
:103E2000C8824490087069FCDEA5B440F6D26001F7
:103E3000BD8BB13AEDC082F5B8E27AB804CCDB951F
:103E40004F5AA5207A7862C9F46B0BC3C62C12F8BE
:103E5000BC70D3C4D266EB4C8840B66441DE912C72
:103E6000654BE599D3252C03DF65C8E4F0F36B9D22
:103E7000C880FDD9C87F93D2A32080152919C01905
:103E80000BF502210C01E1B81AFD879394C819764D
:103E9000DDB695D5EF6B024298009B8BF34CB3BB1C
:103EA000E8CFFDA0CC900010AC42BFF7C449F2A20D
:103EB000E0C5CAC8F59A049CB359C8D39006D3503C
:103EC000037E56D576C812424676C89CF9FF5367E2
:103ED000E4C8A3E0B163B30899FF10F860BB317A7E
:103EE000291CC4F6980F48043CDCF320C35DB1598B
:103EF000AE67792FFCE3A5C18483D9D57F59773983
:103F0000C8C490F82BFB975D829FF2ED9710147553
:103F1000B167C8202825FBD59DEA980110E5D31F7D
:103F200095A897C801C66D9DC89BFE77950822DDB0
:103F30004024AFE9048C82513A9342C17FD42321BB
:103F40001424804910D90102BDFEFF50100AC04060
:103F5000281805FC6020140C8441C4F342AD28A24B
:103F600096F37FC608F9FBE0812C80FE05B1001EA8
:103F7000C48378FD72028805F09A6E4658F5982C35
:103F8000AF5BFFF70F640139D307B0D371E012D3F1
:103F9000C6B0FCBFC88630DAFE6662110E421D183C
:103FA0006AFC20EE879E02BBC1CE15D78881109097
:103FB0006A21B502FBCCBAC0054465D511A1D37600
:103FC000B34103B2C8D39903A3F9CBAFB04F2E448A
:103FD000ED8B6001D34C82ED46C07F7E17128C843E
:103FE00011B0CEDB96B39B10C8C008D3BB61118063
:103FF000C0AF196BF323D37BB348FD98B08B8431EA
:10400000D01657C81D30F77E6B9F5008C60140EC94
:10401000208434EF5D98059AC802CA9B65E02104AC
:10402000D3C7402FC640D681F0FBC9FB533BCC9889
:10403000AE361C31B3A6FF38FB75603C20E5D29D3F
:10404000C878407BA53D20709CDF1910F6F9CB9A0B
:104050004855D140D9C87E529BE0C0B2A897D31C26
:104060003CF30EE80139F7B3F90C2064F53285040E
:104070000AC232246997FE7DDA703001598767FDE4
:10408000FA79787AA50A56F45ABB04D37AAB840F2E
:10409000D8FD041F3009E312001881601F0180FD64
:1040A0008109300226C17744896049D6407A66FA90
:1040B000E584ED6662C124E08169D3844602C506C9
:1040C000C1CA1800C61339C6E1FFD6E0815AF56AA5
:1040D0000210B2D5D339BBD002F3AE0B3350BEEAD7
:1040E000E3E0B3C8C472E0E2F4D320B8F3C69CF3B3
:1040F00008E0FFC830311CF580E9C56280AD88BB9F
:104100001C66C24961F36613CBC8B39B8147461E48
:10411000F3D309C366C6200574B12901323C53119B
:104120000860392053BCB0E0ECFD9B4C8405801046
:1041300088B0B316C10C1923CDE08C0C310DD3F32C
:104140001067C82C844D1968FC7EF0A1B9301AB6EE
:1041500040F298CBC8BC9858FE979FF6E578F58B4F
:10416000F564E798FD7EFCCE7FB698E8FD579998F8
:10417000F9C8B3207E32589FD3FF60FCAFE03CD239
:1041800026EF0098BC98B2C8BD987023F33234FC77
:10419000D911C8E2013920C0E0C51C9040E00EF3FF
:1041A000A0071AFA5269D30FC8C658A3F861B830ED
:1041B00011224781F9C5FC50AF0C2FB8335B4FB3C8
:1041C0001AE0D7033427F698101892F308D3FF7E2D
:1041D0001622FA8045300A15412374609D20810122
:1041E0007D7273500211E7600444E61009B5023590
:1041F000B37D208811300216CC3993603D24827E35
:104200008C26FF9772D3EBAFA0FE5C775C6AB2207E
:104210007C98B823B2C8BCB8B3F50768BBDA900382
:104220002EF8E85FE0F1E3A5E0E06DEB98835F66D0
:104230009870FC7230B830E5D66265C87C058E6631
:10424000BC98BDB8840F10906BFB30D0535EDBE0A0
:10425000C080FCC56BE0413A9BC280DF9662200CB7
:10426000AE82657091FD69DC3D911407CAE0F79854
:104270003211A6AEC0FBDE4360442C964604BF2735
:104280006AB3CB84913CFCA5B6B6F52646FF452B18
:104290001990EA3232D8F871C696FF04FEE4610B39
:1042A000FFE8FB65F9869CF3672CAC226DD3B880E0
:1042B000F9C121FF98D8FF2CD1939CD1638C39F29E
:1042C000F946090D66D8FB825B190C016326447917
:1042D000D08DB1D3C1FA18247CCCB2660C8BFD32E0
:1042E00016B9CC026418EEBFA58588B38E794B83CE
:1042F000CFD87F2AACB3103E76B388FE082EB3B079
:104300008094BCC858BEFE5BF69BFEDB623F56DB6A
:10431000B8FDE7958108BD109B022CD76979887F8D
:104320009BA21FADE1AF1AABF020DB4B09059DEF5F
:1043300040500A7982E123414A980A58EBA08FAF96
:10434000D4A026B3FE4001E4B384A08472AF6E66AD
:1043500038F84BA482F2FC6753B36B90C00C56DF65
:10436000CA621DFDCD6004B419BFAC4E58CF599838
:10437000FFFE03368B801AFFC6A0FCBC40438D1F96
:10438000D2E224F3C4CFD3665410A03A20C57325DB
:104390006844661E7FD2D24380F3135E58CF808775
:1043A00098D89F5B1AF70088FC623D4BEF4002C033
:1043B0003951981267F8B3B1FF6EEC1040FBDF3053
:1043C00080E9FF10B7FF30A9B1C70462BD64B080B7
:1043D000D477CF6D3718FF76B046056BB1D0AF10EC
:1043E0003FD8EC355B76964827BD9690FD9AD1B1C3
:1043F00040C50F018D73F610FE63E23485D8B7C750
:10440000BFF080B0FC4BDDE302871C8963FB497180
:104410003588ED83846B8D3818FACCE39B0AF73529
:104420002103F8FD7988892C3A012FFECCFCFAC1D2
:104430004F566208080BB318056CB0C8FD62907F38
:10444000849861DE6C7A809F5AE520A4B8400C0DF8
:1044500005208B7A9608CEDB8C37E908FC04E5A8AA
:10446000FB08B2DD0BBF108FC4DD2081DCFEAE4245
:104470006CF10121FF630C4120A7E0108482894088
:10448000089102F3341481C6D20660D3414790B13B
:10449000FA9EB323FAB1C77FA774B1FB23EA1B5876
:1044A0001710C7AEE5FEDB7E374F8CD105FA46F319
:1044B0006F68F380EDC4745F336DCAE3F9F814F5E7
:1044C000EDBFB42031CFAE312ECF68C148FABAF576
:1044D0007E449FDB718438ADD895C8FB0DD78040F2
:1044E00029E42021A87F909849A25C266FDC1188DE
:1044F00020AD49360225F87D09ADB2010B2BCFD393
:104500004FFCDC1905A880411926DA5A4199A0050B
:10451000A0DA4A938040044C2CF282CBF2D669B3E5
:104520008005B340A30292D78C10ABB45054726094
:10453000F303FD40A7042F801098F403225240DFBC
:10454000CB2804E48B98F8B50305B70DFE3920E3BA
:104550003786C5B42168B502EE1D41DFC30DE39275
:10456000AF42B4C06D4A68FE8C88FF23F46D3F777C
:10457000574096E96CF2024B970DB8EDE37A34049C
:104580006E8E0800AD13602834228267FDCC7DEE6C
:10459000A8B8BC3DF996DC81BD6EEF88FCB05AF836
:1045A000028B36B42FCCB9EF32D7BD99286EF30900
:1045B000ABD354FF7947EBFC0214D3A8D43408EEF4
:1045C00063ECFF48FCB3B9FAC3CCCD2B50AAAF289B
:1045D000C7DBB010F838EFC4FA1EC688E349D8D953
:1045E000DBEC32D35FCCEF2E6CFFD8FBDFD8E3409F
:1045F000C6981AFF3655E8FEFF8F15E273B8C385DB
:10460000FFC88459C8B630E3503471CFFDA5FF8D83
:10461000E5F785AB65FE1FF5C028844BB908FAB1F4
:10462000C7B37B0167E5AEDE02659BF3FF07C0FF02
:104630006BD69C4EDD77C09E9B0BDCED7CBFF4CF30
:10464000D037373CD3F3DFBAB1F0FB7BF68406C03A
:104650002283EB5F0DE8A1D45E82500368F5B704B6
:104660009FFF9C348006D034F942E0A50D9B843D29
:10467000F31A40030808BBE67B60FA435F0BFDF9C1
:104680006065AD9D403F0AFF3EF83C2006F098B0C3
:104690000312700C53F301C05F3AA703D3E0013D4E
:1046A000677030C0ED312039691E10E00C16018FA3
:1046B000C61DD3BC0FE837E628FFAD34D17F9B027F
:1046C00047050021096CB91625D75BFCD2D6D980E5
:1046D000653B82D3B7C3D27BE690F9E18011B03F4E
:1046E000FEA2836024209F5501060802885C299D54
:1046F0000CCF49309DE261EDFE723D980460C23CF2
:10470000C0DAD3097023E5328C82E66B15E0818331
:104710003C07D232201978675304198807E6F04025
:1047200016F379852C399DB496EDFB9007F2401E67
:10473000DAD3240127C6F3C80319D3200FE610C823
:10474000C2FC80BF30CFFBF9D9C332F306800BF433
:10475000020F4130106711660317295CE6D322C6A9
:10476000B6DE920C829AE660FA5AB3118219701979
:104770004A06573910CEE6C60930FCB53D74AE0680
:104780001880ED7AC4180F0861119220F5E0D01955
:1047900028144CE63E23FCB001340D20CC66406862
:1047A0003A41796DA0061084F4D00868F6BFE6DDC2
:1047B00058205C60DD15FFC6239140B80104A1D3E9
:1047C0002014E0100A30D32853C61402F18250108E
:1047D0002A330DA0E621D854F841CF57EE7FE40CE0
:1047E0004FF94FD48002B206BC98CFD6D2C0F88B16
:1047F00019EED9F498620A0C2F2B3FB8E5BF0D10C3
:10480000E6F6F7EBEE5FEA3EB3ED45DC70865AED77
:10481000A6E070E8408DF33C9874050C84F3C178F1
:10482000FFFB4480081004FB9D147648F2E76323E5
:10483000F2BA644AE6F67AEAEC7CF40A70F80D04FF
:1048400001770544FD8E128CEEA1BE56FFBCBDD390
:1048500098E613F8A9E212727EA367ED24FAB0106D
:104860007F6817095A5EE24DF7D8AF5EF03FB30F8D
:10487000B0302A05043795128EE07824C0891DF3E4
:10488000484AD341FC1C900D31FC78981A052FA69C
:1048900065C5200BD97AC5B2BD8B829478EEE673DC
:1048A0009B8408BF1CFE30D6030B4A7DED2C880587
:1048B000B1C3E0BD0BAF22278BF316C482991896C3
:1048C000E4E6F708A8FC0C75E108B306194004B348
:1048D000A2304FF5DE81B71BA6E91DC95A4AFD9BE0
:1048E000112A4192E0407594CA20F3CA0804D311FA
:1048F00008E67733FA7EFB16E4D323D7C44C8D98B1
:10490000C6C07EBE135BF3714317D79163A60C2319
:10491000C7B057FE7F1374AF0C80199A26D398FD49
:104920007F211719A78BF9A6052128F682EE3B0EE9
:10493000D79820A4BC6AFDDCE635B5EF24442AFCF8
:104940002A750C3759EDED0104159C0AB230F4922A
:10495000C684C694D30DE617F0FC63FC46F7964474
:1049600076D621F88DEC99A9CEB3A4F8ACEEBDB102
:104970002DC0D7037ADD59EB98209BD860406F7C1F
:1049800098B64C54D812041CF50299ED89C13D5ECD
:10499000E0AF5016EEE0BC7E5E9833D30855FA5D6A
:1049A0006F2E56EB276D5DE480E699BC42BB22FD7D
:1049B00087DC74D6DEE5C8D913660EFBFCD3E0288D
:1049C000D3A05F1669E399F48009776D38FD5E4DD9
:1049D000CF0116BA582013EB60040CFD324222C0FE
:1049E0002E8583E2303B5ABD648C3690CFA50BA058
:1049F000B90927ED7346C1A128E0F8D78CC2BF20C2
:104A000006C1201804A35E9841E6BFD0FD60412C8A
:104A1000889F07E21EC08378C0100F5E98DF05F103
:104A2000E28BFB6FE63CEE170E02F7B3511983C918
:104A30004972EDD37EE11C48FB0F60012C8BF38B98
:104A400023D798643ED3F8804010085F7FB4097282
:104A5000266649C1EF218B36E64717F014BFDEAB5F
:104A600005769840DD64AF4023E5E85E9A64FF88F0
:104A70000BE6FB21765E02B3EF0B64205EB316D328
:104A80007F19307F509105D3572D1D1105B39979AA
:104A9000126D1C1FB3E498E62ECFCBC8F5AC50EBDB
:104AA0000308422BC8973DD41FF39B4A35FF796614
:104AB0008A4EEFFDC441FD5965027D8965D5C0D39D
:104AC000F80DA04102B4CBC8F6F66CD3845B8C30F1
:104AD0008D7B64B2CD544CB7C385ECA04047C5DD97
:104AE000019ACDDBF8F9F9ED7DCCDF32EB0801C09E
:104AF000FB1A8378BE00FD7BFCD2CC55429FB339B4
:104B000030F4F54845D3F43FE09C58D38240BFF3DE
:104B1000F43283C6A640C6C0FDEF3F8AE6A1DD0899
:104B2000E5728211F4F37415469B90F712ED744C04
:104B30007F7FC5A3E84F47248B8582E90DD5CA1135
:104B4000E1F356A2B644D328D32BFCF980453009B3
:104B500046F68B9860D02011C1FC941601025808CB
:104B60007D60146975FE98EB248C542B8AFC8C9024
:104B700050E1DFEDB093C8D3304994107315AFB94D
:104B800012248241A3EEE9FCE0D1029DF71ED0037E
:104B900058E6C880B3C81E6D97C83165840EDFFE25
:104BA000E1450949125AED8866D548EF37A5C8C8CE
:104BB000740BE62FA4CBC8FCE5EEA2C431FB46B3D0
:104BC000E862258CE6B7979810DC3AE82C8185D30B
:104BD000FCA3C820F29BD726C8F98296D3FB40B32A
:104BE000B8261956E45CC8F3A001B3CFE1329AB9F4
:104BF000101916E8804008D35EC4E0A5219744EA66
:104C0000F3406FD30A4C2FD32EE5775DC4408279F1
:104C1000981D32C323DE505FF959C8341D0499F43E
:104C200034661048B2FA3FF75D78B12CEDC2C81A6D
:104C30005F37EF418891CFC8004210AD6A2EA26D58
:104C40002308FD340EC432C8885A589FBBA822548A
:104C50005C425FCCE0F7A4C432FCA65E73FA6F93AB
:104C6000BBD6FF2E5AE05DAFEE640F4812E65DF052
:104C70008057705717CB32E6BFD022DD5C32EF9001
:104C8000172C64FDA388EDBBBEC4C3035A800C5D22
:104C90000CDD641E1024D30FE6F7C670F92C7EBC21
:104CA000D026401056ADCD86BEA0FFAF359D81F712
:104CB000A3BD900E224C2CD97BF295B44E5434B83F
:104CC00010B61EFE1BFD268089F3D3607E4F8FB881
:104CD000FC8409E332020664248854FA004C8009FB
:104CE000914D930459897D7F6ADC0A92192CB35344
:104CF000D4F255E48F54105AAFE6124122B413B3E4
:104D0000C80210A4B5F39883D314AC8CF7C808403C
:104D1000FBF9C572D4C4EF7F98E2012C8007F42020
:104D2000FB1ED00278106CF4C8082804874E19A521
:104D3000454457ED2710B026C88359C82B7029C8A1
:104D4000F3C45F2239C6812CD6CEFB8C061006B484
:104D500076BC98BB910125BC667FBF816077E8D99E
:104D600031BAC9FE5F400497ED1064C83B83B2C8F6
:104D70000BF3C81859C821C6ACEDC898FABC984DB9
:104D8000F4184C28F30919EFDC720219B512CD7B27
:104D900080A2B3098EEDCAD51B19AF4CFC6B6B9981
:104DA00098289BF399E6E8FCA2AD343FBC23C86B7E
:104DB00041088523F3FAD9A30152BE909BAC54D08D
:104DC0009EB3EBDD4CF9B2B5EF7A0B8250100AF3CB
:104DD000F64CCCC882D30AD7A528F642DCF939C4F0
:104DE0003060F7A08A5C743C11B9A04089066799CD
:104DF0009882D4D6BF7F31CA880747CCC812AE0686
:104E0000F7E58007C47AD378E6D33CA0EE77300884
:104E10005C7A6B052942D7447DD1F97EDB56B858C0
:104E2000985C26F34D49400264C8EE30FD282F05FA
:104E3000BFB2B61A2199AD776990818F0468634437
:104E400066F6F46BA4C80B7C7E7AC8020822345341
:104E5000C8C83442F0B901D393EBFF8011E7B90D14
:104E60001801C5936035009199E840F3EB02A36007
:104E7000DB6250B0BBB126137CF073C7BAD2C870E6
:104E800049EDCEDFA30805A1AD30C76910AC0A9982
:104E9000BBF383B3FF0C8250300AA9F8E0FD413C1C
:104EA00090073100736A7810BF0BD78BB165F57A24
:104EB00098608EF32E82DDCF41FE340D430952ED12
:104EC000D3F0B53F02766BC840C86BF3B3C8202B54
:104ED000F39D03B0FA84375E0602F564716ADED88A
:104EE000BC40F3E42F30B40FC9C82C7F1D30A5049B
:104EF000D564FAEF81CBC88EE856F30456C84EBB92
:104F0000C61BF814910236EF4DA58BB38C7C9FE83D
:104F100019C408B3E5194975D0C6B39E9AD20720C3
:104F2000B349D3DAA50423CAC8E53009DD0A9D01D7
:104F3000B3410C02D3DD58FBF1FF1FC530DC222842
:104F40000472F3BDB810CA4068C2CBF59069863AC6
:104F5000C580407866CF9B5D794B8E10FA7EF2A5B6
:104F6000EA173C2CF36BD301228E18C8F84C6F293A
:104F7000F43E0EE526B6444E740FD8761BAFAF6CE8
:104F800060F297F3E5FAB1FE2F3034091EF346C004
:104F900003625AF3E7C85626DC121AD5F46E84343D
:104FA000BDED3911E4807C272D9B8801AE0821EAF4
:104FB000F3D3DD400CB1E9F1FE0816E558141DC726
:104FC000460B48FEFCC55DF2C223F99B190CA0FDFF
:104FD00090AFE8194F507EFEAE941D30D380451E31
:104FE000ABF31A01879BDB9AFD45F0EF7E24480462
:104FF000601C5F4C824410E90222C1F313D7000CFD
:105000005F0A9EC88E0EC3F73A0DC0549110ED5D35
:10501000B3A339935E980608FEC60A989103E09000
:105020002C6F88FB6041F72C8005F17AD278EF77FE
:10503000D22C88057AC583B776E4BF419D3006043B
:105040008CEF5E470D4540A7E0D307F120D61EC484
:1050500057C8173D906BF3EED3584077D308C0F98B
:105060008149772B3062C4D21CBB65D3B883450C11
:1050700064E5C8FEE546FCED660340713D1724512A
:10508000F1F32BE688BE4AE1FB8081BDD2041F18F4
:10509000081F600049C0B04681C4989A0219013CBB
:1050A000F36E77BE904020F90903044E330226C800
:1050B00001C043265041791937F35120B519B0FA90
:1050C000C84AA09604B9C8BF21D59810E398B34147
:1050D00077DD65DD17AA55EFB3FC3E1D742F55F241
:1050E000A526E0368191235FD17E68D136D378FF43
:1050F0002DEB982067F712A3FFB96CF84FECEA4844
:10510000244F8D30F3C848AEF83577F5986079C5EF
:10511000DE98E3E080186E037ACEE83D20E766ABC8
:10512000574273D5DD3FCD3AE9ED0979A516E07E0A
:10513000C80FC8013820BD8B1CAFD04C6B0EF339A3
:10514000C61CFF5AB116D4BC9801AA64F9987230F3
:10515000218FBE6EB3D5ECF7435C2249DE2F2827A2
:1051600047E07A98A03382F3131A6614701AF2F4A7
:10517000FC804873EF15A5EED344F390017E32888E
:10518000E759848211E9300102B39B947D962EF990
:105190005E52187988EDAF09A18CE0CB904CC3EF3B
:1051A00002FC2513E4D32C80E60DD0F8717779A5A5
:1051B000F9C8EE100F62F698F1206EF383E223F542
:1051C000C50730B31096EB90FF02F8276F09E8256A
:1051D000ED19E2E0836DD3803C9852F3C6E29DD393
:1051E00050FA847AD2023BF2C81AE56A1108661CAA
:1051F000EBEEF9F1F8A67816A48C5E01D7DF09DF93
:10520000ACB796FA9802BA447E6680180883207973
:10521000C6828130911F80215ED23BC65820BD9846
:1052200090355340EFB858002360C6848CCB89B0CA
:10523000E8FC4B4AA2C7EC45801E840531039D263D
:10524000092322DBE33BE046C2F830EDF8F6B0205C
:1052500090FF0C68FFF7B354F7C073B3CA01ECD8E2
:1052600068046DD370C0FB206DD504967E69F3EFA2
:10527000C4844576542BED9E3040882A28C68BD3B3
:10528000EC7F6C94F7B3C7764A73F86C8DD8BFBDCA
:10529000E3D6E8F9B128E766948E7EB9F4F8ECEC31
:1052A0002B8A697139C1B0FE81660FBFDFBE6428E9
:1052B000505839C71BD661FC1F77B3041416F3C2CC
:1052C000CA05D80DC9E3D6C0FFD80401D14493CA9A
:1052D0003002E07A0C6DD30AB1FDA3E23FCCF67147
:1052E000D398B6FF598A20CBC70875F610C6F224AA
:1052F00028B610E37345F9A08AFDCCB8DF0B402C2B
:1053000067C6D8FF18F90C1205FF19824BB3CDFA06
:105310006798ED5029B3029B66FD1038BFC38666BF
:10532000A8FDC63E84C7D6FF80637A1038AFFCB4B0
:105330000AFD0981926CB604F3E138C182DC37764C
:105340001B400410E532E09234D8FBC641F44EE62F
:10535000800AD8C05EE8DB4BF8283FF0FC011B6CEC
:10536000CFF6F6C00528E38CFD098F10FD6E50B214
:1053700040B3CA401D8A7B5905602DB85B97112048
:105380002135A87BFA90FC60A1EB9804436127B219
:1053900073225ACF3FD3EDFFFED9CA343758EB5DA5
:1053A000EF9E4B031184BECED9F8FF7D82B148C574
:1053B000D2088E36E1D0FF047F6D641056B3FE250F
:1053C00096D43D9BB410146FE788FADAD03FFF60A3
:1053D000D03F68C3F3EFB1B7BDBF96ED35D7F3202B
:1053E000EE9610C1378D305B650201966540A49240
:1053F000EE7E98B0F865A2EEF339F26560609866CB
:1054000060C4B36A1DB604FD08029BEB4E10116C1C
:10541000F268FA7FCD0CB276F5B2408D36D3B8FB88
:10542000097E4B61C2BD40CEEE4F58FBC163EC7F9D
:105430003CD756B8FD206469C2FE596FE26CF3DCBC
:10544000AF235F88E8D3D84C01022DBC4C3353D333
:10545000FB8490769E62E76EAD6136AC1A04FCED7B
:105460006F20FB7AB1106CDEDD160896F66736DF2A
:105470000880DDB16E65653B380430FF338586ED0D
:105480009A5F72D75059FDDA0BB1022DEC7B90FA7E
:105490002FCB3773D43CA3B2C88CF73B37FF053909
:1054A000B86E19BB40ECFCDFD8780CEF9E506C64F2
:1054B00037F1D0F8FDC5A1DEE6BEBC225FA7625978
:1054C000C6B501FB7ECC919FDC710AE6C4D8FB61B6
:1054D000922D40CBEB666EF663B0FB80ABDC90CFD9
:1054E0004C3898A0BC6558CD9E9EFBECAF805AC945
:1054F000400BA9F767C6E8FA6037FA0829F3505459
:1055000028BC081B2B94EF4AB346457A18B0F1B477
:10551000D4EF4029A01B8CC618889CC657FA60FEA1
:105520009140869D18BBC640689B70330684EE444C
:10553000176040C0080CED0924044D38C61EA18038
:10554000FEA58FF3283EBD220280181023FCF19A9D
:105550006C88F8FB8ECC32DFB1903FB181BCEF9C00
:105560000410E130564C3040806594B98E2DF37EA6
:10557000EC2A31930FB632F90AE047F7ADD7029D16
:105580008990FF10B76D7302FF0802B548FB08371A
:1055900080CBB7EB735DB43137C6F5DB2C8BEA15E6
:1055A00001CFE3BEC8AF72CE37EB0495C774AFC26C
:1055B000ADADC5B0E355DB4927CCF8DE3177CE374A
:1055C000F3FE0638FBC933B38FC7EB6035E80863D9
:1055D0005D9696FFD15A0110C3152104AB9D80F84A
:1055E000624BE20240A12CEF58E501E6F6D438FF09
:1055F00023F1FFD84A6EB1019FB07FFDFFDC96FB1F
:1056000033519D8E6AEE40C71BB318F82361C6372D
:10561000C97CF4B648D88CAD56A84029D6B1E0F381
:1056200092E650BB1734A691DA0A01D3BB41318907
:10563000D97D8068D65D90677B1BA020FF34898070
:10564000C0109A4408CF6A41DC0900811BC008E001
:1056500001402119F720E60A30BA64232BD79A308B
:105660008B76905DB3C3CF042DD3CEF160FD8481E2
:1056700097DFC07C77BDD67648B9FFC00647F38F69
:10568000474D3C800173D0837036B4E021B997E078
:10569000E3E69005F0B31006622092E00CC64CF3EE
:1056A000B003CCFC0BFD312BD8B930412FB3527B6A
:1056B00001B130F1F5F7F3081201A0F01167FC9B7E
:1056C0008FBCD0D02810660901893BF946C16F779D
:1056D0004809300870CA4D214020E90522C5FFF96C
:1056E0000610C05B4700F8A62C8805102CD1B5D752
:1056F000E4902005C685C921CE242CF2300A050489
:105700001FABA815083A40E8EDFE2CCB9D16FFF61E
:10571000E0CD810CBAF23F468070200FE04167E592
:105720007B0F9DB5F0801685C058030F685FECBBFA
:1057300007EEECFCCD60090D2AB4FB352921FAA94E
:105740006572460369E30CF30867A36610906697D9
:10575000E59F21E0B7DE456676F52EE8FFFA1040BA
:105760004019505A6E71B31389DFA3089D20B38985
:10577000A8FE80EF30800AFFE9184005AD80113F98
:10578000C5A790856042A10DB32F2DCF78A63430E8
:105790001A60CC2E34270855AFAE3F5647D6840B3F
:1057A0000A057F7F042173BACEA2BD8A7D67FE51B0
:1057B0004538200492807F3C5A40096A418586889A
:1057C000FF094A4099205781B93AB3B0FE37A0F299
:1057D000B13C4648941940F92F2C77EB20810E38C4
:1057E000E7279048B606BDC8941039E0B681FB366D
:1057F000FC9875B9D0F9E7C521EE1EA5E50FC4DD0B
:10580000F07FC5CCBFC0C798E602B894EAB3E313F3
:10581000CC75AF66EFF905C0F74B200CE8452EF8C4
:105820005506A9B40B30C938B820FFAC4FF5031AA0
:105830000B4F196FAC75D1C22019FC3683D603AF5C
:105840001EA1CBD0B0A7852B02C048F0101150602C
:105850007744809FB3F3CC0280C00935C1F3FBEEDF
:105860004010211446C08A1D25F586937B8D2201A8
:105870008D0C0409CCBB1C607B5A98F81F30FA2DA4
:10588000454C8605D908E3902224EB0250E605EF4B
:1058900099BE3231DF22CB6609FC302CF533C405CA
:1058A00053A5E2AF0774DEFB4618100F404FFBBC58
:1058B0008807161A9CF8C4030B92469DB25FE0E974
:1058C000980BC67BD31E0831D3201DDCA4B0FE424A
:1058D00066FFDBAC04F998E546E6984691C1B3EB68
:1058E000FF0D5EBBD5D79820A6CF061E18DBC1984A
:1058F00060C3FE7710A0406C8D00994EB30A64140B
:1059000097B320F8CBD1EA1CAB38D34006841F28CC
:105910004202C080AF90D17F04AEC0D369188641E7
:10592000EB048011D14FFEBA44B410F2A53F83932B
:10593000C80298D1AF24FB32612041A444718C1D70
:10594000DCFCCFF8D41066569A207081E7301A45F7
:1059500001F00A084CA00CA0864C445862CAD3D966
:1059600098E0F8A8099BBB54C04F5AE504EFA23E4B
:105970008C8B8801731C54C0DA86047E1418FF389F
:105980008066F3F36F6B98E0FBC8A823BC788FD8D0
:10599000D166394DAB037071F9A6BEF93281AAB850
:1059A000139FF8195051E46077B798F020B7C00FF3
:1059B000807D527D45A7AB9841DC98FD08843B4231
:1059C000CFA0269F8544C1B7DB035B49B404D798B9
:1059D00092028AD3360BF84911E9C9828ADE02990C
:1059E000D08A20D5C8220C9442F2260142C68BD818
:1059F000D0983430BAFFBE501021260468B305EEAB
:105A0000F71910C2206BDBDA48DEF82650C874E7BD
:105A1000F8933A605D3FAE8003CA080DFF5240D252
:105A20003102426FA0FC3204E6AC70FB462CF2530C
:105A30005F6340CDC705B0DFC99B1A6362C766EFDD
:105A4000229DBF149E8181420212BCB2FE2230D33D
:105A500022E019DB0CFECDB6F62770F8042875F0AD
:105A6000FF519820CEFD917FD17FDC1EB250DF1414
:105A700008F2FB79FF3F988B30B048801E9C6DC3C5
:105A800030FFE181FD90D2A040B398BCC5BDB611F6
:105A90005FCCAFC4FB385360808ABC61E3BB5EE679
:105AA00051078080886D8F213930505F551525E76B
:105AB000A4D3AFE7CC02BCF9A0FB3034A20610940B
:105AC000CD68641F30C04FA61A4193688904B0683E
:105AD00019F7B8BA32C03FAF425D19682120E8B467
:105AE0008880A6B2872F4D0230CCB0A0B208E15119
:105AF0002060AF1D9820D8FADE987F17591BAAE5C1
:105B0000E864237B046D6F701108EC4296DB4C1A3D
:105B10006D56CB830C7C809BD737C8707130FFB932
:105B20007E4DA8A63CFFBF29DD8DC06866F75A30C0
:105B300061433E0F2B10B0A96257D3253020DD25DD
:105B40001B0C3610D3D6DD4878E398B1E0E1FD2098
:105B5000519419CD48A5822ECEB54608F1956EDE3A
:105B6000A841B3FBA013162D08F928CBD39A80586F
:105B700002C071F27DC0F941930410396083228024
:105B80000C53C0F90B8810AE21E6241904D84266E4
:105B90009950E116B56B09FB8A401124024717148E
:105BA0007428B941A312F732946848E7C884585F53
:105BB000D61F24883C6111000470A7A1E2810A5A13
:105BC000AFF54208FBE098F5076EF505580A164355
:105BD000F28BE450038A461D81EC5D8A127D01211F
:105BE000310E4789F7080AE4C85A1EF698200BB808
:105BF0003DD7D798787898F10C90FF80D79198E3AB
:105C00001D28E7CAEDC3FEB92DDCB4D0B4E1D396AC
:105C100075C899C871D36E5684FE375FF198A9CACA
:105C2000D9FA13F598C0FE744BBF09B810BF8312A0
:105C3000FB412148805165AF14FFBC4BCD81B3C8F7
:105C4000C09E24B388400452E0B3261BBE0502E484
:105C50003089E2B378FC775004126CB394B5A2B9E2
:105C60005998BFD0C5B88F1CC284FDB4E732D45157
:105C7000023FDE33196A2820B4A4A0361A5E636896
:105C800041BF6A345F35B610CEC814225DB3E6CB8F
:105C900028FFA202727D2C82102A3D4121AA45EDE7
:105CA000841A57D308F110192659C8AE01147D5330
:105CB000DF6DD2646E9072C00A902FD3BFF2D0FC19
:105CC000A67B22530BB9CA41FD402B650130A0D9F8
:105CD000C82BE037C8027AE5F1BE8FBB4A0B3837D4
:105CE00030205DF98C85EA3358219EA4EC94A0B64F
:105CF000192BD3AEFB2083661D720D033EF841596C
:105D0000A8828963C002982618C4E00B0CFD98D0C5
:105D10007FC6F348D690183AF82881F7B3100214DA
:105D20002BB59A5316C2E23866C20C847906903FAE
:105D3000A27A2625097A9011419212FD3202D9C821
:105D40000C6E202404E0EC2B77F68365C86C4AFDCA
:105D5000FFFC60810C20F9C877E80FE0F3B2F5B7DB
:105D60004979EB100FC0C9C58E8C8F0A85BB415095
:105D7000776567427D2C106998C85A740B9059C892
:105D8000C0401E765DC891812FFED26CF8CC0CBC51
:105D9000AEC8DDC80CA6E29F759785D0A8E2426622
:105DA000EFBC6CCC8F98CBFF6CC2C810C459FABC46
:105DB00041D6786922614009C09234B324D4DC60B2
:105DC00004B301A2CF15F1B5FE880AFF7398041140
:105DD000087A249528C2D1D42D8233C840F90521F0
:105DE0000A28F89DAEB456DD48FEBB0A242C0830C4
:105DF0003D817998F9C8D780A0D3A756A8FADC08C6
:105E0000B55EFB565D8C7A20BD98D0F9821A440BA2
:105E10006A7C7E5FC8CE306804817D17142218FC2E
:105E20007D6C1F9DD7E7F25D20DB2FC8F0980BDC5F
:105E30001B041055ADAA771508A28AF99879E5E7F1
:105E4000E0FDE7FEB2AF623BBA5BA2FCE0F2C82D18
:105E5000063332200FDD3C2DF973C802DEE041D15C
:105E6000F77E8018BB7F7F3DE8EF267C60F198EFDE
:105E7000704657E4C846BC305E98343CFF334A92C3
:105E800004C8F70FF7C58016C209F9C83BA410046F
:105E90009382AAFC1D77B8761F0EAACEDA76FFCCC5
:105EA000500813826040B933FD46C6404A1242D0C2
:105EB0006921E15AFB1FF321460108DC190558123C
:105EC000117BE8160118DE404C08043053F1B3E0B2
:105ED00060BB985E6A1558124CFF0798489108CD30
:105EE000FD248C8880FF2B5CCA0B140A31B311B2DD
:105EF000B8FE26B8306F2B1CCFF5E4010D5AEC69C3
:105F000097C87998DF87EFAE1E076BA2550D2ECB91
:105F1000F598B07B9802580F0F607219722E060820
:105F20008FF3F69828FD03F2C8BEF96DD7403C9870
:105F300003FF7F407F8AE58816FD99BE90A00C661E
:105F400004668EC5B58F0C6990C89C669010660477
:105F5000E10871FC57440D30E11817ACD1FC93FFF8
:105F60005D938389D3517F92989609350430A020A0
:105F7000C08CE3A083184483900BA26159E10358BD
:105F8000AE0243304004AF9C77F9F9B0511FC0CA4C
:105F9000DC244DE3B149D07DB97F5201A0EB49002B
:105FA00081DEE1CE7633C9E7AB679B999D6470349F
:105FB00088FC30136841AF85576B863E30584420CB
:105FC0006012FCDDC8A0C67D59FFBF909808BB7861
:105FD000BD4A48C00DC32F69C8BF268F3DF59E61DD
:105FE0001AF9E59B7998A7B58BD8F8A6C99920BF6F
:105FF000039A303C08F5C506DE985EB829DE66D007
:10600000EE48A45B7DDE6A0CF82560A665C81843DF
:106010007030CDD33872F26BA202702509D3300BE9
:10602000FBAC9AA219208853B1AB40C069E398E950
:10603000517F7C341262D385073A5311CB62ED64F1
:10604000417B98180120B3C7240E34BF28845D64B7
:106050002FD3C8C83AF884CDB3C6DDEA9590B6FE12
:10606000950102100E849857FC3B85803130BFFDAE
:106070006CC7902573B335C0ED98324033C808E63D
:10608000020B21B482567475C81880CACA0CFF323C
:10609000B01058D2FB60CF079219C80356AF74F501
:1060A0001007467FBB98E2013C9DABAE5A8AEE6674
:1060B000570DCDB830FCACC8C0A85859C8AE0D00BB
:1060C00030BD981859C826D366FC0BFE02FCBFF5FC
:1060D0009C7D0806C10775377AB841DBD7E505977F
:1060E000195A7BE6C808BDD840B604FB457CFBC8FE
:1060F000D0FB102946B30510890AB381C006C05DE4
:10610000F45EB82FBC4BB30A71C1B323304E4A3092
:106110002214D5FC08647B835C826BFC4011320F37
:10612000D8FEA0217789852993AE086B301035ED14
:1061300072B930417EBD959865BAE5CFEDC836DDC0
:1061400072772B3084DD9850036ADE98F034224653
:10615000C8AE59F4988945FB72B027CB98EDB84D7D
:10616000483D98825A5276A095885C0DDCF40FC0A9
:10617000A286886B94DBE070F3B439F398F569E894
:10618000CBFDE08090B01CE783C50F403806A00728
:10619000ADB930817F3D304E23A083FAF7EF115027
:1061A0004BF2983FC0F2AC44B3BE7FDBD59881FE82
:1061B000CCFDA009D0695746273020B38206B51020
:1061C000E430A06B04F97510EE460D11EFFE288146
:1061D000869F88E02202C040F0182123646484D3A3
:1061E0006A853566F79811B008C2A0FEAD88BF6613
:1061F000738242E384958547A738BCFF2C80043125
:10620000642CC74AA0AEA11C00E150D06B486CEBD7
:10621000C84120DC9891000A14B4AC83AF2E2C98AE
:10622000DFD7FDC96A0219BBC88B30C7D2F3F12092
:1062300069C93064F377BE7E080F0A01905249DACB
:106240008557F4373005F07130FE982290CA3282BB
:10625000C9C8AA27F32968FDB580F298E3A1F930EF
:1062600010DD06C2FD326240FB3C2479D5E8EA81AC
:10627000D05E4AE5200066EF0F9881775787998BAB
:106280003E9839FF70FDD0B902B3986DC530E498DF
:106290000BD71360ED2541B6E34BC2DCF3A28407B4
:1062A000A020F304C04210C360F80848820120CD4A
:1062B000727753DF5C09F096FCE7E7FFF1B8E7C3BC
:1062C0009AC6BDF3C40330C0CFB3C6011860B20490
:1062D000CCD3E6FF40FBE1506A5CCA6F970BF9B57F
:1062E0007D5C1EF3B0EE9001147D8E44C8A20A2896
:1062F0009AD36EF37BD3D0FA018F3DFF080AAA2A06
:10630000E1ABF6559638D6EC80F82CA3A03893FF75
:106310007B1947419C01B96DA2EC804E206DD35B87
:1063200088FCC79E669490242CE7B30C4811B116E4
:10633000C6D6D1F9FFBC9B9DB8A7FFDD642496C8E3
:10634000DF595F7FEE0B0A8C75F8C21504BBBB05E5
:1063500083D023036FB55CFD51283DF968FE080129
:10636000A9B4E2E351F126FD6A447FEF2F802FB3F9
:1063700040184668D305A9D39BFD4363FEFEB47E57
:10638000D1E666B7D7325E8EC8679136ED9FF0CC06
:106390005B7BF840FC46E386B371CC8F9BFF9B365A
:1063A0003688F8FEE2B8A1C285FF1089B6EAD0FEB1
:1063B000FFBB68B3A341987CB17022CE4B86807836
:1063C00028F18DEF1BD6B8FF3D94047ADD202A0218
:1063D000AAD0E82350488E32C8CDA8CF296E7DD0F0
:1063E000F8CBD243F239762062E71BFC7E26CBF352
:1063F0000866D2F0FFD46BC2CFDACF028C95791445
:106400005647FB9168F98096F441527121F5DA08FC
:106410000B3E0D11FACE236AE0CD6E78F6E3FCD682
:106420005DFC518DFC45633EE25F961E084DB8FC55
:106430000479ED25A711A60A8FF32CB7ADC1481535
:1064400040F6FB0222D7D550721A205CF33E5C075F
:1064500079819BFCB98005C3E824F0025000092033
:10646000046B40A57EAD1402585043A88E28677A6D
:1064700038B30491060A60F318CA4100D756110ACE
:10648000B488805CA2C6F61608500C73666130CCE6
:106490000C82E0284C09C2873901D0A50640F9A03A
:1064A00031421248858DE5D0CCF902A30845DBF3D3
:1064B000845F32F93C4496E62070B3B8859750DC8F
:1064C000265B025F166F19BEE0DBD8FAED7BB7568C
:1064D000409B397D099E195FD95F5242850F850C1B
:1064E000CBA98610EF860CC8FD0631B629E6BD2B78
:1064F000E28BADE2AA178F57B6DBC0F971DEB9C8DF
:10650000A93B9DA58FD2E3ECBE65D4DDCAE629E0A8
:10651000FECF588A02D955EAEE2416CCD87BE4B8CF
:10652000F9BDA08380798D19491CA4633C8801A919
:10653000CFDD416FF464B8B1F815D3028D727124C8
:10654000F5150A255C218595989E051BB0FB8DF7F6
:1065500076C5CE5818808F6DFD087E0D032BB6DEF4
:1065600081BC945EE5B2607E4A58236EFF3C859004
:10657000FF4A06BAC9B301BF7B42624BCD0419DEA4
:1065800023E0F88CEDF12BF45DF6637F7F788E0BC2
:106590002028C976F3D8FFE4B87167ACCE044D303B
:1065A00010B24003F4B27D2710B1FC4F5907485A8E
:1065B00025669897BFA56A48B38D8BFF986FAEADDF
:1065C000313ABD2F5BEC3988FD93A50A350E406248
:1065D0006DEB30FD889872B8D10639EDC490F9861C
:1065E0000BCB1012FDCDA02BFC30AC175BD0B10152
:1065F00018C29780C4BF6B2866A86601D8C4015E24
:10660000B40A70CF33014C8DFEBF178CF175FF02B9
:10661000B94CBA0467A88BFAA5C253FF1FFE0D1828
:10662000FEDFC16716DDF9C06A63B11485B1048964
:106630002F9DFB3BE62C3EEECB60084DD69B405F8A
:10664000C2207E561658428FB68DD8FE77ECB10424
:106650004C098C9AE3D73DDF60DC98FCA3669BCFA6
:10666000EE4080C51621202BDDF8F8F9855E1D6F00
:10667000F7D3E5CB98CF9E040490FC40988181200D
:10668000E6F402F394F2A0DDDA0867F580A81E456F
:10669000FB5A02C447F7B5C1EFEBA8FA0246E0BBCC
:1066A0009579EDE5E0C54CC6FB25F2C5BC3E402022
:1066B000D1660470BBBCF3A2BF00081ED08466F490
:1066C000682259049065A64A87A015D33EED4A0B6F
:1066D00004685BF39BA17279801CA0081267AB5A17
:1066E00008E720032CC625008750D4ACC2CCE84173
:1066F000BB053F28FAA0888D0204CF8034D5C0A006
:1067000014A71542D544844E8F21020140D12CD2CA
:10671000DF7C5E8044A00EC0092E921FE04C926088
:10672000A5A4473EFC0A0701E002446F20040C3098
:10673000DEFA40D2A41088213A023584313155FF67
:1067400041FBD165899E076744A2ED06FED32D412A
:1067500038F7F2D6C95BA762FB56BF204839C0EFB5
:106760002331FC85B7B0E98020B379F7B7DEEA685A
:10677000679FB7C6CB2FEBC9015177DED134FEF648
:10678000853B5F5F4B718B9FD75DB68038F949F2CF
:106790008898F5CF76A520145F2EBA0131B375CF56
:1067A000088FED4BEBAD106EC05A03DE28FDCA2DED
:1067B0007490D9088BE0CCB2BCBCC9E6C95F4780F5
:1067C000C2B1EDDCE3F6F330FB5B6066E410CD585C
:1067D0001A10CFDEC3CC9404AC217960ED8188FB24
:1067E000924E70E630984B9BCB01CC47B297EB644E
:1067F00035870867F1BBBF9DE5F0FE1E000195E6F9
:10680000E7FFF5D890FCB97F369A2410527301F354
:10681000CF18CF2C0460FA651976651BC76BF16F32
:106820001FAFD7051865E300C0FE467D4F82C2B199
:1068300004C3CD3F774A101AC1B66F48FA2BB61879
:1068400014ADAF10D7BFFE27FB12F01A40AD43BD09
:106850008E5BC49618F32AC0CFA001D306C0040BE8
:10686000402233F44CCB30C086124EC6216A242716
:10687000A005011EE8E3B39016182C03265A6EC03B
:1068800020690C95B3F2ABC6F5EB846DF5AEB5AFF0
:10689000C020D4F1E0A7085907F22036E0832BD9B5
:1068A0009A41FCD106E1F72B860FA873AB56B3CC07
:1068B00057F380383C1BF0FC5E70F59802231C9364
:1068C0000D6EC4085890B16AD97DA5D0F809E86664
:1068D000341316FB58E310204083819D91CBC8FAF6
:1068E000A1B36AA993D7DC74260180B187630CFF3A
:1068F000131877DFE8AB8C42CBEC5FA58C800930B6
:106900000ABF90FF7F01304006C44DC00B04C81978
:10691000F0161E2DFC7FE00173E0344B8202DE1680
:106920000C80050262D3C04C1819E2093D22B6F969
:10693000F1E9A26ACFD80601A9B5E489E077C0FCE5
:106940006CD378F7BFCEFB72B0FB4DAD27CE260BD4
:10695000F82802E119A83609037F113E3212B376F6
:1069600016CAF59C467D386839C75C502322EDFB7A
:10697000103D5202D04009DDF1D594C006A018C0E8
:1069800060B268D46E30FC81222AF520B80936FF47
:1069900005049948027FF97F048906FBE79A602382
:1069A000C545A0FB051501BCFD74CF8206572CF030
:1069B00060BFDC890CFAE8E73302C48FB3F1A5B3FA
:1069C000BC044CD1F308AD886D1E48FF57D018FDAC
:1069D000AFDBC5D206F0F383CA6EB380097CB30780
:1069E000F7E20486985CDDE0761CBE98358506E803
:1069F000980889D3889D81F3C8FFC0D857F7F1055F
:106A00000A8F46A010112889400865B466140AFB55
:106A1000FD0B773E7A05857AEBD0241A280925D319
:106A2000AF603298130C6B8021FC77D3FB049F245A
:106A3000D4FFF8396622C0DC9688F25EEEDB107E69
:106A4000B38C472F580504D116216F9304CA588F71
:106A50000802F322408211AC6970198EAA7B23C010
:106A60000302BD982C77B298164443CFD76E4204E8
:106A70000649503CF75E6B7FA7980863880700DDE6
:106A8000D3C0FFDCE0800C2006F8D87ED7404D80D4
:106A9000EEB1EF5D2521E83119F99E982F67FC5C76
:106AA00040EEDA1BFB15D78DB97923E8BF88413B4F
:106AB000E3045859033F3565EA4CB0C9D1B1B8A7D2
:106AC0000AC21C01405F334E090290FBFF45015092
:106AD0007F0A3DDDE05D19C818F04EF34D8431DDCD
:106AE000B308738E231DFE30A489048022C4269827
:106AF00048180FF598C077635A48C20B6AE62DA86C
:106B000021C210CECD2E3091CBDF807DDC6405B369
:106B1000F75F23BF320D0DBE40B79698AD66027C7D
:106B2000ABE6E650FEDB579380F8C5FFEA1006F0AF
:106B3000201E048349F66894656F304B27EE6E3053
:106B400085FCC1F43A1EFA0422D38FEAF678B360CA
:106B5000400C80F03C3458FE8B77F4D94050B3AFF2
:106B60000D9CECF314027730CC4820DBA96614FBB3
:106B700043F86FBE720A811B2114BE4213C5739283
:106B800039E718210BADEB4C0805ED7C77E3827FEC
:106B9000EE6B20F4FE22BD7646440605CA1E00E7D1
:106BA000E71F708B29C3636D801038300608427967
:106BB00066980413AB868C17B108D8B4FCE230F0A9
:106BC000981702F8C5CCBDF13944AEEB595D419937
:106BD0006BF3070D4072E0A071D391C7307B980131
:106BE0007ADD2007ED7E38FE9DB95E2084CA40180C
:106BF000AB6CD68201BF5997025E9F05B79D87E9AE
:106C00009880B62B4DF74568A4192611D1D4801170
:106C1000AF2D30583F5F286EB442E87184C4CDD99F
:106C200027105BE3AE249E64106081227D7B3040A0
:106C300070FB77398602146A1A229ADDEA2CD1CFCA
:106C4000F7AF63AD723675DB099F561A232F38A153
:106C5000EE01A440CC3B440A622FB9156B39B7F65C
:106C6000FB980514ED0148FC3E03FF354DF598C433
:106C7000E22966D7CB98F798143DF8C377730AE9F1
:106C8000E0C0885EF264796BAFBD98212088F8C7B8
:106C9000F7E538FE984B7B01BC26E5E0E4B0B31A7B
:106CA000131F628377B38982944131B35ACF9678A8
:106CB000FBD9C8E8100361863AE537FB02E6C84015
:106CC00002F494A0264B9382F63C57F3D9488A6687
:106CD000D1346625402423E566A55890C83F0B6053
:106CE000840C0809F72001C1FE0CE0AC82ADA700BE
:106CF000AF9EB310060108BE7FFDB29FF9305CF66F
:106D00006723380599CE23CE972A37E7411012A47E
:106D10000C0C1F040112D2F1FF7D88EF6FC5C883F0
:106D2000E25DE73010201EBBC4D598E8F67FC4634F
:106D3000F8FD40070F88F0816E26D078D3C4011883
:106D40002D7EA9B2C84A0CE40DB068647517AF1760
:106D50008A9B41E9EF79F3B166BF44047FC0CC66FA
:106D6000F863A6E9DA42FFEEDD8520CB2593FC67C8
:106D700051F3B3A189DD1F7A1622BC98D5B305B4AF
:106D800082F34C65B3A07B981080BB60633A877830
:106D9000BBF820C87A140842506BB34D04D3C50623
:106DA000EE1AE5402302AAB882D3B350D21803FFEB
:106DB0003BA8A201348206989708FEF9F235D31059
:106DC000D1B4AF7B5E983B9FF0FF6E167DEF771DD1
:106DD00030F67C8DEB11543EA74812BBA80A887E82
:106DE000FDBEF9B4358D86CB19E7C22468FE7F77E6
:106DF0003C418079557D6C775106C13A7BC481FD59
:106E0000E808BE65C812FC0249CC7FB9CD109B0DC5
:106E1000D61C5E4D0338D342DBD6B878B344C6BF28
:106E2000FC2BC8C3A6ACA5C8C1347E452468F32298
:106E300076C8FDA001CFB21F02BFB0AF05117FE23F
:106E4000601BBC1957D30D58C6103C872C88010213
:106E50003DCAF8FCCA5E4B70B6210E4601C03BBC71
:106E6000DCDF4DBAF9DA06C94A2FB6D837C484FC3C
:106E7000E9D27E04E12403BF6E60FF118C840931E6
:106E800001E8FD723905EF2298C77A463C88071061
:106E9000F2C55AF30B9BAFF38D070AC080E049306F
:106EA00090D3B5D0EC6EA03A34D1251932E4E0C6C7
:106EB0000670FFDB450AADFCDF66EA1D01DFEF600F
:106EC00012FFB66FDCF3F346CDDF7B0AB1A3FA0EF7
:106ED000B49A0BB9992840BF7510C2B0399659BB06
:106EE0000DA51080BF969859A649B326E427D3B3C1
:106EF00080228F4430DE407819AC46D28A43F78D29
:106F000095FC86ED4D02200494796692B3FF623BB6
:106F100028A00134C006AF92DAFC637A9811BFA0B2
:106F20000AF5410B2A04E99815D4BFF9A8BED0CBC5
:106F3000CB4235F31573FB5237DB996A75C37DCFAE
:106F4000BF9798227D40AFCDB520E9FDE406E0B4BF
:106F500088F098AFEB64BD8B0EB70214AF96F4F2D5
:106F60002BB319E8CD93F5C218C06BED9880070BD1
:106F700004B34EA50DB308C006F10440F50B02E7BB
:106F8000A5E64D22FFC29C21663C6601739D7A0FE7
:106F900044200514AF4035A5F6988010B4157F59EC
:106FA000420A0C848520DE01A11923C41BFD0B5F5E
:106FB0006B9842C153C723F34C0D9066D7400179BB
:106FC000AC271D38F6BB82CB9868ABCB97FC126C14
:106FD000965913F45A353BD459FAFF0F32778298F9
:106FE0007FBA98A00510CDF5831B39F84BBDBD8E37
:106FF00022DB0D087A98C0135CA7C81916C801AF28
:107000001A4E988056E8FBD3C9B1E3837A7830856D
:10701000C066E7D61B9965C9E2DAE8CFF298327EFE
:107020003DBF6AB5FCFD4680AF8C98B326DD19588C
:10703000FBEC8C946A05E56BEA310334BAF298FBF9
:107040003F273E628488204439C11F2202DCE0F9D8
:1070500080031808C71A437899BBCAA247B5F398AA
:107060005F3DC87343C0FD73FCA02104C106904B73
:1070700018F416DBD598439FC80DA005168901FFAB
:107080006BD5D8C65D7780A047E982B3BB043E15B7
:10709000475F7342DCD3F2E03C3963ED3BAF76955A
:1070A00078DAFC5FD97FD37F61C040DB1EC87C8467
:1070B000379FB3AFFD285533459580C5CD10401C93
:1070C0001C6F83AF38B5BCD5CF806B1C38FC2EBA93
:1070D000E7B2481805BF232FC8FDDF42BE5A1F9EE6
:1070E000669BA75566912011F61040041AABE53453
:1070F000FF5F05F40B61440CB41B70FA69D9E082A0
:10710000CFA38BF88B74BAFE98045B932C1AB3BC94
:10711000F8469573709D985540842BDB13EE5F2FD6
:10712000D3D7A088EE5242D04F1B60FB6F2E98AD94
:10713000DEAEEC605D07115F1EEB980273664CEBF0
:10714000F51D4F92942CE0BC98F2E063D39001AF10
:10715000526B811664EFB4C9F29868FB1001C37BCF
:10716000FD3020066FB6F9FB7863B35F6DA8064467
:1071700076E6C93549EDD8FFEA1980EAB12546CA55
:10718000300D19B308A9D399EB6140F508160594A1
:10719000B3774D989082F9C8BF88DA4BC6D0D5AE88
:1071A00088DDF7A591941417F7B0B881222E34D258
:1071B000B7F35957B23B20A0133680FB12908218C8
:1071C00003279F304A44032814E945A81192F8790F
:1071D000D80B73CBFEC2D44ECADB665CFB28081505
:1071E000FF74CB09AC24AE503010DDA6E3941080C0
:1071F000FCEDC80701338C0F5D3733F3C2D0C0708C
:10720000CBEFA61C0817B373BCDBC53F7980793080
:10721000ED59C86FC73083C7AE20ACABBF8EFBCC77
:107220008026BBCF505E9841E34A96CBF4BD5B8489
:10723000C601246A66735682C5356608CCEE1440D2
:107240004B1ACD667D9890E30822014F88DC02043A
:107250000879662ED64048652047FA0246690C0533
:107260000BF302CB0882B6CB66EB15FFBC8D3F203B
:107270000804890210A081EF4981044A87461A66F2
:10728000EA02E033F031ADF83930315C3077265D19
:10729000685390DBD5980BDD8E2007E2668252762C
:1072A000CA4B023FE09630C8FC3033E2168358EBFD
:1072B0004003603BC888FE7F17D205F89806DE9829
:1072C0007F2019053FBB9ED002C8E1424189B344EB
:1072D0003CCFF32EF2C8D5B3019B404E20CBEB97A9
:1072E00030C28AB3DBF861D6049CBB2937DB40721D
:1072F000F4B0132F65E3CE7A6B403C8152C1B3C822
:10730000F80A00C68CFFA7B3EE6F70B104B6D36065
:10731000FBB232BE9FBC4BEFB31C8DF357B0113E96
:107320008EC667BF7828C6C0D3DCFBD063A563A434
:107330004BFFF6C4672F7438D6EC68FA2C223966F6
:10734000F84CEC67AFF87139CA88FDC78D669EDFCF
:10735000C6E76EF0C715D680F6CCD900B20896E71E
:10736000087BB3062EDC0E40736EE76CC6B6405643
:10737000F3E0DA499131B1B944B1F395CB3002630E
:10738000BB732460C60D5DF331FF308D7DF99C37F2
:10739000639FCCD888FFEFD9CEE7099908CB992114
:1073A000D7FAA0E9AF85C2AFF7CFE50910CBEBFE66
:1073B0006493020614ACFF18BFBF63A947F478A317
:1073C000FDF373EF3440DC8AC797A42197C7DACC6A
:1073D000854961196EEB8F403106021D7128E08CE2
:1073E0006DF93E12C5D6C21226EA62BFEABDFEA200
:1073F0004128FDA1DD1C08630A66043FD3D88540FF
:1074000001C5F2B2A60853EF1728FF647D0FA154FF
:107410002C39206183405EA840BD5CCFB5026B096A
:107420000481CE9B6FCCD0F85C7822BAB919C1A484
:1074300007A090DA81042C600540B43C0DC07D2784
:10744000A70C6B20034823F53B709E507C0B20411A
:1074500061F3BF15E0FEDF24FE082241381042D060
:1074600047C26996BC99F046CF7BB3A031032C0A82
:10747000E580010889205D03098C0E81B5B4413394
:10748000F318A9701B48FC2BEB57DE446992849FCC
:1074900032B508E0ED0E06FEE5334210295CF4310A
:1074A000F8FC12F644F2DC1B20046CCF62DF1DBB3B
:1074B00080A27838875782DEC3F347EAF43AEEB900
:1074C00024FE31B68F375E585020B953B8E68E6629
:1074D000C7CD26CE9FCA900EF4CEEB53C817578C5B
:1074E000B2D59A08DF0C79C2852D9A0440EDA870B8
:1074F000FA95CBAB202991016308BC02ECC5AF041F
:10750000AF6E01F9FDBF01B9751FE8E64835F9D93D
:1075100080B46BF7B6EC3C33D051497E02D1D83001
:10752000FDBF2C45202CE41940EC6E78FCE52C4086
:107530008EF9978B716E365B58FB156DEBFF4C5DCA
:10754000BB65E94A1BF72C9FFCF598108D17625913
:10755000B85E347788D5D3C7A104435EF70AF9C66D
:107560004C7CFE31753FBF18F74004F6ADF8D72CC0
:10757000B677C8B4E0F0A50C57970E0230FDDCFAE0
:1075800058FFC4566BF0E81DCB7D4411ECB0480B9E
:10759000884DD830F95DA2C3C9C5DBF298FF63EB13
:1075A0001E31BC9D6FD402101BBF45FC24EBC2D51D
:1075B000B00495FB04A0B7A9F96159B675BF926FE5
:1075C000669B13F1CA8DF6FF20D87DC73446BCE513
:1075D000CF3FB52C1577EFD90AA4C93FC8BB33C03C
:1075E000FC20F2DDE1406E706400CE64ADF460CC4E
:1075F000BBC655D8F9CFF5120485BEE0B90A87029B
:107600007676D2E8FFE22CB2C2A3FFF5BC40663624
:10761000A0F0F8EB0980F64F1343A583F3AEA54421
:107620005C50AA5020C7FDD1B8B1FB25E7029FF2FC
:107630000088C79B5701805E80FEC6CCD867B7978D
:10764000409FE0A47AF6ED30F80254CE807B781D9E
:1076500017AC2B08876408801078640A40FBF5C8D3
:107660005BDD1A2EDC1185C7C447C6B2D204E0B375
:10767000C5BE525AC3A36E0434F152F8477B653B32
:10768000B6915DA5D9EA19AE6D14207F7F809B412C
:107690008150C28E5D05DA4E4801DE0A6BAE3F06B0
:1076A000C030E7F80C0360A718B82802122EF5487E
:1076B0009203DB7590E8560467F82A285FCBE8351B
:1076C00090FBAD0782812134FA63D0CA8070EB68E9
:1076D00049B003AF46D1B3209FB3C0276809648384
:1076E00001488944C520AF25EC84C95541C3C488ED
:1076F000813E4628FD20808E9906C9FE8439C43B10
:107700002408DA20102E2908F9CCD64B3E4427E86D
:10771000633CE2246DE540FE4F0FF198EA09FD302D
:107720002E9B23D85BC1B31754B1B30108CAD7DB72
:107730001EC9BD9F04779E67B7A220F768ED90F938
:10774000CFC26ED2C3809814C53A94FF6DF784FA05
:1077500056F510126E59025EB0EF019DEA2A406C98
:10776000BCA8FD43677BE12808611956E67E4F827D
:107770006AB3FA85DE00842BFF482FB4E280B84359
:107780005F66FA6BB2739BC282FFCB912FEBD1D7AE
:107790002110A89DFEF3C5B2CF580EDF2CD808EEFD
:1077A000ED2B58FD5651066F5826BAB43059E0E615
:1077B000A6BD0CD8E0FBC6ECE7206336630426D4F4
:1077C000D968FFDF1C6EA8B6095ADA022C88054D6D
:1077D000A64064B6CE90F952B308CD2FF3372632C7
:1077E000AEFDE5107682D767FF98FE026176582FCE
:1077F000B0CFEC83B8FF2C59B401AD710A011B4B1B
:107800007FCB18FFFDA001849006D0E3EDE7A11423
:10781000B885F3B6F1350D19EFFF97818491DE42FB
:10782000D2F6B42157EFD03AFF4060414DC63466DE
:10783000FC8A7D41855E3DB604CF6AD8FE80C001DA
:1078400030C206C0981EF478100F4A6601F3041780
:107850000310020C6C623CE4C760A3EAE0CD2D4447
:10786000EED30DC403E3C6B97097FB30EAE542B32B
:10787000DB81D72110160AE59F02F46E66226C2B7D
:107880004047388544C28CAF1EBEED41086401C636
:107890005BFAC0D0F981300A9AC097986553028C80
:1078A000F30F49F3580813F96021208091E567FC34
:1078B0004D9695495F40E133BA93EB4C05772038FC
:1078C000FAE0E0012CF707F0003919100FE25D3300
:1078D000F3F2F3C0A68346E401C45D190DA004EBE6
:1078E0009E18544BF00906193FF30FE0813C1077C6
:1078F0002F7D115FE304F6EF9CBC8118035FACECB5
:10790000880130EEAF99B5E66C6D60108ED6678356
:10791000ABA602F9E250FCC4FD3011100242983AC5
:10792000E0208C04D292D91AB39A8BB3200CC6CE25
:107930007DB309310802C0E6B3E019330513FA4CF0
:10794000773939B8FB30C0AFA051D21AE879A567B2
:107950002610128342509903F32154B6355ABB24A2
:10796000B2F81284CC2060620A49DB687BE74248A7
:107970001C99D30220E60BFCFD6826639EB56A00C5
:107980005EC96DF679DEA565FF2858F9353308E73D
:10799000C579C87AA5E4FF4E9820A40311EF599841
:1079A00030C9B366ED4FE0401E0403B762F4981E81
:1079B000A2D3DFFAECE817390405B9374340E8EA07
:1079C000CBB902186E57CC215E85CF6427F825B35A
:1079D0000A44A504DD23BA661068D388C712F67D71
:1079E0004BFB7B14300112FF1660F508808145FFC8
:1079F000E8400298088F60049224937ACD51B30531
:107A00009C7A9814C9D01D14142500E1C604907CFA
:107A100009FC60413C1C05F1DD5308DAB1E0F79840
:107A200005B120F01EC00378FD0BE2013D887B9874
:107A30003D905E989B12E0195F7E98B02012C803BB
:107A4000014FC6B92C08C8E5FE884013D91B2EDDAE
:107A5000F5A581258D41580DC97E8219EAFE981D34
:107A60001C6D666C19EF4020147F5A80401008FB93
:107A7000FF909809B346D442977796A5F95416C05B
:107A800082B3DD0861F1ACAC10E1B3D3197898F69C
:107A90003A036422DF7FDD4808FA93846FB9F0FD72
:107AA000E14A45E54208609A78D2BFE93ABA4068AF
:107AB000CEAC01B4CEEFFEA00134E78042D476090B
:107AC0001019BAA040ECAF6E2E6BD9FEF8E6353532
:107AD000C51FE6FF79DBBFD673D7960C4AABF0DD46
:107AE000F7C0E598E48B9E77253060DE8ABEC60637
:107AF000C14016C40560BA9014FF53984004D0FAF0
:107B00008528844DB80201703C838788711C72A956
:107B1000080614010F503009660B8597BBA5C0E617
:107B2000088840B382DB500A0A2840AC48B9171FC6
:107B3000FE80413001CF26C1E0004360FF228081FA
:107B400048301016C1F328180023C88CCB0230E649
:107B500037B5CD04D7FFF998BFF266C0288AB98936
:107B6000444FB90A48FBE0FE013C8807F02016FDAF
:107B7000CB8360F3F923C8F48378200FE60D9B9A3A
:107B80003E22FB62FC98057AAAE5F068F3C85BBD6B
:107B90006B3C3B52FC84F4FC29287F003D78F3AE1B
:107BA000662ECAAE7033300866D3D3D69883DF63AF
:107BB000725981949282E6D748FDE79912C0849861
:107BC0002EC0F6980531F1B3198F010C25C519891E
:107BD0006DE31086D316479D98C73037E658FB7A79
:107BE000C50605102BFE68C3D2EB01A02BC8973049
:107BF00008705D7B10116E190210F4986936899730
:107C0000D03D33D562EDA825B9BD8BF998A758842E
:107C1000BF9BAAF1CA92F3D798FFFA790806F22D12
:107C200084C5290C2D3E7830B5EF825AFC66F3CA24
:107C30008581B730F5980CE351D314AE805CDD023A
:107C4000B9C548FE2BEC8274DC03330088C3B8ABA3
:107C500057FF246008DCB60CFBCC641108D7F70989
:107C60005D83ED98444CAAED0A88F30C98B99AFF0D
:107C7000193080A11DDA623F94448211B020AC100B
:107C8000ADBB46A312D78048587E87DA7FFA982189
:107C9000D7EB1D933083B40C7675C8E8F9EAB2903F
:107CA000F398B2C82F0BE041BF3C3CC8D003583F0B
:107CB0000F64012C676E4926C8F198E06B95C8C621
:107CC00030B9C81EF8EE9D11654018DF8C7F91D247
:107CD000D010F35F8833C57E80BC98F3F7CD533A5C
:107CE00064026FB921F8E48EC234C04453397E5720
:107CF000C82B3001C58B0CAABF14D5F88A6DE89843
:107D00000B3B224C56A44808F2B370B928FF10A2CE
:107D10008480FCDDC808F4F9BC5D09255BFEFC5DD0
:107D200067F16C7B988442157DB46983A67CC8504A
:107D30004803602B0D99F1E8F858622B35103796FF
:107D40005624BF290597E67E6E4EBB96FAE097460D
:107D500007FD32713D716A7517732303107F195D3A
:107D6000A59CA9DC304981B416726B03DFB964832A
:107D700078D3A7E2B9D8FE2CCE0402180844E691C5
:107D80004101E73910180802112D0C6C75B5F3325A
:107D9000B1DC4240508876523B0A57DB562A4F8E60
:107DA000FEFD8409EF900806CFC820118CE0820107
:107DB000B07326C004D3A3FD601124824530B2CA3B
:107DC00006D5198377ED7F603F708CBD08A52259D9
:107DD000C85B5DA481B968E519412C26F9C85EA588
:107DE0005ED29690F39C23AF0B167E6467DCC4468C
:107DF000F403B04012F56BE998B00CE5C80319F331
:107E000003B913FA880A105087D424D65EE5775256
:107E1000842383ECB1C85D6FC2602059660C99C899
:107E20003AB908A1CCC8B02B164CDCC812B359C85B
:107E3000C60219DA1360705D5667DFCCC030D65BBE
:107E4000D7BBB3C004506CF7C80138FD64D5ACD4BF
:107E5000A7C89A0DA0015E8B3DF40240030662465E
:107E60002B69B31EEE63AE496D032C0405E5D3D92F
:107E7000C8A524B90871308D7998B9B39EFF2C66D6
:107E8000FCE5C8F8FA46A786A57E6EC841F58B20AA
:107E90006AFC795DDEF07FD9A5ABE298FABD980364
:107EA000ED62200F0F54D3CF4CE28E30F96B0405F6
:107EB000CFA5C9C8184514E08B89BC4DC48101CB3E
:107EC0000486EF37654887FE44031360DA040C89A3
:107ED0003CB318451DD9B18166BB50DDA52408050A
:107EE00074FE9EA18709064040E68E602F0C820535
:107EF000D8300A871B307608415AF46E96980DA147
:107F00003F7D8250300839FCBB6032C8F146B93041
:107F10001059D55E8BD7B1009198F3DC236A6EB609
:107F200044EB5CCB5D8B30E2F9B5CEC81EC494E364
:107F30000BB90BB0FBDA8440F9A51166FA788BA275
:107F40004A17DA1CFBDF3BEC6FCE3C6E66FFAFAF2F
:107F50002634B9E2F81411F9FA46C022988D5D9ED4
:107F60003F51B01026C282F91801086120B3C6093A
:107F7000306DF6466019C194A3B7226BB3049334F5
:107F8000C882B9D2D8FFA7A0FCBBC883304784A25F
:107F900090F3F198D04BF3343BCBE546FE8ED2659F
:107FA0001949F5B78B98D3FCE5B7F604D838FEB776
:107FB0009F98C64A675B649AF175FE9ECADD28FBEE
:107FC000C64AB9C8020EFEDD64F0EBC561CDF3967A
:107FD0006E48AAF8810BEDC0AF203698EC17E0A3ED
:107FE000D3DBB7F6383BDAFF28B2D5D33EC8412100
:107FF000104095F212E58BD3B3F30400566FB59998
:108000000548E7F8735D0B022D66541A193C2B1CCA
:10801000E0917C98FB80493097E193696F7BE84061
:10802000902BE14BCF3DC8040C807D26BF5B6CFCE0
:108030007FD9E0089F32BF58AEFE6FB970FBCAC847
:10804000F4D204F3EA100F62B088DD07F2C7303BC8
:10805000F3413C0011D6AF01F070E0C0038BBDCB03
:10806000513A8EC4834F0CE2B90890FEBB84ED12E6
:108070000B66C4F288C071C48E08FE31233FA3642E
:10808000522C668F1B2E66EFC390FA5646C24FD510
:1080900025044C82E605310119085746BD984C88E5
:1080A00009819D977AFF5F084436E98B4019BC53DC
:1080B000B3B70FE880FBFCAFC8BB70C69843854AD6
:1080C000F3CDCBC8FC9859E4AEB3A010346E4C028B
:1080D000E2103644F398CED3D674C0FDC532C8CD75
:1080E000CAE2DB0B7E317486FFC0FC32F2C5CEC81B
:1080F0001C10BD980F29BEF3207650C8F3D946381E
:10810000CAD18522D316F57860B75717A698035AB7
:108110000E66B93CB3FAED700F100840D38D4120C4
:108120005F742BF3F8C142082EF6988540CDEF1707
:10813000084130BF859E3D53608101DFC798D30160
:1081400021AE30640320F996C4F0468E180AFFFB76
:108150002C8211811046FDC12448008B2068AFDAC3
:108160005902F4B9B5EA3FB3DB98049896A340826C
:1081700025F33423D0C58C4F6DA0FD6A0F88DFCD69
:10818000984DF3FD9808B4076DBB90037B8201BB4B
:1081900004BF9B1EC0037A201608D7DD98C0831841
:1081A00079982ED3402C66A34F46BDA58221F33F7C
:1081B0009023034033F380C90568BBB5D05D5E886A
:1081C000EA98C2F36B234415CADFD301EC98087018
:1081D000C2B329AC12CEC858EB600AEF2ED20B23E3
:1081E00098F7081362012DE022B8D9D5B3842B0685
:1081F000671C860810F661128C02DE98D70B60AB04
:108200006B81B66AF82FF6177F187DFBFFF8FB5ECF
:10821000935DBB5CBC771920C6F372AC22C6D8D381
:10822000B8F90C121DFF98FF248D1993C6D1383967
:10823000C4C9FA6090662CB3373CC559CB7BEFF0CC
:10824000F908011933448CC0B3E0CCEFA6D3C2FDCA
:1082500023048FD6CC9859C86B800811F59710AFBE
:10826000A8970878DBAC6B859628BAD458C2DFD1C2
:10827000CC80768BF32980FD6718EE4DFB224810E9
:108280004BED18190D96FF107AEE88C335B320E632
:10829000FB21DBFEFD1AFBDF1157EE44E0F7014442
:1082A00040672EE4043FE2E57FE384CB6C40274047
:1082B000953338AF769DB8FFCAEC04FA06F0CC7758
:1082C000A0ACF28153C8D7EE3F0201205EA80A108D
:1082D000CAE5AD10A7E6CCFEFC118600DB10F0FD70
:1082E0001B75A0CF8B4B9005E83F5E610CA002256B
:1082F000298C4B8901657A10E4D0080AFC16092004
:1083000047136E44B281564504201A38D484047E43
:10831000241002421F18A0839B005D04BD85060542
:10832000A84AB0B3BFE534AEFEE65F7766BB46A8A9
:10833000FE50BFE74463DEBC6EB728C082626F8127
:10834000A2265945015DF1D7F8FF5E545D7F6D911E
:10835000C03A47D01BD0E6232FAC4BFEB7B539D37C
:10836000FAFC666AD002DCC6F33E3CB4C53C52D788
:108370003B23B8FD0C7AC6CFF52E80863DB1B78081
:1083800016A7F527FB48FD1631C74FAE80317D8615
:10839000FF58FE5D0FFA96400896FDBF58ED89F62E
:1083A000C3C7CDFF7AA1F5D3E0BED9E3FF9A6182BE
:1083B000FF90CA3319FE03CDEB36759F048AF17D19
:1083C000871A1567962EEC96102731CDFE6C5688CD
:1083D000FB71E0046C1563BFF47FF675F8FBC6E62D
:1083E0003EFF6798BB5BABFC0811C87B0C6396999A
:1083F00070FF326083AD5A98FE873F4067F998BAA4
:108400001902C2CDD8DF018A62E896660451B475BC
:10841000A4E5F3D6B133F61F7F56B1E6CC04F7F8E6
:10842000D3AFA536F0DDE720B181903262E6EE539E
:1084300027E8FC01FD30B7413F72A816F78CF3BD69
:10844000B1E3DEB916B9A07FF6320680CBA1017385
:10845000977EB77358B002F7F66FA8F9FCDC2C6D65
:10846000FFB3E8FC9AF018CD39570267BBA3B8FEFA
:108470002024A2CFE3F43017C7F776FF689979D2AA
:108480001928BFFA6676BE80C77B9CC85D64BD6054
:10849000BE406C2111E4C93067F12EE6CDE696E6C8
:1084A0009FFF9FEB60F910ECFC28DEA38010F09C8E
:1084B0004D42D0B75C912025B7FD2FD92C9BAF5EE4
:1084C0005C9411620CD8F5888AB4407186024143ED
:1084D000623F5F4CC3F0FE03E010B914F3068A124A
:1084E0008B55B0FE148E868A0A66B328EB05D04DF4
:1084F0008F277C7020A0C00DB00F158002184DF2A0
:108500004441ED5E1850FF25A640D498FBEFCB8781
:1085100091F2D8062401268A93027CE42A42188428
:1085200081DDA42DFBBC0252367871A0A1120C276C
:10853000B438069140D8D18BC184771050F4B1EC97
:10854000B8A8FAEEED8908028549D888F5B1FFCCC4
:108550002C34E3E6CD3F78308F204A3508D321AD67
:108560007BEF35F722D6526FA93E80B20110BBEEE9
:10857000E1A3A2C9FB0A27FD12A8FD10287E128CD8
:108580003BD4AD24005F7647E1FDC089E51EB79A74
:10859000739E02407BD3ECFBB1127E2308A1FA0C40
:1085A000C24F26019064FCCFD5DC088AF2E908F3BB
:1085B0000D1ADA46EBFE0486FF98FF960A40BD6965
:1085C0007FC9D083F3A3097DD6F34810EA1501E3F0
:1085D00050FF960862FAAF67992DFF7567F77CF038
:1085E000FF634BCE4012F8E54C47CD9E3F98D8B084
:1085F000F987566430ABF8181DFDCC2018667EFF55
:10860000B101BCD97B205F9AB228CCE5693790B123
:10861000FC9CB097AB6F4C58DBFB99EA1B459B5B0E
:10862000F5C18FFFC680FEEEA00134E3F3F7480DDD
:1086300020F3708406D03D1A400368E6F37BD11125
:1086400014E40426D21AF4E060420D9AA680D39274
:1086500048D1D330B510DB9634C9C64D05BDA860EE
:10866000623F0CE498FC80AD5F07F00004CCC003CF
:10867000F00CC2F33CD006C036A386F310729DE026
:108680004110D381E0660378E0E051E0D37DEB1E3A
:10869000D3C6D378F91C8810E0180203ADA4274094
:1086A000848684335ED9B340ECB3A011616B16A20B
:1086B00086D2806622ED927CF3D5D0D37266A8FB79
:1086C000C77CA126C02458098BE63DA104300211C5
:1086D000E767FC30623E40E6100620BC18BF5D2410
:1086E00037BA11F46DDAD60871037B98E0819F3CAC
:1086F00046F1001ED04A190F7EF38807F2401EC0D3
:108700007D39200FE4819EB435262CFCEC4002E636
:10871000E01900E0415382D306C8DC0379D3870C0B
:10872000A8B8F9564506379383ADD13178CFFCB15F
:108730007A1FBB314D867387884693FFEF43D3661C
:10874000FD73F126C20CC9B313E63E3619228BE441
:10875000011449190418E078192319097819B4C1CA
:10876000241996F81884F590E1D2E9501921812452
:1087700034F180061042FD480809211BF39BFF24B9
:10878000F5B2CBE486124292FAE02221A4013857D6
:10879000F3F4D384DFA7E0DBB10637AC4BF5F30C81
:1087A000AAF806C6FD6F60AFFA1A98F9C03B5AD412
:1087B0009882F35FBF6FE69872B3865F2CE498D31C
:1087C000B820E0FF5A6B040FD313B8FB042904440C
:1087D0002289028877CE8BF3081040DC102B02BE72
:1087E000F7DDB30A6AF88E0579B3460110DB7E65C2
:1087F000F344EFBFC954D371E141FA849AC216FA27
:10880000AC2CC2BBCAF56340BE050920018CF3F64F
:10881000B38504927244D34DE03524DF8C9112D39A
:108820009AA3D3307D69FC60412CAF8FA5D80B6231
:1088300041FF3C9007B22016C482D15810F3887EC5
:10884000EA019F19B02002C08287180BCEE281F3A3
:1088500005B10606C8F1D3C65A15A4882C06946F34
:10886000934728F9174E864A04810C104D82408A9E
:108870006AE54299018140D34317CC4147F397D32E
:108880007CB1EAF980092219D7C6C55C099119C0E3
:10889000BF18010B60028C5DD1678AB3733FE0DBC8
:1088A0006B424C991926C07FA520D34C3AB9007071
:1088B000FFF7FF844611834250940898AFF68590E5
:1088C000100247982B8F33308406FA025FBA832256
:1088D00028BF84A8FEF3F4D331DA1EFC65DE84E8F9
:1088E000FF2116062FAC3CB8FCBFAB863DB083F22F
:1088F0009EF39818E07E1DE08110DB399518E0C7E3
:1089000056789854F36AD339B9F8FEF2F2844026C7
:1089100001248FEEF6A60980D91C20621A72F78115
:1089200009A02029D742ED0144AAB837A94893D31A
:108930007980FA1A4117090640F70458009177FE2A
:108940004110FF0122C02898048B60F6104C824928
:10895000469B9E74187990987F099DF5D326BA3965
:10896000C146BA44D3C63CAFF0FEE045CF30B42098
:108970001EC84A820FE6508805B823B830E3F37565
:10898000B322ABF8F101922D73E0B93018DF200F5C
:10899000E98BF0B06AD3F50C2098F9D964086640E9
:1089A000931FA4FC1CB1C18D2EFC3FD96F09EA377F
:1089B000F38BCDF3DAD3D8FF00B3FE5E3043B3ECD4
:1089C000300416634FAFE3304D098F4236E0498BD8
:1089D000B31066D318F9B2E22AF2C5E330F2C8BF89
:1089E000AAD467E5C8BE747D8211D6AFD0F77040B7
:1089F000282165C86CF6B6F376D3109CF947D84E9B
:108A00004796C334DBFAA8FC804108F3A56E2530F5
:108A1000F3017C522B03FE5FDDD9126AF8C7E50132
:108A20007F3910C40338D3D2E201C6C172F3048384
:108A3000D3F6C6E0FE5D62C4B646AF932171F3394A
:108A40007F86C9A3049F3D19897067E2BC8040E11D
:108A50000C14F22004061188C7C989D3B913AFFBDF
:108A6000E8AC0810936FF501C8C8101618CE68C896
:108A70000866B8EA9F8612208045307E6EC820279F
:108A800083B92131F87E6CC8F2ACDBC8F0E5C89F31
:108A9000AAAFE6008FFCD6C8586BC8018B0337C855
:108AA000C0E4C8F7C60028FBE6D5C4137CA3C8867B
:108AB0001ACBC856FB8320ECDFC83096C8DCCA034B
:108AC0006BFE4560C05D9BE4C8B1B31CDBC8146D90
:108AD000411EED19E61340411901E219D316501950
:108AE0005858FC3D8434807BD242084D028D22A62A
:108AF0005CC8DEA321DE3C6769EEB04942FC02455A
:108B000003282221F8A735801002D51A92C8D33144
:108B1000B93655F95FD9A1FEB8B3053C7C0232DC09
:108B20007F2330667230F8FEBB64C5D28EFE982B70
:108B3000F3D1B81C57D7315944FEE5EB88013CA965
:108B4000B1AE8359C87F2803F0EAE3D39A0CB8FA90
:108B5000CBC88106D250EA4C57FD320902040C38CA
:108B6000861830B4CD336EB56CFE8009B202502643
:108B70009060222689B318011490AAD32720F36AA3
:108B8000FDCA8444A157B388D7326E5144CDC82260
:108B90007F9F201165761746D5F80339AB1206E0A2
:108BA00023B52CCFC882E00A12C100CC5CA1D34C03
:108BB0009EC6BCF0FA60B830BDD216BBC4D7986868
:108BC00078C5F5831EC483EDB8E2419FB795786BF5
:108BD00008B01F0EC0031920E70BE0419005F0001C
:108BE000D30902D36201F90C0898FE885B76ED0B7D
:108BF00008B85DB2C8EF038B10AD0C2328E93CFF29
:108C0000B701087E519B667103F9C82ED3CE9BA98C
:108C1000FA5F33F8CC18CE6FB38821CDC89864F5CD
:108C20000E8C8805DFE523EAAAF849320076E519BB
:108C300042FFF93EF30440081368D34CF3564D56F7
:108C4000C871D51242E848B3BDC5859110C7A41AB2
:108C500082D7FE2159BCE5B3C430FA77A0A52275AE
:108C6000A80134EB3142CED3F08B1B50F81BE34309
:108C70007FB33A393018629E98DF58F8E5D2B709C9
:108C8000FE324275F308079EF5880310BD8B01671D
:108C9000EDEC79857103FB490A02B428B803BA27C1
:108CA000E2D31AB904FED103FD7F11B5FFDFB2A2F2
:108CB0001088E150FC7E59E8BE98A501D9122FB367
:108CC00040EEEB30808FC63FD3DF8BFAFB80511034
:108CD000FC0A024128080164CDA784F346C0202382
:108CE00087F5601484F25FCDCF2F05CC8C2881A14D
:108CF000E9D48C029E4625C68CE9D3515AD6E0FFB2
:108D00007DD58005B0007898DC950BF3BB0739C89A
:108D10008378F37659E8ADB3E2811D539ED50218EE
:108D200020B9030CE59007B0F3EAD3E0F698A8FF6A
:108D3000FC96D57C9EC545F3F7BF6A426196F34029
:108D40004EDA9F9C12085FD97E5C9BFA598E7F5F3A
:108D500064EC8B19F8FFC0B00886C02498024DB1AE
:108D60002C8866C8264DD3BA1366F58159E0BFCD6D
:108D700036C404B988E5A34042B3ECF308406C0B59
:108D8000620B8CBD983893FA0DFE403A4342483B43
:108D9000828F3DEE084203EF23678B55B0A0BFAE34
:108DA00098B0FD8C18766A22B83D13BD6B4A5D0BF6
:108DB00073D31411D828F8E66DF201561902DC219C
:108DC0005F585E98B11036D3E0FB32D346BCA53372
:108DD000BA17F4F3F0091EF3927891F3DD204205FF
:108DE000BF4A172648E0803FEB8F3D4BC60C5FC75C
:108DF000D3ED10FDF22804068048BF81905ED39425
:108E000030F33BE1024108E609810D04CFF2E7DDD2
:108E1000FD12733D435045D0CA3D043FC6EE424467
:108E2000D312FFB8FE8009B00026C1164856B6CE50
:108E3000E3F3300891F398A360FB020C82093FF53D
:108E40007F10E50CD324911327EDD34030FE01268B
:108E5000C02400118368D34CD31F50F9E0BB413DBF
:108E6000D52016C4792D713D7023E7F31EC4191067
:108E70000F2CE6FF9CEA333CA002E0BCA5BD986243
:108E80005C035E6BDA16C021D30CF5C8F984D29E60
:108E9000E3D326DB7381D3B2570465B830C47E694F
:108EA000FF2E985C0003D369D52AB7F613D386400A
:108EB000FF47263B195808439A1905307E964818F3
:108EC000010861026CE089F2B4F24A06694C87B38A
:108ED00042D0D351C6E5799010B30FD31921E8FCE5
:108EE00076CF98FE1042085C6A7E5FB3B7D4E53057
:108EF0008865C61AA07B984008A422E035ADF23FF1
:108F0000A02703D53010C1ECFD6152FF02DBEC77E6
:108F10004F9F30B8FFC001385D101718808A0305D5
:108F20000E7D9FFE98E1C00370CD0F8F0CB1D7B6B8
:108F3000AEF5E8E530E0799872300EEE513D07C6A7
:108F400016D3899DC659F2FB20048608B4026B181B
:108F500004C898F3FF0F980CD18121889F9A7B91C8
:108F6000FF9912021B9045D3CAE0E2306FD38160B3
:108F70007DD3043200CBFDD975C846C1C27E2360C3
:108F8000220C95F309F89F58D5A3A5DCF59FB6F4FC
:108F900086B3DDA91DFD17AE80D7D104D78C9B8B7E
:108FA00070EAAFC6DB26FAF998716AA7BB98F12080
:108FB0001EFDC5E22146DA0736BB9003C519A5346C
:108FC000EE78C883581A69D30C88D30628F3D39F48
:108FD000F30070FA8081779D989BC86189A0F3C2E5
:108FE000DB201805F3B4056DBBD0024D66B8308D9B
:108FF000A3751540772E3020C89B189BF95D113062
:1090000040736A58102B193EC81132094660D318B4
:109010009DF3404C7023B33339CA0469CF304110FB
:109020000B02E9420C84B3469FC27A10136202E934
:109030008C841148FA639EF4B704F3EC085BFFBC20
:10904000FF2FCC59E3F339AC22636CD3B8F906098E
:109050000EFF98FF24C68C93E3D11C6239EBF830E5
:10906000486C66C9FA12DB190801193344CCD06D7B
:10907000D3A388FCC123E5CC6688EDB2B9F6B0660F
:1090800096D1CDDCC4B180861950FFC7FC4BC7C850
:10909000FF9CD7B68BFB081F886F9B6E883066C716
:1090A000FBC601634DE3B8FE825F9BE57E9808C274
:1090B00025D1808DB746B8FD8B0CB00B977A20FE7A
:1090C0001C04CBFEFED8FDC8348A0564012CDA5C92
:1090D00056BDA8887785A26DE6CE5BB3C8FF72C97E
:1090E00014F5E80AEAECA03CCDD6C51B7014A04FDD
:1090F0000C552E40410D11CB2B5057981105609403
:10910000FAAEF787842263FF537B9604C58B264112
:109110003CDA02E320CA9280F11D41F46804AB08F6
:1091200088FC615FDED64CA041F8F7208285667B23
:109130008FFB4079E0851E0FBC88D8B2FCCEF9A821
:10914000A5D918FD1D5471B49DDB1A023FA44FDE52
:10915000DEE014D3948067D36FC4B5FFB3FA4C3804
:10916000E5F310BF587F424BB1FECEB391FB944460
:10917000632DB3C8F99CC863BCBAB10895915C87EC
:109180003D6467FB76D8FB5FC37998FFB666695587
:109190008A71C9B9D31CE0D309B1D3717D85DD6C67
:1091A000631B71611EECE3028D23B3391AFD7FFE50
:1091B00085866833B34999B0B0FBE3EC8DFFDF28B7
:1091C00098E64B142C15806BD63D303BF67F147916
:1091D0007A8C7E3280C33D58AE08C96685EB4C98C8
:1091E0000CFBFE0262BA62B1FD85E2048C7E302285
:1091F000C4DB1A18F95EDEEB02D9770667713F8B84
:10920000F4B10633DDB168F8BFEC1701915EAD61D2
:1092100097968A91FC72EB9F448DBB56F30286654C
:1092200076E8E320F0C65B65C8F853D6376F2C3676
:10923000F13059996158B3FB08BBF4C77B664063B2
:109240000DE0F8FD8F1980FAFAB1045E9D100DE073
:10925000F919E2DE215F25629E08B888AC3B151D36
:109260003AE720FFA69F4AF6D9FA4A14BFFEECABB4
:1092700053CE5B51D382C490C640D313F358FE66DD
:1092800079598FFAF110D89CCACA2EC8C0A9833860
:109290006CB32EA52380EDC5988202D59640F07F51
:1092A000F77D1108E812A3F66FFCE8D34FBC6051BC
:1092B000A0FCDB057CD9E8B34221480BBD998A08A4
:1092C000D1B30A0BE21CD6DDB3C0C01DB5B516FF85
:1092D000D14A2801BF30D1960AB8400260A7EEE01B
:1092E000F9BD8042988F020744C6C1D72284F38219
:1092F000464ADD889B01F35AFE31FFA1305655C026
:10930000C029CC5784CE147F600D09C8E9025805E6
:10931000B4189C30062202F9BE5E010630660DAF1D
:10932000C0AC6FA7998272623FBB6E5DB3043F0C05
:10933000106AE5B6F82FBFB5F6EB0DBFFC4149CF7B
:1093400022F967F94937600281FFAC400168B8D95A
:1093500020081EE4D9F8105989B6805AF30AF8DBC0
:1093600021188F5FC3D746FD86BF5E39F3D8D4F985
:1093700049E4E87479B38DEF1B18FB6106D7BE1B77
:109380001FA8B040F1C5FB1570B7FCF9BD4864AC2F
:10939000B0017B714920D9DDACF4141038F8E56BCD
:1093A000D7C5FDFDB8F3D879928A5620D99514789F
:1093B000D3D7D9089F58B5FCDD9EA8F8892C86180C
:1093C000686CCF371E513848198FE9B4BA0B10DFDB
:1093D00088EF5DDC19DDFB60B0FB876512BC924F46
:1093E000BC0893CF3D6166FB6266C119E52F657BC2
:1093F0008FE69428CDF97F5962AE330478FFC6F624
:109400000FDD75086226037BF528FF67ACE508E5EC
:10941000CC20A9E08FBAFF38FD025F4A23D19EED30
:109420000100C9AF25943621899735BDAE1402C01D
:109430004126D324F390C867838804CC78FD157245
:109440001E84005A124046BD09E4412414D078100D
:10945000E4F37C0820B3D0D8B34120EE5AB012799F
:109460002404909E80A4822028FF6E1760F9F40CDB
:1094700048B6F5C935AC6BC6FC18ACFFD857ED7FC4
:10948000720AC70CC3E6E018FA0715A002FFB48001
:109490000A50012A4005A0A8F37754BFF3C004B8CE
:1094A00000136067F76317E0FF025C800BF0032E88
:1094B000C0CD05B8F360B2F30F84F3B918F99F0C6F
:1094C00094013353FF06CC4019280365C03FF3993C
:1094D000326006CA3FF3488364200DD9A641DC46BA
:1094E000FF0C9001324006C804F319200364F3A472
:1094F000B54153F313F31401E300FBFFB008FFFF82
:10950000FFFFFFFFFFFFFFFFFFFFFFFFFFFFFFFF6B
:10951000FFFFFFFFFFFFFFFFFFFFFFFFFFFFFFFF5B
:10952000FFFFFFFFFFFFFFFFFFFFFFFFFFFFFFFF4B
:10953000FFFFFFFFFFFFFFFFFFFFFFFFFFFFFFFF3B
:10DFF00054657374265365727669636538168FB3FA
:10E00000F89404B7087011F00C940000FF246AE53E
:10E0100011E0E12E1FEFD12E11E2612E10E1712EE1
:10E020001FE111BDF1BCC798BF9A1FEF1DBF10E1E2
:10E030001EBFE0E0F0EEEBBEC0E0D0E187D631F7E6
:10E040009F9B1EC07ED6E1F41E9818E111BDFFCF44
:10E0500024D6E4E9FFEE23D674D661F4E8EAFFEEB5
:10E060001ED618D6E6E9FEEE1AD6E0EFFFEDD7D5BC
:10E0700011D6EACF01E305D6ECEAFFEE10D655D66D
:10E0800019E718BB17E817BB18E01093610010934D
:10E09000620011E01EB910E71DB9F092980015E07A
:10E0A00010939900F0929B001EE010939D0018E0E1
:10E0B00010939A00E0ECFFEEF2D5E8E8FEEEEFD523
:10E0C000E0EFFFEFACD5E9D5E6E9FEEEE8D5992023
:10E0D00021F0EAE7FEEEE3D503C0E0EFFFED9FD5C8
:10E0E000DCD5009BFECF05E021D6EEEDFEEED7D5C8
:10E0F0001091610011601093610013E91A95F1F716
:10E10000109161001E7F10936100019BFECFE0EF34
:10E11000F0EFEBBEC0E0D1E010E8079009920FB835
:10E12000779BFECFD150DF70DF5F52E04FEF110FD2
:10E1300011F41791111F441FD0F75A9549F402E0CA
:10E14000459580F00395439551F053E04FE3EFCFB1
:10E150005A95B1F4469508F35395E9CF040F54E06E
:10E160004FEFE5CF4395D1F45395479558F1551F9F
:10E17000110F11F41791111FC0F7050F56E0D7CFFB
:10E180005A9511F401E00BC05A9529F4439531F4E6
:10E1900055E04FE1CCCF5A9509F7542F47915A9546
:10E1A000A42FB52FAC0FBD1FB150BF70BF5F0D9036
:10E1B00009920FB8779BFECFD150DF70DF5F0A95D1
:10E1C00099F7B3CF029BFECF10E51DB91E9AC79AEF
:10E1D00064D5E0E0FFEE63D5E2E1FFEE60D5F092BA
:10E1E000B406C09A10E24ED3C0982FEFEAE4FEEED8
:10E1F0005ED32A9511F401E044C20130B9F7E0E59D
:10E20000FEEE55D380E002FF80E414E03BD307E745
:10E210003ED312E037D309E630D3082F2ED33ED3B6
:10E22000002341F002FFF3CF01E431D30023E1F7F3
:10E230007ED30AC07CD3882339F00AE728D31CD3C5
:10E240000093B40615E01ED3A0E0B0E0C0E0D0E03B
:10E2500084D377D311F003E014C2EEEB00810F7783
:10E26000A1F4E2EC0081013051F0043041F00630BD
:10E2700031F00B3021F00C3011F00E3031F4E6ECBF
:10E28000A191B191C191D0812CC0E0E0F4E035853D
:10E2900000E010E028E037950F1D2A95E1F70A9578
:10E2A00009F4139506850784002909F0139503895D
:10E2B0000488002909F4139500A101A0002902A0F7
:10E2C000002903A0002909F413950589007F003F68
:10E2D00009F41395143009F0BECFC0E0D0E0A0E0FF
:10E2E000B0E0A0938D06B0938E06C0938F06D093B6
:10E2F000900633D326D309F0AECFE0E0F4E00385F7
:10E300000023D1F704850230B9F7C0E0D0E0A68938
:10E31000B7890B2F0A2B21F4A4A1B5A1C6A1D7A1BF
:10E32000A0938706B0938806C0938906D0938A0687
:10E33000C0E0D0E0A389B4890B2F0A2B21F4A0A15F
:10E34000B1A1C2A1D3A1A0939506B0939606C093A4
:10E350009706D0939806A189B289C0E0D0E00B2F30
:10E360000A2B19F000E1D4D3ED01DF93CF9300899C
:10E3700000938106A0918706B0918806C091890616
:10E38000D0918A060A95AA0FBB1FCC1FDD1F0A95E4
:10E39000D1F78F919F91D5D38685978580938B06F2
:10E3A00090938C06CED3A0939106B0939206C0931F
:10E3B0009306D0939406E5E9F6E0ADD3E0E0F4E00F
:10E3C000058500938206A4D3A0939906B0939A067C
:10E3D000C0939B06D0939C0602E0DD2359F4CC2326
:10E3E00049F4A53FBD0530F401E01FE0A53FB107AA
:10E3F00008F400E000938006A0E0B0E0C0E0D0E0C8
:10E40000002331F00A9521F0A4A5B5A5C6A5D7A58E
:10E41000A0938306B0938406C0938506D0938606A6
:10E42000A093A506B093A606C093A706D093A8060E
:10E43000AF93BF93CF93DF93A0918B06B0918C06DF
:10E44000C0E0D0E0EDE8F6E073D3A0939D06B09372
:10E450009E06C0939F06D093A006E7E8F6E068D337
:10E46000A093A106B093A206C093A306D093A406DE
:10E47000DF91CF91BF91AF9111E00A2E0B2A0C2AA8
:10E480000D2A39F01F93B7D2A4D21F9110F413951F
:10E49000F9CF1093A906C0E0D0E065D2C0E0D0E08B
:10E4A00006C02196B096F63011F45DD2B9F403851A
:10E4B00003FDF7CF04FDF5CF0081053E91F3002366
:10E4C00069F0EF93DF01ECE5FEEE0791002341F0E8
:10E4D0001D910117D1F3FB2FEF91E3CF04E0D1C0E1
:10E4E000FB2FEF91A28DB38DC489D589A093AB0684
:10E4F000B093AC06C093AD06D093AE06A48DB58D97
:10E50000C68DD78D0A2F0B2B0C2B0D2B09F440C079
:10E510008FEF91E016D3F3D21197CF09DF09009165
:10E5200082060A950A2303950093AF06009182069E
:10E53000EFD2A093B006B093B106C093B206D093C9
:10E54000B306F092AA060CD30093B606F092B50675
:10E55000C0E0D2E0A0E0B6E09924AA2440E8099106
:10E560000D9301D44A95D9F79A2891F479D181F481
:10E57000A0E4BB24CC2428E03D91369550F08D2CAE
:10E58000FCD3E9F1C79AB5FEC7982A95B1F7F3CF46
:10E5900077C0AF93BF933F932F930091B5060023AD
:10E5A00061F4C0E8D2E0A0E0B1E0442709910D9306
:10E5B0004A95E1F7E092B5061BC0C0E8D3E0A0E0C1
:10E5C000B1E040E809910D934A95E1F70091B60654
:10E5D0000023F1F2C5D20093B606F092B506C0E072
:10E5E000D2E0A0E8B1E040E809910D934A95E1F747
:10E5F0002F913F91BF91AF918824BFD319F6BB24CF
:10E60000CC2428E03D91369528F001D4C1F12A951B
:10E61000D1F7F7CFAF93BF933F932F930091B506F8
:10E62000002361F4C0E8D2E0A0E0B1E04427099102
:10E630000D934A95E1F7E092B5061BC0C0E8D3E020
:10E64000A0E0B1E040E809910D934A95E1F700910F
:10E65000B6060023A9F084D20093B606F092B50660
:10E66000C0E0D2E0A0E8B1E040E809910D934A95FE
:10E67000E1F72F913F91BF91AF91B2D341F6E8CC32
:10E6800005E00093B506C09A1FEF1DBF10E11EBF45
:10E6900004D3EEE9FEEE03D301E3F3D20091B50615
:10E6A000013021F4EAEAFEEEFAD211C0023021F480
:10E6B000E0EBFEEEF4D212C0033021F4ECEBFEEE00
:10E6C000EED205C0043039F4E0ECFEEEE8D2E2ED23
:10E6D000FEEEE5D203C0E6ECFEEEE1D2E091B50637
:10E6E000C79A05E010D3C79805E020D3EA95C1F793
:10E6F00018E110939A00D1D2E0E0FFEED0D2EEE123
:10E70000FFEECDD214E11F9303E4C0E0D6E07CD04D
:10E710001F9119F41A95B9F795CC9A2891F008E150
:10E72000DAD2D9D2D8D2D7D2D6D2FFD2E8E6FFEE0B
:10E73000B6D2B3D201E3A5D2EEE6FFEEB0D2F5D267
:10E7400081CC8ED061F7A0E4BB24CC2428E03D919D
:10E75000369528F03DD3B9F02A95D1F7F7CFC0E030
:10E76000D1E006E051D021F4043049F005E1FACFC0
:10E7700006E04AD029F4043011F005E1FACF33C0A5
:10E780008824FBD249F7A0E4BB24CC2428E03D91A7
:10E79000369528F41DD331F02A95D1F7F7CF8D2C7B
:10E7A000ECD2D1F7BB24CC2428E03D91369528F05B
:10E7B0002ED3B1F02A95D1F7F7CFC0E0D1E006E033
:10E7C00023D021F4043049F005E1FACF06E01CD053
:10E7D00029F4043011F005E1FACF05C001D351F757
:10E7E00006E079D281D2043006E029F008E173D244
:10E7F00072D271D270D26FD298D2E8E6FFEE4FD2C9
:10E8000027CCC058DF0905E166D216E0C79A10FD93
:10E81000C79840E050E7E5E041505040E04021F427
:10E820001A95A1F70027089566D2B1F30430D9F301
:10E83000013091F7C79AB1FEC79856D255D29924A4
:10E84000AA2440E851D209938ED24A95D9F74CD2E6
:10E85000102F4AD20915A9F61A1599F69894089519
:10E86000E8E6FEEEEBBEA0E0B6E007911D910117D1
:10E8700011F40A31D1F708950FEF0FB9779BFECF4E
:10E880000FB108950FEFF9DF1A95E1F708950F938F
:10E8900012E0F8DF0F91F1DF0027EFDF0027EDDF57
:10E8A0000027EBDF0027E9DF0FEFE7DF08C012E00A
:10E8B000E9DF16E0EBBE0791E0DF1A95E1F710E221
:10E8C0000FEFDBDF0F3F11F41A95D1F70895C098D1
:10E8D000EF93FF930091B40606FD07C0AA0FBB1F7C
:10E8E000CC1FDC2FCB2FBA2FAA2715E0CBDF01E5F9
:10E8F000C4DF0D2FC2DF0C2FC0DF0B2FBEDF0A2FAE
:10E90000BCDF0FEFBADF8FEFDADF8A9571F00E3FD1
:10E91000D9F7FF91EF9180E092E0AEDF019301978C
:10E92000E1F714E0AFDFC09A089502E0AACE0BE74A
:10E93000AEDF0023E1F7E6E5FEEEB9DF0023D9F70D
:10E940000895EEEFF5E001910535008109F40A3AEA
:10E950000895E0E0F2E0BBDF0895E0E0F4E0B7DF27
:10E96000E0E0F4E00895CF93DF93DE01C0E0D0E073
:10E9700000E1CED0AF93009182060F93C9D00091F1
:10E98000A9060A950A1738F4CF91CF91DF91CF915C
:10E990000FEF00230895C091A706D091A8060A2F73
:10E9A0000023A091A506B091A60629F00F9323D0CD
:10E9B0000F910A95D9F781D00F900A940F910021F9
:10E9C000A00FBF1DCF1DDF1DC8DFDF91CF91002736
:10E9D00008951FE000918006002319F4A73FB107B6
:10E9E00008950A9519F4A73FBD050895A73FBD05F1
:10E9F000CD05D107089500918006002339F10A95CD
:10EA000079F0AA0FBB1FCC1FDD1F0A2FAB2FBC2F25
:10EA1000CD2FDD270AD03196C191D081DF700895C6
:10EA2000C0E0D0E00A2FAB2FBB270F93CF93DF932B
:10EA3000EDE9F6E07DD091DFDF91CF910F91E00F0E
:10EA4000FF1DE00FFF1DA191B0810895FD01EE0FA4
:10EA5000FF1FEA0FFB1FF695E7950A2FAF2FBB2785
:10EA6000CC27DD27A6950F93EF93FF93EDE9F6E012
:10EA70005FD0AF93BF9371DFBF91AF91DF91CF9123
:10EA8000D170EC0FFD1FC191F63031F4CF93C0E08F
:10EA9000D0E0119662DFCF910F91B081AC2FC0E032
:10EAA000D0E0069540F4B695A795B695A795B6958E
:10EAB000A795B695A795BF7008950D2F0C2B0B2B1E
:10EAC0000A2B59F4E1EAF6E0A0918706B091880696
:10EAD000C0918906D0918A062BC01297CF09DF0911
:10EAE0000091820604C0AA0FBB1FCC1FDD1F069534
:10EAF000D0F7EDE8F6E01CD0E1E9F6E019C0AB2F65
:10EB0000BC2FCD2FD0E001E0D695C795B795A7953E
:10EB10000795D0F7089501910A1BA02F01910B0BC7
:10EB2000B02F01910C0BC02F00810D0BD02F089539
:10EB30000191A00F0191B01F0191C01F0081D01F52
:10EB40000895A80FB91FCF1DDF1D0895D8DFE7E88E
:10EB5000F6E0E1DF0A2F007F0B2B0C2B0D2B089525
:10EB6000E0EBF6E001911191012B1191012B119134
:10EB7000012BE1F1A091AB06B091AC06C091AD06BE
:10EB8000D091AE069ADF0091AA06A00FBF1DCF1D3F
:10EB9000DF1DDFDEA091AB06B091AC06C091AD06E3
:10EBA000D091AE060091AA0603950093AA06109193
:10EBB00082061017C9F4F092AA061DDFA093AB06D7
:10EBC000B093AC06C093AD06D093AE06E0EBF6E092
:10EBD00000810150019300810F09019300810F0909
:10EBE000019300810F0901930FEF0895A091AB06E7
:10EBF000B091AC06C091AD06D091AE065EDF00913B
:10EC0000AA06A00FBF1DCF1DDF1DA3DE0091AA061F
:10EC100003950093AA061091AF06011B089502E325
:10EC200030D02CE00791002321F01AF054D02A951F
:10EC3000C9F700E250D0ECEFA791B7910A2F0F71FE
:10EC4000E1F01B2FAA0F111FAA0F111FAA0F111FEE
:10EC50001F7099F01D3088F42B2F26952F732930C3
:10EC600060F024D00EE237D0012F20D00EE233D056
:10EC700000E228D0022F1AD0B7FD0895E0E9FEEE99
:10EC80000EC00F930BE127D00BE525D00F911AD0C2
:10EC90000DE621C0EEE6FEEE02C0E0E7FEEEEBBEC2
:10ECA0000791002311F017D0FBCF0895005D07FFF7
:10ECB0000053085E06FF0851045F05FF0C500A5F11
:10ECC00004FF06500F93029501D00F910F700A3088
:10ECD00008F0095F005D1F9310919B0015FFFCCFAA
:10ECE00000939C001F91089500919B0007FFFCCFAB
:10ECF00000919C00089500919B0007FF03C00091C4
:10ED00009C0098940895FDB814E6169A1E9808D0B1
:10ED100016981E9A05D01A95C1F70A95A9F7089575
:10ED200084E695E00197F1F708950EE14EE15EEF7C
:10ED3000C895C895C895C895415050400040C1F746
:10ED40000895E0E0F0E0FBBEC0E0D0EF9D2CAD2CDC
:10ED5000079109D0079107D0C79AF5FFC798219767
:10ED6000B9F79A280895A02618E0990CAA1C10F467
:10ED70009624A7241A95C9F70895EE27FB2DCBBE3C
:10ED800065EA03E04BD0839491F0EE27FB2DCBBED8
:10ED9000C0E0D1E010E80990199001E03FD0329630
:10EDA0001A95C9F7EE27FB2DCBBE05E037D001E160
:10EDB00035D06AE5882061F0C0E0D1E0EE27FB2D78
:10EDC000CBBE442707911991011729F54A95D1F730
:10EDD000BE0CCF1C1C2D113011F41B2D103E0895BC
:10EDE000C0E0D1E065EAE199FECF1091680010FD26
:10EDF000FCCFCFBABEBA09910DBB653A71F4E29A65
:10EE0000E19AC79AB4FEC798B39469F76AE5CE0C45
:10EE10001C2D103108950EE176DFF8C81F93109174
:10EE2000680010FDFCCFF894E199FECF00936800D4
:10EE3000653A99F7E8950000000000000000109185
:10EE4000680010FDFCCF1F91089540000000009560
:10EE500048000001AA875000000200FF5A5845569A
:10EE60004F5F465742494E005A5845564F1A0D0AB1
:10EE70000D0A1B5B313B33376D001B5B33316D4239
:10EE80006164204352432100626F6F743A20000096
:10EE90002062657461006D61696E3A200000534420
:10EEA000206572726F723A20000043617264000044
:10EEB00052656164206572726F72000046415400B1
:10EEC00046696C65000057726F6E672066696C65F5
:10EED0000000206E6F7420666F756E6400000D0A6E
:10EEE0005365742074656D706F7261727920636F01
:10EEF0006E66696775726174696F6E2E2E2E0000E2
:10EF0000547279207570646174652066726F6D202B
:10EF1000000053442D636172642E2E2E0000525364
:10EF20002D3233322E2E2E0D0A1B5B306D4E6F7735
:10EF30002C2073746172742066696C652074726130
:10EF40006E73666572207573696E6720582D4D6FFC
:10EF500064656D2D4352432070726F746F636F6CE4
:10EF60002E201B5B33306D000D1B5B4B000044619A
:10EF7000746120697320636F7272757074212055FB
:10EF800070646174652069732063616E63656C658C
:10EF9000642E00005265636865636B20666C617364
:10EFA000682E2E2E202020004F6B210055706461AA
:10EFB0007465206973206661696C7572652E000046
:10EFC0001B5B303B33303B34306D1B5B324A2020BF
:10EFD0001B5B313B33316DDBDB1B5B33336DDBDBC9
:10EFE0001B5B33326DDBDB1B5B33366DDBDB0D0A0A
:10EFF000201B5B33316DDBDB1B5B33336DDBDB1BDA
:10F000005B33326DDBDB1B5B33366DDBDB20201BC0
:10F010005B33376DDFDFDFDFDB20DB202020DB2011
:10F0200020DBDFDFDFDF0D0A1B5B33316DDBDB1B3A
:10F030005B33336DDBDB1B5B33326DDBDB1B5B3345
:10F04000366DDBDB20202020201B5B33376DDCDFBF
:10F05000202020DFDCDF202020DBDCDCDC2020DBCC
:10F06000202020DB20DCDFDFDFDC0D0A1B5B3331FF
:10F070006DDB1B5B33336DDBDB1B5B33326DDBDB4B
:10F080001B5B33366DDBDB202020201B5B33376DB1
:10F09000DCDF20202020DCDF20DFDC2020DB202044
:10F0A000202020DFDC20DCDF20DB202020DB0D0A1D
:10F0B0001B5B33336DDBDB1B5B33326DDBDB1B5BDD
:10F0C00033366DDBDB20202020201B5B33376DDFE8
:10F0D000DFDFDFDF20DF202020DF2020DFDFDFDFBA
:10F0E000DF202020DF20202020DFDFDF0D0A0A00C4
:10F0F000FF1F627FC23C006088FFFF8008900122F2
:10F10000400488C60011850302E24410015C41F30B
:10F110009320F5E6101A00CD6EFF0C1046D3086C54
:10F12000E033F306D398E9200364F301FFD8FD0030
:10F1300015E0025480F00A50012AF30468FBA0DEB7
:10F1400002B4F3E64005A8E6A01B39B312B9A0D378
:10F15000D00DB0E0CEF30BD374C005B838F3027015
:10F16000F84C121BFF98FF0229B38048FC40ED1DAC
:10F17000F458FF06848BCB400856A82106BFD8CC94
:10F180001FA6B307E9B3FC866AF8639DD1D870FD6A
:10F1900046B36DCB28041B76DA50FB08090D1981A4
:10F1A000FE824FF6CC89FE097F7FB004486CB3FA2B
:10F1B000F90FCF304B7FFE7FD8FBC12CB3C12C1988
:10F1C000C127B6B19004BFF632DCFB071FB64BABCC
:10F1D000FC0C9C3060FE19607E713083FF7617B2A4
:10F1E000FD071EF649C9FA07A718301FBC30607E1C
:10F1F000F23010C958F4884CB3607EDF60C00264FE
:10F200002CF4183EAE92F040C858F4287D4B11C043
:10F210002A70C4FF18242CB3580F2E3130FEB1CB06
:10F22000CFD852B3EE5BC87ABA01C2258DB98EF23F
:10F23000CA04D56602611266E0C73515806AB3B0AC
:10F24000508DB31BB0FD8C6658114419D8F8FB25BE
:10F25000A6B320CF80BF5202A5403C019CF36718A3
:10F26000D1D9D38277AC982811CC6613A677C12365
:10F27000ECCC137649C096FB320ECCB30FD3B3035C
:10F28000F4B3C0FD30B33F56B310090BB3CC04CB7D
:10F29000B0AD370CB30FD3B303F4B3C0FD59B38093
:10F2A0002DF409FE9AE3607EFDCC81FAB3B240AA48
:10F2B00092C129668961F7AC982095F4B881C3F6AC
:10F2C0003207EE18E13F98B31FA6B307E9B381FAFE
:10F2D000B3607E98B31FABB30C55F8068DB6DA70E9
:10F2E000FD11ADB30856F80436DAEC50FB08121BDA
:10F2F0001981FE077C3147FFD87F042436B3FAF921
:10F3000004062C94404DEA88604CE2940CC121B371
:10F31000F2B0F9D3F6324324EBD8A8F866B4D8C0DB
:10F32000039D6CD3F834311936B3F1F9030486B375
:10F33000A8FCC127F632DC0725B62CABFC0F3C300D
:10F3400060FE1960FE669604B304CF989824E7C85F
:10F35000B2FD608EB5EC300288123F323CD61020F0
:10F36000D8962300668EF9C12019C34E30303F6D08
:10F3700079BAB0FD260C190DFDDC9620B360C7F6F6
:10F380007F0FF5DFD8D8FB22B9B3800501FB608C75
:10F3900019A0E0B41BF80804526660B308FE3048B8
:10F3A00000B3CC30B33F6E60DA6CEC73F652B33B13
:10F3B000DBB10255F801844D8DB9FC8EE172AA666D
:10F3C00002C22666E0FAC73E0FD5B350611BB31BDD
:10F3D000FD611866B0118919F8B0FB4B4DB320CF11
:10F3E000807F5202404B3C0138F3CE31D1B3D3047D
:10F3F000EF589828242C6690130C66123ECCC13B23
:10F400006C4912CC660FCBB0603F6EADC6B7868834
:10F410006040DE6080C53489C0FDF3E503F4B3C00D
:10F42000FD30B33F4CB30FD3B303F4B3DE365BB858
:10F4300004AA1940AE60C0CDFD7F408A18B318669B
:10F44000193F8D8254FB8395D860FFC76D01824FB1
:10F45000B29808101558662398B2275E6010C12133
:10F46000B3CC6099E64B06F9B381FB36C407EFD8FD
:10F47000CC1FA6B307E9B381FAB3B50C58F806DB85
:10F48000DA70FD61265AECACF8046DDA50D8FB084E
:10F4900024361981FE04C6ECE304121BB3FAF90307
:10F4A000EFCC4B1FFE7FAC79C12CB3C12C19C12707
:10F4B000B6B190040FD8321FB7606071DF13BAFD88
:10F4C0006072F9E58131A6AF069F18307F86E107AB
:10F4D000EF98981FBC30607EF13081FB766007EDBD
:10F4E000D8601FABB31053F81CFE52A2FCC716BA6B
:10F4F00002ABF80108968DA83BCBCA04556602847E
:10F500004D66E0FA8DADE18056B35011B6B339FFC8
:10F51000118B6611089B19F8FB04B4B320D7CF8078
:10F52000F45202403CB3018CF3E3D11B30D34EF5CF
:10F530009824823966826F183024FDCC8277183087
:10F5400024186615FC7D607E98B31FA6B307E9B347
:10F5500081FAB3607E98B31FA6B307E9B381FAB30B
:10F56000607E98B31FA6B307E9B381FAB3B0104821
:10F570006CB3CCFB12CC660DF3B303F4B3C0FD3017
:10F58000B33F4CB30FD3B303F5B30C6AF8B106B66F
:10F59000DA70FDC235B308AAF804C6DDDA50FB08FC
:10F5A000824319B2FD604C7E7F04C121B3C9B0FA19
:10F5B000260C190E3FEC7FD8FB12CCB312CC1912DB
:10F5C0007BB19060FFF63207EBB3BAFD6071B619FC
:10F5D00089FE0FC66607EF3630FAF9071F2C308117
:10F5E0000ACF30983F7A17C1FF8CCA0FDDB0493F70
:10F5F0006E60C0FDBB6003F7D69810A6F839FD52C7
:10F60000C0FA8E2DB30256F80111368DE8F938E0B4
:10F61000B5045866024466D8E0FADAE080D5B35003
:10F62000611BB320FE611866B0118919F8B0FB4B5D
:10F630004DB320CF807F5202404B3C0138F3CE3196
:10F64000D1B3D304EF30984830664ECBC80257EBA5
:10F65000CC2CC80953660623B303F4B3C0FD30B302
:10F660003F4CB30FD3B303F4B3C0FD30B33F4CB33F
:10F670000FD3B303F4B3C0FD30B33F4CB30FD5B3D6
:10F68000108243B3CCFB609666606F98B31FA6B33D
:10F6900007E9B381FAB3607E98B31FABB30C55F89A
:10F6A000068DB6DA70FD11ADB30856F80436DAB03F
:10F6B000504AD66289FEC188B3C1FFFB32BAFD044D
:10F6C000B3660395B3046090B3D8D8FB2598B325EF
:10F6D000AC19081216B39007D6D8E3F9FF81FBD610
:10F6E0001705A6D8961FBC30607EF13081FBC67D21
:10F6F0000FFF7FB08163BB6007FEECB1FAF90C2FFE
:10F7000030E53F7830C0FDE33003F5B3106AF863AD
:10F710009F52D8A2FCE2BA02D5F80161128DA8C7A7
:10F720006F13046A66B0028966E0B1FAB5E180AA97
:10F73000B350C236B339FFC2316611611319F8FBF9
:10F740006096B39A20CF80FE520240963C0171F33E
:10F750009CD16366D309DE98B024472D6630AF4A4A
:10F76000E330049FB0CC4EC3E104836602BF8C7DBE
:10F770000FD3B303F4B3C0FD30B33F4CB30FD3B3D7
:10F7800003F4B3C0FD30B33F4CB30FD3B303F4B3B2
:10F79000C0FD30B33F56B310090DB3CCFB825966A0
:10F7A00081BEB3607E98B31FA6B307E9B381FAB3F5
:10F7B000607EADB30C56F80636DAD870FD46B3B5A8
:10F7C0000858F804DBDA50FBB004486C19C9FA1287
:10F7D000CCB312FF7F086090B3D8B2FD1D1E4B6002
:10F7E0007E98B31FA6B307EBB389FE60C4B360FE77
:10F7F00019B0BA23B930406CF7B0D8267C98C1272D
:10F800005615D808597BB52358F8F820E7C8C00327
:10F81000B4016CF748FC1073C8036AF8C090FC6030
:10F8200090B39698B3090BFFDC0638B05C7FC647EF
:10F83000A3FCC18B8C301FFBB1EBB0F8397415C041
:10F84000FBABDF07FF2A98305E5830193F7D9810D8
:10F850006AF8638BD3881DE57D02AAF801C2258D65
:10F86000A88EFA4B04D56602611266E0C723F680C3
:10F870006AE2B0508DB368B0FA8C6658114419D85A
:10F88000F8FB25A6B320CF80BF5202A5403C019CC7
:10F89000F36718D1D9D38277AC98281216668109FC
:10F8A00094F86091F6CC099C30D8FAF912BF326016
:10F8B0006018B31FA6B307E9B381FAB3607E98B3AB
:10F8C0001FA6B307E9B381FAB3607EB6B3DCFB06CB
:10F8D000DA1904D8B3C13019C0DB5AB380ACF89040
:10F8E000090F5A9801C5A9822A6604C12BD7E502DF
:10F8F000ACB3FD12FF32106090B3B0CCB819C0FDAC
:10F90000DBE303F4B3C0FD30B33F4CB30FD3B30319
:10F91000F5B30C6AF8B106B5DA70849A15B608CB5F
:10F92000941B76DA50FB04090D19EBF8824BB3C92E
:10F93000FA6097FB7F080486B3A3FCC0FCF34B0777
:10F94000FFEC7FB2FD09831904BEB0FE7E30193F83
:10F950005BB3BAFD038D1989B0FE260C190E3EEC7F
:10F9600017FAF9125BB3D8FB025B76498107479817
:10F97000981FBC30607EF13081FBC530C67D071F0B
:10F980002C3090167E32C0FD5AB31098F8E7EC5236
:10F990008077B61702ABF80108968DA83BBBE3044D
:10F9A000556602844D66E0FA8E1A47ACB350236C5C
:10F9B000B328FE23166611113619F8FB0969B32026
:10F9C000CFAF80E95202403C016719F3C6D136D36C
:10F9D000609DEB9824048666EBF8C12E6C2A123EDB
:10F9E000CCC1339B30A3FC04836602BF8C7D0FD354
:10F9F000B303F4B3C0FD30B33F4CB30FD3B303F440
:10FA0000B3C0FD30B33F4CB30FD3B303F4B3C0FD69
:10FA100030B33F56B310090DB3CCFB82596681BE9B
:10FA2000B3607E98B31FA6B307E9B381FAB3607ED3
:10FA3000ADB30C56F80636DAD870FD46B3B50858A3
:10FA4000F804DBDA50FBB004486C19EBF8125BB336
:10FA5000C9FA04BFD87F082436B3A3FC07E7984B44
:10FA60003FFE7F90C099301949EDFED883FD98C6BE
:10FA70001FADB389FE8311B383FB19BAFD607E7994
:10FA8000E583FF7617FAF90C5CCA60FFBD4981FE79
:10FA900081CBE6E50717D77F1830131DB160617978
:10FAA000E581FB766007EDD8601FABB31053F81CFF
:10FAB000F56B808EF27D02D5F80161128DA8C76FBB
:10FAC000FA046A66B0028966E0B1FAC34755B350DA
:10FAD000846DB328FE84626611C22619F8FBC12D1D
:10FAE000B32035CF80FD5202402C3C01E3F338D1E6
:10FAF000C6CCD313BD9824608E66609B7660093FA8
:10FB0000CC609D86E1090666057F187D1FA6B307B8
:10FB1000E9B381FAB3607E98B31FA6B307E9B38156
:10FB2000FAB3607E98B31FA6B307E9B381FAB36056
:10FB30007EACB3101216B3CCF1A9607EFD7F81FAC2
:10FB4000B3607E98B31FA6B307E9B381FAB3B0DC04
:10FB50009356FC0CABF8061B6CDA70FD235AB30805
:10FB6000ACF8046DDA50D8FB04243619EBF8092DF3
:10FB7000B3C9FA825FEC3208121BB3A3FC03F3ACE7
:10FB8000FE1FFF7F90604C981924F6FED8C1FECC72
:10FB9000C60FDF6C98B2FD0E2F2D98B09625CC19AC
:10FBA0000E4EEC17FAF918B8CAC1FFBBB181FE03BB
:10FBB00097CCE50E3FEC7F89FE098EB0B130BCE5F5
:10FBC000C0FDBB6003F6EC600FD5B310A9F88E7AC8
:10FBD0006B80C7797D026AF8B001898DA863B7137D
:10FBE000B5045866024466D8E0FAE147AAB350C2A9
:10FBF00036B328FEC2316611611319F8FB6096B363
:10FC00009A20CF80FE520240963C0171F39CD16352
:10FC100066D309DE98B024472A66B0DF4BAB920466
:10FC20008FB0CC4EA31104836602BF8C7D0FD3B37B
:10FC300003F4B3C0FD30B33F4CB30FD3B303F4B3FD
:10FC4000C0FD30B33F4CB30FD3B303F4B3C0FD30AA
:10FC5000B33F56B310090DB3CCFB82596681BEB3D6
:10FC6000607E98B31FA6B307E9B381FAB3607EAD97
:10FC7000B30C56F80636DAD870FD46B3B50858F816
:10FC800004DBDA50FBB004486C19C9FA12CCB31289
:10FC9000FF7F086090B3BBB2EC7F0FDF304B3F4C6F
:10FCA000B30FD5B3DC81C96D2CABFC824BB389FE9D
:10FCB000606698191FBDB16093AD15FAF9824BB318
:10FCC000D8FB604B66C881C1FFACFE0FD5B3BA81CB
:10FCD000C98B478903F7CC981FFB179060726E4958
:10FCE000D8C166ECFA0FDBDA601098F8E7AC6BB3BA
:10FCF00077963002ABF80108968DB93B7BFA045534
:10FD00006602844B66E01C954380AAB350C236B3AA
:10FD10001BFDC2316611611319F8FB6096B39A207E
:10FD2000CF80FE520240963C0171F39CD16366D3B2
:10FD300009DE98B024486C66EBF81279CAC9B0FAAB
:10FD400048FBCC04CDEC49A3FC095FB032ECB3C056
:10FD5000FD30B33F4CB30FD3B303F5B3106090B392
:10FD6000B0CC78BBAD03F4B3C0FD30B33F4CB30FA0
:10FD7000D3B303F4B3C0FD30B33F4CB30FDC30E179
:10FD80003F4CB30FD3B303F5B306608AB6FB04014F
:10FD90008021FD1540E440810801B120D4BF20DB63
:10FDA000BD8027F401FDD0F9604CFF7F15A0FF0254
:10FDB000B4800A50012A40D005A8F33B54D0F3C0C8
:10FDC0003EB80017E002CE22D0D343E0D068D33D46
:10FDD000E05C800BC0F3E4A8D389E6FFF080081054
:10FDE000017F410488001120064483F36F22407E86
:10FDF000F30364800C9001CD38B4D381E00CD0D3F0
:10FE00007BE032400699F31045D3F2140128FFFF3E
:10FE1000C020FFFFFFFFFFFFFFFFFFFFFFFFFFFF10
:10FE2000FFFFFFFFFFFFFFFFFFFFFFFFFFFFFFFFE2
:10FE3000FFFFFFFFFFFFFFFFFFFFFFFFFFFFFFFFD2
:10FE4000FFFFFFFFFFFFFFFFFFFFFFFFFFFFFFFFC2
:10FE5000FFFFFFFFFFFFFFFFFFFFFFFFFFFFFFFFB2
:10FE6000FFFFFFFFFFFFFFFFFFFFFFFFFFFFFFFFA2
:10FE7000FFFFFFFFFFFFFFFFFFFFFFFFFFFFFFFF92
:10FE8000FFFFFFFFFFFFFFFFFFFFFFFFFFFFFFFF82
:10FE9000FFFFFFFFFFFFFFFFFFFFFFFFFFFFFFFF72
:10FEA000FFFFFFFFFFFFFFFFFFFFFFFFFFFFFFFF62
:10FEB000FFFFFFFFFFFFFFFFFFFFFFFFFFFFFFFF52
:10FEC000FFFFFFFFFFFFFFFFFFFFFFFFFFFFFFFF42
:10FED000FFFFFFFFFFFFFFFFFFFFFFFFFFFFFFFF32
:10FEE000FFFFFFFFFFFFFFFFFFFFFFFFFFFFFFFF22
:10FEF000FFFFFFFFFFFFFFFFFFFFFFFFFFFFFFFF12
:10FF0000FFFFFFFFFFFFFFFFFFFFFFFFFFFFFFFF01
:10FF1000FFFFFFFFFFFFFFFFFFFFFFFFFFFFFFFFF1
:10FF2000FFFFFFFFFFFFFFFFFFFFFFFFFFFFFFFFE1
:10FF3000FFFFFFFFFFFFFFFFFFFFFFFFFFFFFFFFD1
:10FF4000FFFFFFFFFFFFFFFFFFFFFFFFFFFFFFFFC1
:10FF5000FFFFFFFFFFFFFFFFFFFFFFFFFFFFFFFFB1
:10FF6000FFFFFFFFFFFFFFFFFFFFFFFFFFFFFFFFA1
:10FF7000FFFFFFFFFFFFFFFFFFFFFFFFFFFFFFFF91
:10FF8000FFFFFFFFFFFFFFFFFFFFFFFFFFFFFFFF81
:10FF9000FFFFFFFFFFFFFFFFFFFFFFFFFFFFFFFF71
:10FFA000FFFFFFFFFFFFFFFFFFFFFFFFFFFFFFFF61
:10FFB000FFFFFFFFFFFFFFFFFFFFFFFFFFFFFFFF51
:10FFC000FFFFFFFFFFFFFFFFFFFFFFFFFFFFFFFF41
:10FFD000FFFFFFFFFFFFFFFFFFFFFFFFFFFFFFFF31
:10FFE000FFFFFFFFFFFFFFFFFFFFFFFFFFFFFFFF21
:10FFF0005A5845766F415652426F6F749F958CC226
:00000001FF
